:020000040800F2
:1000000000000220E9320B086D330B08158006084A
:100010006D330B086D330B086D330B0800000000C7
:100020000000000000000000000000006D330B081D
:100030006D330B08000000006D330B087548050890
:100040006D330B086D330B086D330B086D330B08E4
:100050006D330B086D330B08190E05081D0E0508CE
:10006000210E0508250E0508290E0508F93F04088C
:100070000D400408214004083540040849400408A4
:100080005D400408714004086D330B086D330B08A4
:100090006D330B086D330B086D330B082D0E0508FF
:1000A0006D330B086D330B086D330B08214A0408C0
:1000B000354A0408494A04085D4A04089132040894
:1000C00085320408C5320408B93204086D330B08C0
:1000D0006D330B08815404088D54040899540408A6
:1000E000310E05086D330B0800000000994A040822
:1000F000E94A0408114B0408854A040885400408AD
:100100006D330B0805620408714A04086D330B084F
:10011000A55404086D330B086D330B089D74040857
:1001200099400408AD400408C1400408D5400408C3
:10013000E94004086D330B086D330B086D330B0871
:1001400000000000000000000000000000000000AF
:10015000FD4004081141040825410408B154040875
:10016000F9320408ED3204086D330B086D330B08C7
:100170006D330B086D330B086D330B080000000066
:100180006D330B086D330B08BD540408C9540408C3
:100190006D330B086D330B086D330B086D330B0893
:1001A0006D330B086D330B086D330B086D330B0883
:1001B0006D330B086D330B086D330B086D330B0873
:1001C0006D330B086D330B086D330B086D330B0863
:1001D0006D330B08216304086D330B086D330B0876
:1001E0006D330B086D330B086D330B086D330B0843
:1001F0006D330B086D330B086D330B086D330B0833
:100200006D330B086D330B086D330B086D330B0822
:10021000AD4A0408C14A0408D54A04086D330B08E6
:100220006D330B086D330B086D330B0800000000B5
:10023000096204086D330B08000000006D330B08E1
:100240006D330B086D330B086D330B086D330B08E2
:100250006D330B086D330B086D330B086D330B08D2
:100260006D330B086D330B086D330B086D330B08C2
:100270006D330B086D330B086D330B080000000065
:100280006D330B08000000006D330B080000000008
:08029000000000006D330B08B3
:08029800E0220B000100000050
:1002A000288901240201000002012C004889012450
:1002B0000202000002012C0068890124020A0000E9
:1002C00002012C00888901240203000004012C0093
:1002D000A88901240208000004012C00C889012417
:1002E000010B000000017700E8890124010C0000E7
:1002F00000017600088A0124011000000001760048
:10030000288A0124010D010000017700488A012498
:100310000112000000017600688A01240114000027
:1003200000001E00888A0124011A000000000D0050
:10033000A88A0124011B000000002C00C88A0124A7
:100340000115000000000C00E88A012401160000DD
:1003500000000C00088B0124011C000000000E00AE
:10036000288B0124011D000000001E00488B012481
:100370000117000000000C00688B01240118000028
:1003800000000E00888B01240119000000000C0001
:10039000A88B0124011F000000000C00C88B012461
:1003A0000120000000000C00E88B0124012901005D
:1003B00000011800088C0124012100000001480000
:1003C000288C01240122000000014900488C0124EE
:1003D0000123000000014A00688C01240124000070
:1003E00000014B00888C01240125000000014C0015
:1003F000A88C01240126000000014D00C88C0124B6
:100400000127000000014E00E88C012401280000B3
:1004100000014F00088D0124012C0000000029007C
:10042000288D0124012D010000002900488D0124A0
:10043000012E010000007000688D0124012F0100D1
:1004400000005200888D01240130010000012800C5
:10045000A88D01240131010000012800C88D01246C
:100460000134000000003C00E88D01240137000049
:040470000000200068
:020000040804EE
:10000000836B5A6D12F0500F5A6D1AD1196842F471
:1000100000725A650A6812F0080FCA6816D012F406
:10002000406F15D1CA68920412D45A6D22F48072BE
:100030005A655A6DD1040BD45A6D42F001025A65CB
:100040007047D20604D4DB6CDB6C18479007ECD009
:10005000704700BF704700BF836B5A6D42F040028B
:100060005A659A6D42F004029A65704702685549D4
:1000700038B5554B554D564CAA4218BF9A420CBF45
:10008000012300238A4208BF43F001033031A2421A
:1000900008BF43F0010330348A4208BF43F0010334
:1000A0003031A24208BF43F0010330348A4208BF16
:1000B00043F0010301F55C71A24208BF43F0010364
:1000C00004F55C748A4208BF43F001033031A24258
:1000D00008BF43F0010330348A4208BF43F00103F4
:1000E0003031A24208BF43F0010330348A4208BFD6
:1000F00043F001033031A24208BF43F001038A42BA
:1001000008BF43F0010313B9324B9A4208D10423CC
:1001100080F83530136823F001031360002038BDE8
:100120002D4B2E4D1168AA4218BF9A422C4C21F03B
:100130000E0105F13C050CBF012300231160A24212
:1001400008BF43F0010311682834AA4208BF43F0F6
:10015000010321F00101A24208BF43F0010314345E
:100160001160A24208BF43F001031E498A4208BF42
:1001700043F0010313B91C4B9A4217D10123856D3B
:10018000D0E91714226801F01F0122F480728B401D
:1001900022606B60C36ED0E91921516033B11A68D7
:1001A000D0E91C1422F480721A604C6000210122F4
:1001B000036D80F8341080F83520002BAED09847BE
:1001C000ACE700BF4000024010000240280002409F
:1001D00058000240B80402401C5402580854025807
:1001E000305402588054025894540258002280F827
:1001F000422090F84130292B04D090F841302A2B2E
:1002000018D070474FF0280C2123016880F841C0B6
:10021000036390F8413003EA0C0363450B6814BF95
:100220006FF0F20C6FF0420C03EA0C030B6080F8E5
:10023000402070474FF0280C2223016880F841C00D
:10024000036390F8413003EA0C0363450B6814BF65
:100250006FF0F40C6FF0440C03EA0C030B6080F8B1
:10026000402070470023202210B4174C4363C4621F
:10027000036380F8412080F842304B07026811D5B3
:10028000526A436A1A70436A028D013343624AB16B
:10029000438D013A013B02859BB24385436C43F099
:1002A000040343640368102490F84120002190F86F
:1002B00041201A6822F0FE021A60DC615DF8044BEE
:1002C00080F84010704700BF0000FFFF70B50023AA
:1002D00090F84120424D044680F84230283AC562E9
:1002E0004385022A406C236840EA0100606439D8E3
:1002F00094F84110282094F8412001F0280102F0E0
:100300002802282914BFF6214621282A1A680CBF82
:10031000C9436FF0F6010A4032491A60002284F89E
:10032000410022631A68616312F4804231D01A6876
:10033000A06B22F480421A6098B100222A4B036518
:1003400084F8402090F83520022A3CD08022426573
:10035000BDE87040184794F84130602B3AD084F8DB
:10036000401070BD94F8412094F841201A6822F0A2
:10037000FE021A6094F84120602A02D0202284F8FC
:1003800041200022114622631A68616312F4804200
:10039000CDD1196811F40041DDD01968E06B21F46A
:1003A000004119600028DCD00F4B036584F8402021
:1003B00090F83520022AC9D1FFF758FE0028D0D086
:1003C000E06B036DC4E7FFF751FE0028C9D0A06BB6
:1003D000036DBDE7202384F8401084F8413070BDE0
:1003E0000000FFFF65040408F106040803689A6929
:1003F000196810B4D40528D50C0606D4416C11F048
:100400000B0F1FD15DF8044B7047416C4FF48074A3
:1004100041F0010141645105DC6120D5416C4FF48C
:100420008064920541F008014164DC61E6D5426CCC
:100430004FF4007142F002024264D961416C11F044
:100440000B0FDFD05DF8044B40E7540502D50906D9
:10045000E4D4D3E79405D1D50906E8D4CEE79205D4
:10046000E5D4CBE72DE9F84390F84030C76A012B7B
:1004700000F0D780012304460D46164680F8403030
:10048000880601D591065FD4EA0621D5F3061FD56B
:10049000638D9BB2002B40F0AA8094F84130B7F1F5
:1004A000007FDBB202D1282B00F0198194F8413093
:1004B00017F5803F2268DBB202D0292B00F0D380F1
:1004C0001023D3610023184684F84030BDE8F88338
:1004D0006A071BD4280702D5310700F19880AA07C4
:1004E000F0D5B307EED5638D9BB2002B00F0A4804E
:1004F000616A236811F8010B228D9862638D013ABD
:100500006162013B22859BB26385DBE77307E1D51E
:10051000638D9BB26BB12268636A526A1A70638DF5
:10052000616A228D013B0131013A9BB261622285F1
:100530006385638D17F5803F9BB2C3D0002BC1D17B
:100540002046FFF753FEBDE723682022664819685E
:10055000DA6194F8412094F841201A6822F0FE02F2
:100560001A605A6842F400425A605A6802405A605F
:100570009A69920701D500229A629A69D00703D43A
:100580009A6942F001029A614A044DD5A26B1AB1F0
:1005900011684A6892B2628569074BD55A6A25F09C
:1005A0000409636A1A70636A01336362238D002B46
:1005B00052D1638D9BB21BB1636C43F0040363643F
:1005C0000023236384F84230D4F844806363B8F195
:1005D000000F58D1E36ADFF814914B4531D194F8FC
:1005E0004130202384F8408084F841304CE7236870
:1005F0001022DA61636C43F00403636437F08073A4
:100600007FF460AF616C2046FFF760FE5AE794F814
:100610004130226803F02803282B42D00823D361FD
:1006200050E70220BDE8F8830804B5D5E26B002A44
:10063000AED1B1E7A946BCE737F080737FF442AF93
:100640007EE72046FFF7D2FD2023C4F82C9084F8E3
:10065000408084F8413017E7013B2385638D013BDF
:100660009BB26385A5E71023D3619369980701D5F1
:10067000002393629369D9073FF562AF936943F012
:10068000010393615CE7616C2046FFF71FFE94F85D
:100690004130282B7FF4F8AE49462046FFF7E2FDB3
:1006A000F2E6E1689369022990699368D56811D1EF
:1006B000C3F3C21383EA104313F006030AD1A16CFB
:1006C0000131A164A16C02297FF4FCAE0821A3646E
:1006D000D161F7E6136823F0B8031360F2E6294608
:1006E0002046FFF7BFFDEDE600E800FE0000FFFF3B
:1006F000836B0022D3E90E0102650A6593F841205D
:10070000602A02D1202283F841207047026870B429
:10071000D4072DD597490B69896A03F03803102B4C
:1007200000F0F180182B00F0E9804368B3F5803FBA
:1007300000F05581002B00F05B81B3F5A02F8D4BAD
:10074000196800F02C8221F480311960196821F4B5
:1007500080211960884B41F2883C864C1D6804E07A
:100760001968491B614500F2408121688E03F7D565
:1007700091072DD57F490B69896A13F0380300F082
:10078000A680182B00F0A080C3687A4C002B00F0E4
:100790006381216821F019011943774B21601D689D
:1007A00004E01968491B022900F21F8121684907EA
:1007B000F7D5724B01691D6841F20303B3EB154F86
:1007C000636880F0958023F0FE4343EA0163636031
:1007D000D5064CD4150713D54369664C002B00F0A1
:1007E0009E80616F644B41F0010161671D6804E008
:1007F0001968491B022900F2F880616F8907F7D553
:10080000940613D583695B4C002B00F007812168A7
:10081000594B41F4805121601D6804E01968491B5F
:10082000022900F2E28021688904F7D5540700F11B
:10083000A780426AC2B14F490B6903F03803182BF5
:1008400000F07F81022A0A684B4B22F080720A6016
:1008500000F01881186804E01A68121A022A00F2DF
:10086000C4800A689201F7D4002070BC70474149E7
:100870000B69896A03F03803082B63D0182B5DD00D
:10088000C3693C4C002B00F0D88021683A4B41F002
:10089000800121601D6804E01968491B022900F2EB
:1008A000A4802168C905F7D5344B056A196841F25F
:1008B0000303B3EB114FC0F09081636823F0F8435A
:1008C00043EA8563636085E78D077FF45DAF294B5D
:1008D0001B685C0701D5C368F3B1284C41F20303E0
:1008E00001692468B3EB144F224C6368FFF46BAFCB
:1008F00023F47C3343EA0133636069E701F00301C9
:1009000002297FF412AF1B4B1B689B037FF530AFAE
:100910004368002B7FF42CAF012070BC7047616FDF
:10092000154B21F0010161671D6803E01968491B3F
:1009300002295AD8616F8E07F8D461E701F00301EC
:1009400001299DD10B4B1B68DC0502D5C369802BA7
:10095000E2D10A4941F20303046A0968B3EB114F7B
:100960000449C0F088804B6823F0F84343EA84636D
:100970004B602FE700440258A02B00240010005CBD
:100980009C499D4B0A6842F480720A601C6803E02F
:100990001A68121B642A28D80A68D505F8D5826817
:1009A000012A00F02181002A00F00181052A934AE2
:1009B000116F00F0278121F001011167116F21F003
:1009C000040111671D6841F288348C4903E01A68FC
:1009D000521BA24209D80A6F9207F8D529E7874926
:1009E0000B6843F480330B60B4E6032070BC70479F
:1009F000824C41F28835804B216821F4803121609E
:100A0000216821F4802121601E6803E01968891B98
:100A1000A942EAD821688903F8D4A9E62168764B6F
:100A200021F4805121601D6803E01968491B0229E7
:100A3000DBD821688E04F8D4F8E621686E4B21F0EB
:100A4000800121601D6803E01968491B0229CCD888
:100A50002168CE05F8D4BDE62168674B21F001017D
:100A600021601D6803E01968491B0229BDD821686F
:100A70004E07F8D4ACE6CB6823F07C5343EA04631A
:100A8000CB60A7E61C6803E01A68121B022AACD8E8
:100A90000A689501F8D48C6A594A2240846A224334
:100AA000C46A42EA04128A62D0E90D24013A013C88
:100AB0005202240492B204F4FE042243046B013C6B
:100AC000C4F308042243C46B013C240604F0FE4432
:100AD00022430A63CA6A22F00102CA624A6B846C2A
:100AE0006FF3CF0242EAC4024A63CA6A046C22F07E
:100AF0000C022243414CCA62CA6A406C22F00202D4
:100B00000243CA62CA6A42F48032CA62CA6A42F4C2
:100B10000032CA62CA6A42F48022CA62CA6A42F0D9
:100B20000102CA620A6842F080720A60196804E031
:100B30001A68521A022A3FF658AF22689001F7D578
:100B400092E6012A8C6A0B6B3FF4E6AE04F00302D6
:100B5000816A8A427FF4E0AEC4F30514C26A94420B
:100B60007FF4DAAE026BC3F30801013A91427FF4DD
:100B7000D3AE426BC3F34621013A91427FF4CCAE2F
:100B8000826BC3F30641013A91427FF4C5AEC26B5A
:100B9000C3F30663013A981A18BF0120BDE641F479
:100BA00080211960196841F480311960D2E5134938
:100BB00041F288350A6F22F001020A670A6F22F0BB
:100BC00004020A671C6804E01A68121BAA423FF676
:100BD0000CAF0A6F9607F7D42BE6E36823F07C533B
:100BE00043EA0563E360F5E504490A6F42F0010258
:100BF0000A67E7E600480258A02B00240044025888
:100C00000CFCFFFF41F004011167116F41F001017D
:100C10001167D7E6334B30B4996A9C6ADD6A14F4E5
:100C20007C7F5A6BC4F3051036D0C2F3CC0205F0BA
:100C3000010501F0030107EE900A05FB02F201290C
:100C4000B8EEE77A06EE902AFAEEE96A02D00229B7
:100C500042D019B3DFED247A87EE876A1B6BC3F3AA
:100C6000080307EE903AF7EE005AF8EEE77A77EECF
:100C7000A67A77EEA57A67EE867A1A4B1B6BC3F3DA
:100C80004623013307EE103AF8EEC76A87EEA67ADC
:100C9000FCEEC77A17EE900A30BC70471A689206CD
:100CA0001DD51968F7EE005A104A1B6BC1F3C1013C
:100CB000C3F30803CA4007EE903A06EE102AF8EE96
:100CC000E77AB8EEC66A77EEA66AC6EE077A36EE1F
:100CD000A57A67EE877AD0E7DFED057ABCE7DFED2E
:100CE000057AB9E7004402580024744A0090D00302
:100CF00020BCBE4B0024744CF0B5344AB0F1804F98
:100D0000334CA0EB02020368A0EB040E4F69B2FA69
:100D100082F28E68BEFA8EFE0D684FEA52124FEADA
:100D20005E1E20D0FAB9DFF8B4C0604532D00CF5B1
:100D3000806C60452ED00CF5806C604513D0BEF100
:100D4000000F10D1234C244A904218BFA04225D056
:100D500002F58062904221D023F080033B43036080
:100D6000C662856213E04C6823F070032343CC68AD
:100D700023F44073234323F080033B430360C662A4
:100D8000856212B9BEF1000F12D00B690363012313
:100D90004361F0BD23F070034A681343CA6823F42B
:100DA0004073134323F080033B430360C6628562B4
:100DB000084A094B984218BF9042E6D003F5806379
:100DC0009842E2D001234361F0BD00BF0000014022
:100DD0000004014000400140004401400004004084
:100DE000836ADA0710B406D50168C46A4A6822F437
:100DF000003222434A609C0706D50168046B4A68AA
:100E000022F4803222434A60590706D50168446BB8
:100E10004A6822F4802222434A601A0706D50168F4
:100E2000846B4A6822F4004222434A60DC0606D5FD
:100E30000168C46B8A6822F4805222438A60990652
:100E400006D50168046C8A6822F4005222438A6045
:100E50005A060AD50168446C4A68B4F5801F22F42A
:100E6000801242EA04024A600BD01B0606D50268D3
:100E7000C16C536823F400230B4353605DF8044BAB
:100E800070474A68846C22F4C00222434A60ECE74F
:100E90000022836BA3F85E20A3F85620704700BFA2
:100EA000124B41F2883C124A01461B68A2FB032305
:100EB0005B0A0CFB03F33BB14A6B12F0450F01D008
:100EC000920404D5013BF7D14FF0004070474B6BC3
:100ED0005B0707D4486B10F0010014BF0123054BDA
:100EE0008B637047042318468B637047000000240F
:100EF000D34D6210C5002000036942681F2B70B4F7
:100F000030D9A3F1200520215468A940214227D0DF
:100F10008169087C022835D048681F2BC9681B4DA1
:100F20004E680169C1F30324194951F8244015F8AA
:100F300004C0056856F80C4024F0010446F80C4043
:100F4000407901EB4001088CE96800F4F05021EA97
:100F50000001E96010D9A3F1200120238B40D36068
:100F600070BC70472021146899402142F8D08169F3
:100F7000087C0228D0D105E0202101FA03F370BCDF
:100F80009360704700200874C6E700BF6CBC0B0874
:100F9000D0BA0B08436BDA692DE9F0419706044695
:100FA00013D5586AE36AC0B2002B79D0216B9847F9
:100FB000636B1A6822F480721A609A6822F0010248
:100FC0009A609A6942F008029A61DA69D60701D5F7
:100FD00001221A62DA69950701D502221A62DA69DA
:100FE000500701D504221A62DA69110701D50822D7
:100FF0001A62DA69120612D5D4F8B420212A0ED06A
:10100000D4E909128A4257D0A169895C0132C9B278
:1010100099622169B2FBF1F001FB1022A262DA6948
:10102000570601D4BDE8F081DA6940F60F0C1D685F
:1010300004F1340012EA0C0F996823D0724E0E406E
:1010400042D1724F3D4240F0CD80D60202D54F02D0
:1010500000F1D080160606D501F4000105F08006E7
:101060000E4340F0BA805106DCD56A06DAD51A681C
:101070002020002122F040021A60C4F8B400C4F815
:10108000A410CFE79606E0D505F0200601F08057C2
:101090003E43DAD0D4F8A030002B40F08E80C1E778
:1010A000E3696269D054E369E2680133B3FBF2F1AA
:1010B00002FB1133E3617BE70022A4F88A201A685F
:1010C00022F080021A60AAE7D70709D5EF0507D5F5
:1010D00001271F62D4F8BC7047F00107C4F8BC7048
:1010E00097076DD4570709D5CF0707D504271F6287
:1010F000D4F8BC7047F00207C4F8BC7017070BD5D2
:1011000005F02007374307D008261E62D4F8BC60DC
:1011100046F00806C4F8BC6017050AD56E0108D56C
:101120004FF400661E62D4F8BC6046F02006C4F896
:10113000BC60D4F8BC60002E3FF474AF92060AD5B0
:1011400005F0200501F080510D4304D0D4F8A02013
:101150000AB19047636BD4F8BC109A6801F028017B
:1011600002F040020A434CD019682020284A21F49A
:101170009071196099680A4000219A60C4F8B8001B
:101180009A68C4F8A01057067FF54CAF9A68D4F857
:10119000AC0022F040029A6000283FF443AF90F880
:1011A00035201C4B022A036528D1FEF75FFF00287B
:1011B0003FF438AFD4F8AC00036DBDE8F0411847F8
:1011C000CF079BD502271F62D4F8BC7047F00407F5
:1011D000C4F8BC70570791D588E7D4F8A430002B29
:1011E000EBD11FE7D70789D5EF053FF571AF97071B
:1011F00084D477E74FF480121A6213E780224265A5
:10120000DBE7C4F8BC200DE701000010200100045A
:10121000FEFFFFEF910E0408D0E907239A423CBF7E
:10122000C1685218D01A7047D0E9092300699A4260
:1012300038BF12180138D31AC01A7047D0E9090212
:10124000101AB0FA80F04009704700BF016A0346E7
:1012500040694A1C405CD9688A4228BF00221A6251
:10126000704700BF436A826910B4D154436A416B2E
:10127000046901330A68A34228BF00235DF8044BC8
:1012800042F0800243620A60704700BF436BD86936
:1012900010F0100002D0102201201A62704700BF27
:1012A000B24BD3E9011270B58C0F93F88850100E31
:1012B000C2F3072C83F83040C1F383640001012D91
:1012C00083F83140C1F3016483F83240C1F307442D
:1012D00083F83340C1F30724C9B283F83440C2F322
:1012E000035483F83510D886C2F3C030D98E89B242
:1012F00041EA0401C2F30344D986C2F3403183F8C2
:101300003840C2F3803483F839004FF0000083F88E
:101310003A4083F83B10C2F3003183F83C10D9689F
:1013200083F83D0040F2D480022D00F0B0802A20E6
:101330004FEA4C0C83F84940C1F3C01201F07F0121
:101340000CF07E0C83F84AC04FF0010C93F84A4031
:1013500014431A6983F84A40D40F83F84B10910D57
:1013600083F84C40C2F3417401F00C01C2F3815583
:1013700083F84D40C2F3826483F84E4083F84F10E7
:1013800093F84F105C69294383F84F10C2F3405122
:1013900083F85010002183F85110C2F3004183F804
:1013A0005210C2F3C03183F85310C2F3803183F876
:1013B0005410C2F3403183F85510C2F3003183F862
:1013C0005610C2F3812183F85710C2F30121C2F3F2
:1013D000460283F85810C4F3074183F85920220EBF
:1013E000090283F85AC083F85C20C4F30722A3F8EB
:1013F0005E102406B3F85E1089B21143A3F85E10A4
:1014000099691C660C0E1A6E42EA04421A660A0AB0
:101410001C6E02F47F422243C1F30724C9B21A664C
:101420001D6EDA692C431C6683F86410110E83F874
:101430006510110C0906996611029C6E0A4601F4AA
:101440007F01214392B21C6A9966996E0A439A669B
:10145000C4F30352996E41EA1461996693F86C10D3
:101460001143C4F3072283F86C10210A01F4706160
:10147000A3F86E10B3F86E1089B21143C4F346029C
:10148000A3F86E1083F8702083F871C070BD120449
:10149000C1F3072C0D0E02F47C121A64C1F307424B
:1014A0001C6C44EA05241C641C6C22434FF4007439
:1014B0001A641A6CC3F88040013240F10004A4029F
:1014C00044EA92549202DC67C1F380349A672FE7B2
:1014D0004FEA8C2CC1F3C26594000CF44062C1F356
:1014E000072C04F47F741A641A6C1443CA0B1C642E
:1014F00002F006021C6C44EA91741C64C1F302649D
:1015000083F84450012583F84540C1F3425483F8E1
:101510004640C1F3824483F84740C1F3C03483F8A6
:10152000482093F84820224383F848201C6C93F805
:10153000482093F83860023205FA02F2B540D61717
:10154000A2FB052EC3F8805005FB06EE04FB0EEE51
:101550000134A2FB0424A644520AC1F3803442EAB7
:10156000CE529A674FEA5E22DA67E1E6A02B0024AA
:10157000704700BF704700BF014BD3F88C00704725
:10158000A02B0024044B93F82C03A0F10300B0FA25
:1015900080F04009704700BFA02B0024012380F891
:1015A00049307047064AD2E9D932581E9342A0EB1F
:1015B00002008CBF0023012300EB0330704700BF03
:1015C000A02B002401F00F01D0F8D022C1EBC10103
:1015D00002EB8102D0E9AE30D2F8142203F5037198
:1015E00010B5C468D3F80402C3F80C22A047002049
:1015F00010BD00BFD0F8BC3283B110B5D0F8B842EE
:1016000094F80002FF2807D09B68214694F8012235
:101610009847FF2384F80032002010BD0020704757
:101620000346432201481A80704700BF040000248B
:101630000346432201481A80704700BF4800002437
:101640000346432201481A80704700BF8C000024E3
:1016500003460A2201481A80704700BFD0000024C8
:10166000064B4FF0120C064AA3F11400526DA1F87C
:1016700000C0022A18BF1846704700BFF0000024BF
:1016800000400058042301480B80704704010024E7
:101690001D48D0F80038D0F8082830B59B184FF016
:1016A0001A040C8001D1194830BD184A0024D0F822
:1016B000040802F1100511464FEA137EB3F1204FE2
:1016C000CC7001F102010EF1370C38BF0EF1300C75
:1016D0008D424FEA031381F800C0EDD102F10805F5
:1016E0000024010FB0F1204FD47402F1020201F185
:1016F000370338BF01F1300395424FEA00101374ED
:10170000EFD1024830BD00BF00E0F11F0801002406
:1017100000207047212808B527D0222818D020287B
:1017200014D199B1072A11D1184A194B0868B1F898
:1017300004C0D2F86C238979C3F82401A3F828C126
:1017400083F82A1112B1014600209047002008BDFD
:101750000029FBD0022AF9D10C4BD3F87033002BAF
:10176000F4D0098800209847F0E70029EED0072A36
:10177000ECD1074BD3F82401B3F8282193F82A3190
:10178000086000208A808B7108BD00BFA02B002458
:1017900000000024034B93F89803003818BF012081
:1017A000704700BFA02B0024304B0021304A1B683B
:1017B0003048A2FB032310B5DB0C2F4C82B0013B59
:1017C000C4F8DC13C4F8D41342F20F7194F809245E
:1017D000C4F8CC03C4F8D813C4F8D033002A3FD0DF
:1017E00002232649234884F80934FFF785FA244B5D
:1017F00001220621372084F80924D3F8E82042F09A
:101800002002C3F8E820D3F8E83003F02003019366
:10181000019B6BF02FFED4F8CC334FF40000194934
:10182000194A4860D96841F00101D96099680A40B5
:10183000062A06D0B2F5803F03D01A6842F00102B2
:101840001A600020D4F848331049114AC3F8100236
:10185000C4F87003C4F86C03C3E9812102B010BD61
:1018600002F0FF0084F80804BAE700BF000000247B
:1018700083DE1B4300140040A02B0024702F0024A3
:101880000044025800E100E0070001001C4A002467
:101890001C3A0024F8B51C4F03460846D7F84823E5
:1018A000D2F814120029FBD160B31918DFF85CC01C
:1018B000013B0139D7E9D95213F8016F541C0CF8D8
:1018C0000260C4F30B02AA42A5EB020434BF002657
:1018D000012604EB0634012C10D1C7F8682313F05D
:1018E0001BF804460D4613F017F8001B61EB0501C9
:1018F000B0F57A7F71F10001F5D3F0E79942DBD1C1
:10190000C7F86823F8BD00BFA02B00241C4A0024A0
:10191000F8B50C4E96F82C33032B00D0F8BD0D46CD
:101920001446D6F80C7408E0FFF7B4FFD6F80C3470
:10193000241A0544DB1B322BF0D8002C2146284604
:10194000F2DCF8BDA02B0024F8B590F848305D1CFF
:101950000344EDB280F8485083F8341090F84930D1
:1019600053B1132D07D9002380F848300E4F97F854
:101970002C33032B05D0F8BD80F84830002DF5D16D
:10198000F8BDD7F80C6400F1340429462046FFF76F
:1019900081FFD7F80C342D1A04449B1B322BEAD854
:1019A000002DF2D1F8BD00BFA02B0024F8B5002314
:1019B00090F84850A0F8483005B9F8BD0B4F97F89B
:1019C0002C33032BF9D1D7F80C6400F134042946E9
:1019D0002046FFF75FFFD7F80C342D1A04449B1BF9
:1019E000322BEAD8002DF2D1F8BD00BFA02B002485
:1019F0002DE9F047046982B0C3681C4046D0814697
:101A000088464FF0004501F1500701F13806B4FA5D
:101A100084F325FA03F21B3BD2431440C9F810208B
:101A2000B8F1000F5FD0042B2ED8DFE803F0524846
:101A30003D320300D8F81030D9F82CA033B19B68A0
:101A400023B11FFA8AF108F108009847D8F8283026
:101A500033B19B6823B11FFA8AF108F1200098473F
:101A6000D8F8403033B19B6823B11FFA8AF108F1EE
:101A700038009847D8F8583033B19B6823B11FFA23
:101A80008AF108F150009847002CC0D102B0BDE89F
:101A9000F087D8F8103008F10800D9F834105B68E6
:101AA0009847002CB3D1F1E7D8F8283008F120008E
:101AB000D9F838105B689847002CA8D1E6E7D8F829
:101AC00040303046D9F83C105B689847002C9ED1D6
:101AD000DCE7D8F858303846D9F840105B689847AA
:101AE000002C94D1D2E7042B07D8DFE803F01903C8
:101AF000140F0A00D9F83C300193019B002C86D1C9
:101B0000C4E7D9F82C300193019BF7E7D9F83430BA
:101B10000193019BF2E7D9F838300193019BEDE77F
:101B2000D9F840300193019BE8E700BF234938B55D
:101B3000D1F810346BB1D1F88C20002AFAD0013AD8
:101B400013F8014BC1F88C20C1F8103412B12046B3
:101B500038BDFEE7D1F84833002BF8D091F8A0004B
:101B6000D3F80452D1F86033A8B91A690121C3F837
:101B700030024FF40070012AA3F81812C3F824525F
:101B800003F50671C3F82C0214D01868D2B26FF0B6
:101B9000B9F8204638BDC3F8302201211A69402027
:101BA000A3F8181203F50671012AC3F82452C3F8EA
:101BB0002C02EAD1C3F82852E7E700BFA02B00248B
:101BC000D0F8B822002A3DD001EB810300EB83035B
:101BD00070B5DC69D0F8D05224B90023C2F81432B1
:101BE000002070BDC1EBC10C05EB8C0CDCF844602F
:101BF000B4FBF6FC06FB1C44002CEED101F07F0286
:101C0000DC6101F00F031C2102EB820201FB035196
:101C100000EB8200C3EBC3023C31C46105EB8200E0
:101C20000122846480F83C3080F83D20C0E91444EF
:101C30002A69012AD2B208BFC464286823B96FF0A8
:101C400071F9CDE7022070476FF05CF8C8E700BF7C
:101C5000184B0A68C3F81004C3F88C200AB100209E
:101C60007047D3F848130029F9D010B593F8A000B5
:101C7000D1F80442D3F86033A0B140200121C3F869
:101C80002442C3E98B021A691868012AA3F81812C2
:101C9000D2B203F5067108BFC3F828426FF032F8DC
:101CA000002010BD4FF400720121C3F82442C3E9A3
:101CB0008B20E8E7A02B002470B5037C0446D0F805
:101CC000D002002B45D14FF40073022281216EF027
:101CD00019FF01214FF400730222D4F8D002E1620F
:101CE0006EF010FF0126082303228221D4F8D002CF
:101CF000C4F86C616EF006FF4FF40770266478F04C
:101D0000BDFC0546C4F8B802002842D0D4F8BC3265
:101D10001B6898470022217CC5F81422D4F8D032E1
:101D2000D5F80402C5F8182209B3C3F830224024BC
:101D30001A6903F50671C3F82402012AA3F8186290
:101D4000C3F82C4222D01868D2B26EF0DBFF00201C
:101D500070BD4023022281216EF0D4FE0121402378
:101D60000222D4F8D002E1626EF0CCFEBAE71A6922
:101D70004FF40074C3F8301203F50671B242C3F891
:101D80002402A3F81862C3F82C42DCD1C3F828025D
:101D9000D9E7304670BD00BF70B5D0F8D05240F2E0
:101DA0000112044695F8BC33A5F85820012B09D040
:101DB00001222868114685F8BC236FF08FF90023B3
:101DC00085F8BC33D4F8D05200260121E66295F89C
:101DD000BC33A5F818128B4207D03246286885F824
:101DE000BC136FF07BF985F8BC63D4F8D0520026A1
:101DF0004FF48172C4F86C6195F8BC33A5F8742077
:101E0000012B08D001220221286885F8BC236FF03D
:101E100065F985F8BC630025D4F8B83225644BB168
:101E2000D4F8BC325B689847D4F8B80278F02EFC3E
:101E3000C4F8B852002070BD2DE9F0410B7882B093
:101E400000260D4613F060070446D0F8B8828DF8DE
:101E50000560ADF8066035D0202F0DD08021D4F874
:101E6000D0026EF0F5FE0021D4F8D0026EF0F0FE44
:101E7000022002B0BDE8F081CA884878002A37D035
:101E80001B064FD5D4F8BC3241469B6898470223C5
:101E9000EA884FF48071C4F89432D4F8D032C4E99F
:101EA00007221A651A69998703F13C01012AC3F8D0
:101EB00048805E6501D1C3F84C80D2B218686FF0DB
:101EC00031F819E04D780A2D1DD00B2D16D0002DBC
:101ED000C4D190F89C32D0F8D002032B55D0802189
:101EE0006EF0B6FE2946D4F8D0026EF0B1FEBFE720
:101EF000D4F8BC329B6898470020BAE790F89C322F
:101F0000032BF9D0AAE790F89C32D0F8D002032B2B
:101F100023D080216EF09CFE3946D4F8D0026EF0BA
:101F200097FEA5E7032388F8000288F80122C4F889
:101F30009432D4F8D032C4E95722C3F8102203F502
:101F4000FE711A69C3F80882012AC3F81462A3F863
:101F5000FC6108BFC3F80C82AFE7022201234FF4F3
:101F60008071C4F894220269E3612362012A036547
:101F70000DF10503818700F13C018364476516D0AC
:101F8000D2B200686EF0CEFFB6E70223026900F11C
:101F90003C01C4F89432012AC4E9073303654FF4C5
:101FA0008073456583870DF106038364E8D1C364BC
:101FB000E6E700BF08B520B904486AF095FD04487B
:101FC00008BD04486AF090FD014808BD30690C085E
:101FD000B42F002454690C08024808B56AF084FD47
:101FE000014808BD78690C08B42F0024024808B5E0
:101FF0006AF07AFD014808BD80690C08B42F0024FE
:10200000024808B56AF070FD014808BD8C690C08EB
:10201000B42F002470B5124D124A2B68A2FB032383
:102020009B09013BB3F1807F01D3012070BD4FF0CC
:10203000E0220D4900240F2853614FF0F0030646BB
:1020400081F823304FF0070394611361EDD8014606
:102050004FF0FF306BF00EFA2046C5F82C6170BDD2
:1020600000000024D34D621000ED00E0034A01306F
:10207000116813685B1A8342FBD37047A02B0024BE
:102080003749024603688B4233D01831591AB1FAE6
:1020900081F1490969BB3348834240D018308342FB
:1020A00040D01830834236D0183083423DD01830AB
:1020B000834240D0183083422CD000F556708342C2
:1020C00037D029498B4233D018318B4236D0183162
:1020D0008B4236D018318B4236D018318B4236D0F5
:1020E00018318B4236D018318B4236D023F0FF00A6
:1020F00013E0DBB21D491E48103B10B41D4CA4FB7D
:1021000003435DF8044B01EB131393F82810C2E965
:102110001601704716211848D16590657047102147
:102120001348F9E716211248F6E706211248F3E7AB
:1021300006211248F0E710210F48EDE710210F4863
:10214000EAE716210D48E7E700210D48E4E70621FC
:102150000B48E1E710210A48DEE716210848DBE7D3
:10216000100002404000024028040240D0BA0B0890
:1021700000000240ABAAAAAA0400024000040240E8
:10218000040402400C4A136903F03803102B0DD0ED
:10219000182B09D063B913689B060BD51368074841
:1021A000C3F3C103D8407047FEF734BD04487047FD
:1021B0000448704701487047004402580090D0031B
:1021C00040787D0100093D00194A136903F0380386
:1021D000102B10B526D0182B09D02BBB13689B06EB
:1021E00024D513681348C3F3C103D84001E0FEF7B8
:1021F00011FD0F49104A8B69104CC3F3032313449C
:1022000093F8303003F01F0320FA03F32360896949
:1022100001F00F010A4492F8300000F01F0023FA89
:1022200000F010BD0648E4E70648E2E70148E0E7B1
:10223000004402580090D003D0BA0B0800000024DC
:1022400040787D0100093D00474A70B4946A956A60
:10225000D66A15F47C3FC5F30533D16B5BD0C1F36F
:10226000CC01C6F3001604F0030407EE903A06FB17
:1022700001F1012CB8EEE77A06EE901AFAEEE96A5F
:1022800003D0022C6AD0002C4AD0DFED387A87EEDA
:10229000876A936BC3F3080307EE903AF7EE005A90
:1022A000F8EEE77A77EEA67A77EEA57A67EE867A89
:1022B0002D4AB7EE006A936BC3F3462307EE103A3C
:1022C000B8EEC77A70BC37EE067AC7EE876AFCEEC6
:1022D000E66AC0ED006A936BC3F3064307EE103A5B
:1022E000B8EEC77A37EE067AC7EE876AFCEEE66A82
:1022F000C0ED016A936BC3F3066306EE903AF8EE05
:10230000E66A76EE866A87EEA67AFCEEC77A17EE64
:10231000903A8360704770BCC0E9003383607047B7
:1023200013689B061DD51468F7EE005A936B10498D
:10233000C4F3C102C3F30803D14007EE903A06EE9E
:10234000101AF8EEE77AB8EEC66A77EEA66AC6EE1D
:10235000077A36EEA57A67EE877AA9E7DFED057A88
:1023600095E7DFED057A92E7004402580024744AAD
:102370000090D00320BCBE4B0024744C474A70B47C
:10238000946A956AD66A15F07C7FC5F30553516C43
:102390005BD0C1F3CC01C6F3002604F0030407EEC2
:1023A000903A06FB01F1012CB8EEE77A06EE901A9E
:1023B000FAEEE96A03D0022C6AD0002C4AD0DFED95
:1023C000387A87EE876A136CC3F3080307EE903AF6
:1023D000F7EE005AF8EEE77A77EEA67A77EEA57A6E
:1023E00067EE867A2D4AB7EE006A136CC3F3462374
:1023F00007EE103AB8EEC77A70BC37EE067AC7EE31
:10240000876AFCEEE66AC0ED006A136CC3F306430C
:1024100007EE103AB8EEC77A37EE067AC7EE876A4B
:10242000FCEEE66AC0ED016A136CC3F3066306EEC8
:10243000903AF8EEE66A76EE866A87EEA67AFCEEC9
:10244000C77A17EE903A8360704770BCC0E90033DA
:102450008360704713689B061DD51468F7EE005A19
:10246000136C1049C4F3C102C3F30803D14007EE53
:10247000903A06EE101AF8EEE77AB8EEC66A77EEF2
:10248000A66AC6EE077A36EEA57A67EE877AA9E7DE
:10249000DFED057A95E7DFED057A92E70044025813
:1024A0000024744A0090D00320BCBE4B0024744C1E
:1024B000D0E9041283680B43C16970B51343044625
:1024C000056886B0626E0B4328681343A44A666AA7
:1024D00002401343E2682B606B6823F440531343BC
:1024E000A2696B609F4B9D4200F02D82236AA86811
:1024F0001A439D4B03401A43AA60EB6A23F00F0373
:102500003343EB62994B9D4228D0994B9D421AD0A0
:10251000984B9D4217D0984B9D4214D0974B9D42AB
:1025200011D0974B9D4219D0964B9D420BD0964BA4
:102530009D4208D0012000234FF00112C4E91A2364
:10254000236706B070BD914B5B6D03F00703052B4D
:10255000F0D8DFE803F0C65F7AAE8D9D8B4B5B6DE4
:1025600003F03803282BE5D801A252F823F000BF6E
:1025700011280408352504083525040835250408E4
:1025800035250408352504083525040835250408B3
:1025900015260408352504083525040835250408C2
:1025A0003525040835250408352504083525040893
:1025B0004B2604083525040835250408352504086C
:1025C0003525040835250408352504083525040873
:1025D000B3260408352504083525040835250408E4
:1025E0003525040835250408352504083525040853
:1025F0007126040835250408352504083525040806
:102600003525040835250408352504083525040832
:1026100091260408B1F5004F00F0468103A8FFF7AA
:1026200013FE049B002E40F08280626803EB52038D
:10263000B3FBF2F39BB2A3F110014FF6EF7291429C
:102640003FF678AFEB60002075E7B1F5004F00F082
:10265000FD806846FFF792FE019B002EE5D0013E0B
:102660000A2EE2D84A4A52F82620B3FBF2F3DCE7FE
:10267000B1F5004F00F03981002E56D0013E0A2EF0
:1026800053D8444A444B52F82620B3FBF2F3CCE72C
:10269000B1F5004F00F01781002E43D0013E0A2E05
:1026A00040D83E4A4FF4004352F82620B3FBF2F3E1
:1026B000BBE7B1F5004F00F02481344B1A68920655
:1026C0003FD51A68364BC2F3C102D340002EACD0BE
:1026D000013E0A2EA9D8334A52F82620B3FBF2F362
:1026E000A3E7B1F5004F67D0FFF76EFD274A2E4BE9
:1026F000D269C2F302121344626A93F8303003F0D5
:102700001F03D8403AB1013A0A2A04D8274B53F89C
:102710002230B0FBF3F0626800EB5203B3FBF2F33C
:102720009BB288E74FF400437FE71B4B7DE7013EF8
:102730000A2E3FF67AAF1E4A52F82620B3FBF2F378
:1027400073E7002E00F0FD80013E0A2E00F2F980B2
:10275000184A134B52F82620B3FBF2F365E700BF8B
:10276000F369FFCF000C0058FFF4FF110010014087
:102770000044004000480040004C00400050004031
:102780000014014000780040007C004000440258E2
:1027900010BB0B0810BB0B0800093D0010BB0B0859
:1027A0000090D00310BB0B08D0BA0B0810BB0B086D
:1027B00010BB0B0810BB0B08FFF706FDB34AB44B68
:1027C000D269C2F302121344626A93F8303003F004
:1027D0001F03D8403AB1013A0A2A04D8AD4B53F846
:1027E0002230B0FBF3F06268530803EB4003B3FB05
:1027F000F2F39BB2A3F110014FF6EF7291423FF654
:1028000099AE23F00F02C3F342031343EB601AE7C0
:10281000B1F5004F2FD0FFF7D7FC9C4A9C4BD269F3
:10282000C2F302221344626A93F8303003F01F03AC
:10283000D840002A3FF46FAF013A0A2A3FF66BAF47
:10284000954B53F82230B0FBF3F064E76846FFF78E
:1028500095FD01993EB1013E0A2E04D88F4B53F8E5
:102860002630B1FBF3F16268530803EB4103B3FB7D
:10287000F2F39BB2BEE7FFF7A7FC844A844BD26910
:10288000C2F302221344626A93F8303003F01F034C
:10289000D840002AA7D0013A0A2AA4D8804B53F87E
:1028A0002230B0FBF3F09EE703A8FFF7CDFC0499BC
:1028B000002ED8D0013E0A2ED5D87A4B53F82630B8
:1028C000B1FBF3F1CFE7002E36D0013E0A2E33D80C
:1028D000754B53F82630B1FBF3F35B00626803EBF2
:1028E0005203B3FBF2F39BB284E746B3013E0A2ED8
:1028F00025D86E4A6E4B52F82620B3FBF2F35B00EC
:10290000ECE7624B1A68910640F1C2811B68694A84
:10291000C3F3C103DA403EB1013E0A2E04D8664B30
:1029200053F82630B2FBF3F261684B0803EB420325
:10293000B3FBF1F39BB25DE74FF48033CEE75F4B1F
:10294000CCE75C4B71E6A9685D4B0B4013434F4AE3
:10295000AB60EB6A23F00F033343EB62936D03F03C
:102960000703052B3FF6E6ADDFE803F0D0C1B277F1
:102970006803002E00F07881013E0A2E00F2748177
:10298000504A4FF40040402352F82620B0FBF2F0AA
:1029900000283FF458AE656805EB450282423FF6D9
:1029A000C9ADB0EB053F3FF6C5AD202B00F27E81EF
:1029B000023B1E2B3FF6BEAD01A252F823F000BF32
:1029C000152C040835250408EF2B040835250408C8
:1029D0003525040835250408C92B040835250408C5
:1029E000352504083525040835250408352504084F
:1029F00035250408352504088F2B040835250408DF
:102A0000352504083525040835250408352504082E
:102A1000352504083525040835250408352504081E
:102A2000352504083525040835250408352504080E
:102A300035250408352504083F2B0408002E00F036
:102A40001781013E0A2E00F213811F4A20231848E5
:102A500052F82620B0FBF2F09AE70C4B1A68950664
:102A600040F109811B681348C3F3C103D840002E0D
:102A700000F0F880013E0A2E00F2F480134A102381
:102A800052F82620B0FBF2F082E700BF0044025863
:102A9000D0BA0B0810BB0B0810BB0B0810BB0B08FF
:102AA00010BB0B0810BB0B0810BB0B0810BB0B08AE
:102AB00000093D000090D00310BB0B0800127A0003
:102AC000FFF4FF1110BB0B0810BB0B0810BB0B0869
:102AD0006846FFF753FC01983EB1013E0A2E04D828
:102AE000864B53F82630B0FBF3F0082350E703A8D9
:102AF000FFF7AAFB04983EB1013E0A2E04D8804B92
:102B000053F82630B0FBF3F0042341E7FFF75CFBFA
:102B10007C4B7D491B6A626AC3F302130B4493F832
:102B2000303003F01F03D8403AB1013A0A2A04D8E2
:102B300001EB82010B6CB0FBF3F0022328E7616A22
:102B4000002900F0CE8001390A2900F2CF806F4BB6
:102B50006F4803EBC103D3E90023002170F0AAFB07
:102B600003460902180241EA13616B0818182A4645
:102B70004FF0000341F1000170F09CFBA0F54072A2
:102B8000644B9A423FF6D6AC634BD8605BE55D4A36
:102B9000636A1168880640F19680126800215F48D8
:102BA000C2F3C102D0404BB1013B0A2B06D85C4AAC
:102BB00002EBC303D3E9002370F07CFB090203029C
:102BC00041EA10616808D1E76846FFF7D7FB636AFE
:102BD00001980021002BF1D0013B0A2BEED8514A7D
:102BE00002EBC303D3E9002370F064FBE6E703A81C
:102BF000FFF72AFB636A04980021002BDED0013B1B
:102C00000A2BDBD8484A02EBC303D3E9002370F058
:102C100051FBD3E7FFF7D8FA3A4B3B4D00211B6A33
:102C2000626AC3F302132B4493F8303003F01F039E
:102C3000D84042B1013A0A2A05D805EBC205D5E9C8
:102C40001C2370F037FB62680902030241EA10613D
:102C5000500818184FF0000341F1000170F02AFBF2
:102C60008CE72E48102396E64FF40040402392E66E
:102C7000274820238FE6002EF3D0013E0A2EF0D8FD
:102C80002A4A1023254852F82620B0FBF2F07FE6AE
:102C900056B1013E0A2E07D8254A204B52F826206D
:102CA000B3FBF2F35B0019E6224B17E6616AA9B1A8
:102CB00001390A291DD8204B4FF4004003EBC10312
:102CC000D3E9002349E773B1013B0A2B0BD81B4A18
:102CD000124802EBC303D3E900233EE74FF40000A0
:102CE00043E7174841E7174803213EE7144800210E
:102CF0003BE74FF40000002137E700BF10BB0B0893
:102D000010BB0B0800440258D0BA0B0840BB0B089C
:102D100000093D00FFFC0F00000C00580090D0039C
:102D200040BB0B0840BB0B0840BB0B0810BB0B089B
:102D300010BB0B080020A10740BB0B0840BB0B08D1
:102D40000000093D000090D0344A136830B423F0ED
:102D50008063334C1360256803E023685B1B022B00
:102D600054D813681B01F8D4936A056823F47C33A4
:102D700043EA053393628368C568013B013D5B020A
:102D80002D049BB205F4FE052B434568013DC5F3B8
:102D900008052B430569013D2D0605F0FE452B4333
:102DA0009363D36A456923F0C0032B43D362D36A8C
:102DB000856923F020032B43D362D36A23F01003E9
:102DC000D362D36BC0696FF3CF0343EAC003D3630D
:102DD000D36A43F01003D362D36AD1B101290CBF87
:102DE00043F4801343F40013D3620C4A136843F096
:102DF00080631360216803E023685B1A022B05D807
:102E000013681B01F8D5002030BC7047032030BC8C
:102E1000704743F40023D362E7E700BF0044025841
:102E2000A02B0024344A136830B423F08053334C71
:102E30001360256803E023685B1B022B54D81368DA
:102E40009B00F8D4936A056823F07C7343EA05532A
:102E500093628368C568013B013D5B022D049BB210
:102E600005F4FE052B434568013DC5F308052B43DA
:102E70000569013D2D0605F0FE452B431364D36A19
:102E8000456923F440632B43D362D36A856923F4F5
:102E900000732B43D362D36A23F48073D362536CE1
:102EA000C0696FF3CF0343EAC0035364D36A43F4AA
:102EB0008073D362D36AD1B101290CBF43F40003FC
:102EC00043F08073D3620C4A136843F0805313605D
:102ED000216803E023685B1A022B05D813689B0066
:102EE000F8D5002030BC7047032030BC704743F455
:102EF0008003D362E7E700BF00440258A02B002400
:102F00004B4B10B41B684B4CA4FB03435B0A03FB05
:102F100002F25AB18446531E4748DCF83420013B84
:102F2000024201D0920406D55C1CF6D14FF000405D
:102F30005DF8044B7047DCF834305C0741D4DCF8B2
:102F40003430D80709D43D4BCCF83830DCF8103099
:102F5000DBB2994205D00120EAE70123CCF83830F2
:102F6000F9E7DCF81430364818400028E0D0002B90
:102F70002CDB5A002DD49C002DD4D9002DD41A015D
:102F80002ED45C012FD4D90130D41A0231D45C0282
:102F900032D499023CD4DA0237D45C0332D4990398
:102FA0002DD4DA0340D41C043BD4590436D49A04FB
:102FB00031D413F0080F0CBF4FF480304FF40000F1
:102FC000B6E704231846CCF83830B1E74FF000706C
:102FD000AEE74020ACE78020AAE74FF48070A7E777
:102FE0004FF40070A4E74FF48060A1E74FF4006055
:102FF0009EE74FF480509BE74FF4005098E74FF462
:10300000802095E74FF4003092E74FF400408FE7BF
:103010004FF480408CE74FF4800089E74FF40010B4
:1030200086E74FF4801083E74FF4002080E700BF6D
:1030300000000024D34D621045002000C500200090
:1030400008E0FFFD38B5134D41F20D13124941F26E
:103050008832D5F85805D5F814450004A060E0681A
:10306000014020460B430D21E360FFF749FF38B1D3
:10307000D5F84825034600201343C5F8483538BD28
:10308000606900F4F050A0F50060B0FA80F04009EB
:1030900038BD00BFA02B0024C0E0FEFF0A4B013B5F
:1030A0000FD00269002AFADA0369074A43F00103E4
:1030B0000361013A05D0036913F00103F9D1184601
:1030C00070470320704700BF410D03002DE9F84F02
:1030D000066880460C46C6F3100535BB654B9E421C
:1030E00079D903F500339E4274D903F500339E422B
:1030F00040F2B48003F500339E4240F2B18003F504
:1031000000339E4240F2AE8003F500339E4240F20F
:10311000AB8003F500339E4240F2A880B6F1016F08
:10312000C0F0A680052011F053FC534F354697F8A8
:10313000A435012B00F0898006F178464FF0010993
:103140000023B6F5801F87F8A495C7F8A83536D3B5
:1031500002206AF033F9002874D1484A4FF002097E
:10316000D2F80C3143EA0903C2F80C31BFF36F8F78
:10317000BFF34F8F04F1200254F8043B944245F80A
:10318000043BF9D1BFF36F8FBFF34F8F48466AF00E
:1031900015F9B9F1010F394A5BD0D2F80C3123F09F
:1031A0000203C2F80C31002387F8A43500284CD163
:1031B000D8F800302033C8F80030BDE8F88F484612
:1031C0006AF0FCF800283DD12C4AD36843F0020392
:1031D000D360CBE70125284F97F8A435012B0ED0FB
:1031E0004FF0010A4FF0000B504687F8A4A5C7F82E
:1031F000A8B56AF0E3F8814628B187F8A4B54FF086
:10320000FF30BDE8F88F5046DFF870A0DAF80C30D8
:1032100023F4E663CAF80C30DAF80C3043EA0523ED
:1032200043F0A403CAF80C306AF0C8F8DAF80C20AE
:10323000134B1340CAF80C3087F8A4950028DED150
:10324000354679E7002387F8A4356FF00100BDE823
:10325000F88FD36823F00203D360A4E70225BAE70E
:103260000325B8E70425B6E70525B4E70625B2E748
:103270000725B0E7FFFF0108A02B00240020005223
:10328000FBF8FFFF0148FDF7B1B800BF5031002443
:10329000084810B4D0F8B035D0F8E44599691A68F8
:1032A0002CB1234600F5B6605DF8044B18475DF875
:1032B000044B7047A02B00240148FDF797B800BFCE
:1032C000A0310024084810B4D0F80036D0F83446B5
:1032D00099691A682CB1234600F5C0605DF8044B6B
:1032E00018475DF8044B7047A02B00240148FDF7F8
:1032F0007DB800BFF0310024084810B4D0F8503633
:10330000D0F8844699691A682CB1234600F5CA6042
:103310005DF8044B18475DF8044B7047A02B002460
:103320002DE9F04FDFF8689300EB400583B04300D0
:1033300009EB85050093D5F830310193002B00F09F
:1033400066818046B5F8360169F0F6FB95F83401E0
:103350000DF0B4FD044695F835010DF0AFFD08F110
:1033600001030746DBB2002C00F0768140F60C1218
:10337000A1882372E2802268002800F06181037234
:1033800040F60C23C38091613B68BA889A61112191
:10339000204609260DF04EFD112138460DF04AFD5C
:1033A0006525002C00F036812268A38811690B4244
:1033B00000F030811B04936111F0AEFA05468B4694
:1033C00011F0AAFA401B61EB0B01052871F1000115
:1033D000F6D314B12368A2889A6111F09DFA0546CC
:1033E0008B4611F099FA401B61EB0B01052871F136
:1033F0000001F6D3013ED3D11CB1A38822681B047F
:10340000936111F089FA05460E4611F085FA401BCA
:1034100061EB0601052871F10001F6D31FB1BB88ED
:103420003A681B04936111F077FA05460E4611F0D5
:1034300073FA401B61EB0601052871F10001F6D318
:1034400014B12368A2889A6111F066FA05460E4607
:1034500011F062FA401B61EB0601052871F10001D1
:10346000F6D317B13B68BA889A61009B20463E218B
:103470004FEA8805434409EB830393F83B41224616
:103480000DF0FAFC224638463E210DF0F5FC7B4C4F
:1034900008EB8803019A04EB0313C3F8B025784BBB
:1034A0009A4200F0C880FEF78FFE764BDA69C2F3CD
:1034B0000212754B134493F8303003F01F03D840C9
:1034C000009B434409EB830393F83831022B00F04F
:1034D000BE80032B00F0B680012B14BF4FF4C871DF
:1034E0004FF4487169F0B6FB034605EB0802002172
:1034F00004EB0212C2F8B815C2F8C015C2F8C41520
:10350000C2F8CC15C2F8D0150121C2F8B435C2F802
:10351000BC1592F8F11501F0FF00002900F0A4801D
:1035200005EB080123F0706224274FF4004C04EBF4
:1035300001115648D1F8B03581F8F1751E6826F0B2
:1035400001061E601A619A6822F400429A60C3F86C
:1035500008C05A681043D1F8C82558601202D868CC
:1035600020F40040D860DA6000221A60186840F049
:10357000010018602020C1F8F42581F8F105C1F898
:10358000E02581F8F22591F8F1052028C6B217D17F
:1035900091F8F005012813D081F8F175186820F032
:1035A00001001860186820F48050186018681860CE
:1035B000186840F00100186081F8F16581F8F02585
:1035C000009B0221DFF8CCA04544434404EB0514E2
:1035D00009EB830999F83A71384669F04BFF99F87D
:1035E000396107F01F034FF001097F09304609FADE
:1035F00003F302214AF8273069F03CFF06F01F036D
:10360000760909FA03F34AF8263084F8AC9503B03A
:10361000BDE8F08F013D2AD011F07EF983468A463D
:1036200011F07AF9B0EB0B0061EB0A01052871F19A
:103630000001F5D3B5E6FEF7C7FD124B1A6A36E76F
:103640009161A4E6C82169F005FB03464DE76421BA
:1036500069F000FB034648E700283FF498AE037288
:1036600040F60C23C3808FE682F8F00558E7002C63
:103670003FF4A2AEA38822689CE600BFA02B0024E2
:10368000001C005800440258D0BA0B080080000209
:103690000000002400E100E02DE9F04F441C83B05D
:1036A00091469DF8342031D000EB800CC04D064689
:1036B000870005EB0C104FEA0C1C90F8ACA5BAF192
:1036C000000F23D0AC44B9F1FF0F9E464FEA4108EA
:1036D0000CF5B66400D0FBB9002A40F0B180BA19ED
:1036E00005EB021292F8F115202906D1BEF1000F68
:1036F00016D14FF40073C2F8F435B5F89C36304655
:1037000001339BB2A5F89C36FFF70AFE4FF0000A82
:10371000504603B0BDE8F08F90F8F125202AECD197
:10372000BA1905EB021292F8F0150129E5D0012132
:10373000D5F800B082F8F015D2F8B01505E02A6887
:10374000A2EB0B02192A00F2ED80886910F4004008
:10375000F5D1BA194FF0210C0C9B05EB021282F83F
:10376000F1C54FF0400CC2F8D43582F8F2C5C2F86A
:10377000E405C2F8F4058F48A2F8DAE54B68019237
:1037800003408D4843EA08031843486059462046E1
:1037900069F0EAFD002840F06F81019AD2F8B01577
:1037A000C1F8289005E02B68A3EB0B030A2B00F26D
:1037B00056818A6912F08002F5D0BA1905EB02121F
:1037C000B2F8DA359BB2FF2B40F26E814B687B4832
:1037D00003407B4843EA08031843FF23A2F8D83587
:1037E000486007EB060905EB091905E0B9F8DA3579
:1037F0009BB2002B00F009815946204669F0B4FDC8
:1038000000287FF47AAFD9F8D435D9F8B02513F869
:10381000010BB9F8D8159062C9F8D4350139B9F857
:10382000DA3589B2013BA9F8D8159BB2A9F8DA3587
:10383000B9F8DA359BB20029D8D1002BD6D0A1E057
:10384000BA1905EB021292F8F11520297FF455AF51
:1038500092F8F01501293FF450AF0121D5F800B0DE
:1038600082F8F015D2F8B01505E02A68A2EB0B0239
:10387000192A00F208818A6912F40042F5D1B819B8
:103880004FF0210C0C9B05EB001080F8F1C54FF0B8
:10389000100CC0F8D43580F8F2C5C0F8F425A0F8B3
:1038A000DAE5B0F8DA35C0F8E4259BB2FF2B40F238
:1038B0000B814B683F4A1340424A43EA08031A43CC
:1038C000FF23A0F8D8354A6007EB060905EB091974
:1038D000B9F8DA35594620469BB2002B00F09780A4
:1038E00069F042FD00287FF408AFD9F8D435D9F843
:1038F000B02513F8010BB9F8D8159062C9F8D43582
:103900000139B9F8DA3589B2013BA9F8D8159BB26B
:10391000A9F8DA35B9F8DA359BB2002BD8D00029EE
:10392000D6D115E037442021002205EB0717D7F840
:10393000F43587F8F0250B43C7F8F43587F8F1150F
:1039400087F8F225D9E62B68A3EB0B030A2B3BD8AB
:10395000916911F08001F6D0B9F8DA359BB2FF2BEE
:103960006DD9536815490B40154943EA08031943BB
:10397000FF23A9F8D8355160AAE72B68A3EB0B0306
:103980000A2B21D8916911F08001F6D0B9F8DA3507
:103990009BB2FF2B29D9536808490B40084943EAD9
:1039A00008031943FF23A9F8D83551601EE700BF6B
:1039B000A02B0024009800FC00200181009C00FC4A
:1039C0000000FF010020FF81374405EB0717D7F8FF
:1039D000F43587F8F01543F02003C7F8F4352023B9
:1039E00087F8F13587F8F21587E6B9F8DA353E48F9
:1039F0009BB25168A9F8D835DBB2014048EA0343CD
:103A00000B4343F000735360F0E65946204669F0DB
:103A100081FC00287FF471AED9F8B0352021334CF9
:103A20003744D9615A6822405A60002205EB0713D7
:103A300089F8F11589F8F20583F8F02568E6B9F8F8
:103A4000DA3529489BB25168A9F8D835DBB2014074
:103A500048EA03430B4343F00073536038E7BB1954
:103A6000202005EB0313D3F8F4150143C3F8F41534
:103A700083F8F10583F8F225BB19002205EB031347
:103A800083F8F02539E6BB192020002105EB03134C
:103A9000D3F8F42583F8F0150243C3F8F42583F82E
:103AA000F10583F8F21528E6B2F8DA350E489BB234
:103AB000A2F8D835DBB24A6848EA03430240134310
:103AC00043F000734B608CE6B0F8DA354A689BB27D
:103AD000A0F8D835DBB2064848EA03430240134356
:103AE000044A1A434A60EFE6009C00FC00E800FE2E
:103AF000009800FC002000822DE9F04F451C83B0A7
:103B000014469DF8342000F08B800746DFF8CCA3E4
:103B100000EB8000BE000AEB001C00019CF8AC9595
:103B2000B9F1000F7CD05044FF2C9E464FEA41086B
:103B300000F5B6657AD1002A78D09CF8F125202AC4
:103B400065D19CF8F025012A61D00122DCF8B0157E
:103B5000DAF800408CF8F02505E0DAF80020121BB6
:103B6000192A00F221818A6912F40042F5D1F01974
:103B70004FF0220C0C9B0AEB001080F8F1C54FF0BF
:103B8000100CC0F8D43580F8F2C5C0F8F425A0F8C0
:103B9000DAE5B0F8DA35C0F8E4259BB2FF2B00F285
:103BA0001C81B0F8DA354A689BB2A0F8D835DBB290
:103BB000C44848EA034302401343C34A1A434A60D5
:103BC00006EB070B0AEB0B1BBBF8DA359BB2002B9D
:103BD00000F0D481DBF8B0250CE0DBF8B02591696A
:103BE00011F0200140F05481DAF800301B1B0A2B41
:103BF00000F276819369214628465B0700F10D812A
:103C00009369DB06EBD569F047FB0028E5D0BAF8ED
:103C10009C36384601339BB2AAF89C36FFF780FBEE
:103C20004FF00009484603B0BDE8F08FF2190AEBE7
:103C3000021292F8F1152029E9D10C99002900F01F
:103C4000C480BEF1000F00F0C08092F8F015012989
:103C5000DDD00121DAF800B082F8F015D2F8B01505
:103C600006E0DAF80020A2EB0B02192A00F29C8091
:103C7000886910F40040F4D1F2194FF0220C0C9B2B
:103C80000AEB021282F8F1C54FF0400CC2F8D435AD
:103C900082F8F2C5C2F8E405C2F8F4058948A2F832
:103CA000DAE54B680192034000F1044043EA08035F
:103CB00000F50840184348605946284669F054FB0F
:103CC000002840F0A380019AD2F8B0158C6206E07B
:103CD000DAF80030A3EB0B030A2B00F28A808A6922
:103CE00012F04002F4D0F2190AEB0212B2F8DA35FF
:103CF0009BB2FF2B40F266814B68724803407348C9
:103D000043EA08031843FF23A2F8D8354860F419A2
:103D10000AEB0414D4F8B01506E0DAF80030A3EB8F
:103D20000B030A2B00F2EB808A6912F00402F4D034
:103D30004A6AD4F8D4351A70B4F8DA35B4F8D8250C
:103D4000013B013A9BB292B2A4F8DA35D4F8D435EB
:103D5000A4F8D8250133C4F8D435B4F8DA359BB2C9
:103D600013B1002A00F0EC80B4F8DA359BB2002BD6
:103D7000D0D15946284669F0CDFA034600287FF491
:103D800046AFD4F8B0252020514DD061516829406C
:103D9000516084F8F10584F8F2353E4400230AEBC3
:103DA000061A8AF8F0353DE7F319202000210AEBC6
:103DB0000313D3F8F42583F8F0150243C3F8F42570
:103DC00083F8F10583F8F21521E7F3194FF4007237
:103DD0000AEB0313C3F8F42519E74B68394A13407B
:103DE0003A4A43EA08031A43FF23A0F8D8354A6049
:103DF000E6E6F31920200AEB0313D3F8F415014388
:103E0000C3F8F41583F8F10583F8F225F3190022BD
:103E10000AEB031383F8F025F9E6526ADBF8D43590
:103E20001A70BBF8DA35DBF8D425013B01329BB2BE
:103E3000CBF8D425ABF8DA35BBF8D835BBF8DA25A2
:103E4000013B92B29BB2ABF8D835002A3FF4BCAE2E
:103E5000002B7FF4B9AEDBF8B01504E0DAF80030DF
:103E60001B1B0A2B4BD88A6912F08002F6D0BBF8D4
:103E7000DA359BB2FF2B53D94B68164A1340164ACA
:103E800043EA08031A43FF23ABF8D8354A609BE6A0
:103E90009369590703D5BBF8D835002BBDD1202035
:103EA0000B4CF319D06151680AEB031321405160A8
:103EB0000022C3F8F42583F8F02583F8F10583F890
:103EC000F225A4E6009800FC002400820024FF8173
:103ED00000E800FE009C00FC0000FF01A02B002475
:103EE0003E440AEB0616D6F8F43586F8F01543F092
:103EF0002003C6F8F435202386F8F13587E6F31958
:103F00000AEB0313D3F8F41583F8F02541F02001F0
:103F1000C3F8F415202183F8F11583F8F22576E62D
:103F2000BBF8DA352F489BB24A68ABF8D835DBB21C
:103F3000024048EA0343134343F000734B6043E6F7
:103F4000D4F8B01505E0DAF80030A3EB0B030A2B28
:103F5000D5D88A6912F08002F5D0B4F8DA359BB270
:103F6000FF2B1FD94B681F4A13401F4A43EA08031F
:103F70001A43FF23A4F8D8354A60F5E621462846BF
:103F800069F0C8F900287FF442AEDBF8B035202193
:103F9000164CD9615A6822405A608BF8F1158BF89B
:103FA000F205FAE6B4F8DA350E489BB24A68A4F88E
:103FB000D835DBB2024048EA0343134343F00073B1
:103FC0004B60D1E6B2F8DA3509489BB2A2F8D83591
:103FD000DBB24A6848EA034302401343054A1A43E6
:103FE0004A6094E6009C00FC0000FF0100E800FE2F
:103FF000009800FC002400820348D0F8603113B11F
:1040000000F5AA7018477047000000240348D0F854
:10401000803113B100F5BA701847704700000024D2
:104020000348D0F8A03113B100F5CA7018477047A3
:10403000000000240348D0F8C03113B100F5DA7055
:1040400018477047000000240348D0F8E03113B14E
:1040500000F5EA7018477047000000240348D0F8C4
:10406000003213B100F5FA701847704700000024C1
:104070000348D0F8203213B100F505701847704797
:10408000000000240348D0F8403213B100F50D7051
:1040900018477047000000240348D0F8603213B17D
:1040A00000F5157018477047000000240348D0F849
:1040B000803213B100F51D701847704700000024CE
:1040C0000348D0F8A03213B100F5257018477047A7
:1040D000000000240348D0F8C03213B100F52D7061
:1040E00018477047000000240348D0F8E03213B1AD
:1040F00000F5357018477047000000240348D0F8D9
:10410000003313B100F53D701847704700000024DC
:104110000348D0F8203313B100F5457018477047B5
:10412000000000240348D0F8403313B100F54D706F
:10413000184770470000002410B41C4643688446AA
:104140006FF30F0323434360036843F001030360ED
:10415000036843F400730360002C3AD040F2E93066
:10416000DCF814309B0748D5002A49D012F8013BEF
:1041700040F2E9308CF82030DCF81430DB0720D432
:104180000138F9D1214B9C450CD0A3F578439C45CF
:1041900038D003F580639C4536D003F578439C45C1
:1041A0000BD103201A4A00EB400002EBC002B2F828
:1041B000683301339BB2A2F8683300205DF8044BEA
:1041C00070479CF83000C0B209B101F8010B013C06
:1041D000C4D1DCF814301B07FBD5DCF81830012003
:1041E0005DF8044B43F01003CCF81830DCF80030D5
:1041F00023F00103CCF8003070470138B0D1C1E79B
:10420000FF23B5E70120CDE70220CBE700300140D6
:10421000000000242DE9F84300242C4E804603685A
:1042200056F83450AB4209D001340E2CF8D1284A4C
:104230000021052006F0AAFE002019E0254B03EB23
:104240008409D9F8A076AFB198F8051000204B1C6E
:1042500001EB410203EB430307EBC202DB00C2F8B0
:104260000C80C2E90400F854182303FB01700830E5
:10427000BDE8F8830721682006F0FCFE0146C9F876
:10428000A006E8B13946682276F0C8FAD9F8A01637
:1042900006EBC4043B4689600C60096289630965CA
:1042A00056F83320954205D001330E2BF8D14F60DC
:1042B0000F46C9E7084F07EB83174F600F46C3E768
:1042C000064A052006F062FEB6E700BF98BB0B0861
:1042D0009C690C08A02B002478320024C4690C08C7
:1042E00030B40C4C0022234603E0013214330E2A72
:1042F0000CD093F804C08445F7D1DD68294201D180
:104300000029F2D1142303FB024000E0002030BC5E
:10431000704700BFB4030024F0B44468A37913F0DD
:10432000020266D002224FF0080C036864795B68D1
:104330009D48204493F83C40012C90F8380156D019
:10434000012483F83C40022483F83D40142848D8D7
:10435000DFE810F08600470047004700C100470033
:10436000470047003601470047004700F600470076
:1043700047004700150047004700470051001868F4
:104380008A4E046AB04224F480340462046A4568A8
:1043900024F4003444EA0242446D24F0700444F0F2
:1043A00060040ED006F58066B0420AD0804F06F554
:1043B0008046B04218BFB84203D006F58066B042CE
:1043C00001D145F480354560446581650262426DE6
:1043D00042F008024265426D22F004024265426DDD
:1043E00042650121002283F83D1083F83C20F0BC97
:1043F0007047944699E718686C4E046AB04224F4FA
:1044000080140462046A456824F4001444EA0252E9
:10441000446D24F4E04444F4C0440ED006F58066B4
:10442000B0420AD0624F06F58046B04218BFB8428B
:1044300003D006F58066B04203D125F4003545F47B
:10444000802545604465C1650262426D42F40062A8
:104450004265426D22F480624265426D4265C0E76A
:104460001868544D046A514E24F00104B0420462AD
:10447000046A24F0020442EA04024468876905EAF7
:10448000070545F060050FD006F58066B0420BD0F9
:1044900006F57056B04207D006F58066B04203D0EC
:1044A00006F58066B04207D122F0080244F4407459
:1044B0004CEA020222F00402446085614163026218
:1044C000826942F008028261826922F004028261FC
:1044D0008269826185E71868374D046A334E24F09B
:1044E0001004B0420462046A24F0200444EA021278
:1044F0004468876905EA070545F4C04500F09980DE
:1045000006F58066B04200F09480294F2B4EB042F1
:1045100018BFB84203D006F58066B04201D144F41A
:1045200040644460856181630262826942F4006292
:104530008261826922F4806282618269826150E7CD
:1045400018681A4E046AB04224F480540462046A63
:10455000456824F4005444EA0232C46924F4E64471
:1045600044F4C0440ED006F58066B0420AD0104F25
:1045700006F58046B04218BFB84203D006F5806603
:10458000B04201D145F480454560C46101640262D6
:10459000C26942F40062C261C26922F48062C261EF
:1045A000C269C2611DE700BFD0BA0B08000001401C
:1045B000004001408CFFFEFFFF8CFFFE00440140E5
:1045C00018681F4D046AA84224F480740462046AC7
:1045D000466824F4007444EA0222C46924F0730497
:1045E00044F060041ED005F58065A8421AD0154F2E
:1045F000154DA84218BFB84203D005F58065A84202
:1046000001D146F440564660C461C1630262C2698A
:1046100042F00802C261C26922F00402C261C269AA
:10462000C261DEE622F4006242EA0C2222F48062D9
:10463000E7E722F0800242EA0C1222F040026EE725
:1046400000000140004001400044014042685379AD
:10465000032B0FD8DFE803F00B0805021068403089
:10466000704710683C3070471068383070471068E9
:104670003430704700207047D0E90002064B517972
:1046800092790B44406893F83811530701D56CF0C8
:1046900087BD6CF0A7BD00BFD0BA0B08F0B5446869
:1046A000374A2469C368C4F303245B6852F8246062
:1046B000EFF31184102585F312884568314F95F882
:1046C00005E0D0F80CC002EB4E02D5F800E0158CE6
:1046D000DEF80C2005F4F05522EA0502CEF80C2095
:1046E00017F806E0DCF8102053F80E501F2A25F0CA
:1046F000010543F80E5039D9203A2025DCF804C0D2
:1047000005FA02F2CCF80C20E2B282F31188BA5D0D
:10471000DFF874C003EB020E46684569DEF804401A
:1047200004EA0C0C4CEA0101CEF80410717903295B
:1047300024D8DFE801F01815120231684031CEF8B4
:104740000C500124CEF80810995841F010019950EE
:104750009958214399500474F0BD31683C31EEE71B
:1047600031683831EBE731683431E8E72025DCF88F
:1047700004C005FA02F2CCF80820C5E70021DEE704
:10478000D0BA0B086CBC0B080000FFFF03681A7E50
:10479000012A2ED0002293F83010012909D093F875
:1047A000481001290ED093F8601001291BD02ABBB4
:1047B0007047022142F4806283F8301093F8481069
:1047C000012904D1022142F4006283F8481093F8D1
:1047D0006010012907D01B6800211B685962D96845
:1047E0000A43DA607047022142F4805283F8601075
:1047F000F1E702214FF400721976CCE74FF4007212
:10480000E9E700BF08B5204B98420ED003F580635E
:1048100098420AD01D4A03F58043984218BF90423F
:1048200003D003F5806398421BD1FDF7CDFC1849F6
:10483000184BCA69C969C2F30222C1F302211A44A2
:1048400092F8302002F01F02D040114A1269C2F3E0
:10485000C03241EAC202134493F83C3103FB00F03A
:1048600008BDFDF7B1FC0A490A4BCA69C969C2F320
:10487000021CC1F3021103EB0C0292F8302002F08B
:104880001F02D040E1E700BF0000014000400140AE
:1048900000440258D0BA0B0870B50E4605EE102A37
:1048A000D0E90031013E1A680868B6B25C68156844
:1048B000FFF7A8FF07EE900AB8EE455A9FED527A2F
:1048C000F8EE677A87EE850A30EE070A71F0F0F8A5
:1048D00023680138AB4280B252D0C4E900500023B3
:1048E0008022E660A360A261C4E9043394F83D30FD
:1048F00003F0FF02002B62D00223211D284684F81A
:104900003D30FCF7F9F9414B0122B5F1804FA5EBA1
:10491000030384F83D20B3FA83F34FEA531334D0F2
:104920009BBB3B4A95420CD002F58062954208D071
:1049300002F58062954245D002F57842954241D019
:1049400070BD94F83C30012BFAD00222314B01218A
:1049500084F83D20A8680340AB6084F83D1084F8DB
:104960003D206A68A96822F0700221F080010120D0
:1049700000236A60A96084F83D0084F83C3070BD73
:10498000636883423AD06060A9E794F83C20012A2A
:10499000D6D002211F4A002084F83D10A9680A40A1
:1049A0000121AA6084F83D10022284F83D206A6843
:1049B000A9680BB90028D6D022F47002D3E784F896
:1049C0003C2099E794F83C20012AB9D00221114AF1
:1049D000114884F83D10A968281A0A40B0FA80F0FE
:1049E0000121AA600022400984F83D1084F83C208F
:1049F0000A4A9542D8D00028D6D170BDE368B342A8
:104A00007FF46DAF70BD00BF0AD7233C00000140AA
:104A1000000400408800CEFF00040140000C00406C
:104A2000024B0348D3F8A016FCF7E2BFA02B0024EA
:104A300000000140034B4FF08040D3F8A416FCF770
:104A4000D7BF00BFA02B0024024B0348D3F8A81601
:104A5000FCF7CEBFA02B002400040040024B03480B
:104A6000D3F8AC16FCF7C4BFA02B0024000800400C
:104A7000024B0348D3F8B016FCF7BABFA02B0024B2
:104A8000000C0040024B0348D3F8BC16FCF7B0BF43
:104A9000A02B002400040140024B0348D3F8CC169D
:104AA000FCF7A6BFA02B002400180040024B0348CF
:104AB000D3F8D816FCF79CBFA02B0024004001407F
:104AC000024B0348D3F8DC16FCF792BFA02B00245E
:104AD00000440140024B0348D3F8E016FCF788BFBE
:104AE000A02B00240048014010B5064C0648D4F81D
:104AF000BC16FCF77DFFD4F8D0160448BDE8104082
:104B0000FCF776BFA02B002400040140001C0040ED
:104B100010B5064C0648D4F8BC16FCF769FFD4F86B
:104B2000D4160448BDE81040FCF762BFA02B002457
:104B30000004014000200040BFF34F8F0549064BA1
:104B4000CA6802F4E0621343CB60BFF34F8F00BF2B
:104B5000FDE700BF00ED00E00400FA0500210120A0
:104B600008B50DF083FF72B6FFF7E6FF2DE9F043BD
:104B7000BFB0BFF35F8F8A4C0021626A0B460D46BF
:104B800022F4803262620A46C4F89410C4F8983065
:104B90000133C4F89C20112BC4F8A020F6D10523C2
:104BA000C4F89430636A43F480336362BFF34F8F79
:104BB000BFF36F8F7B487C4A7C49121A74F006FD64
:104BC000D4F888207A4B012142F47002C4F888207E
:104BD00019601D611A6842F080021A601A680A435F
:104BE0001A601A6842F480321A601A6842F48052DD
:104BF0001A609D61DD611D629D62DD621D635D6302
:104C00009D63DD631D645D641A6822F480221A606E
:104C10001D664FF00063674AC2F80811A3606DF08B
:104C200023FC654AD36813F0040FD36840F0A380D7
:104C3000624B0021604A0591D96A21F00101D962D5
:104C4000DB6A03F001030593936943F440439361E6
:104C5000936903F440430593059B93699E04FCD537
:104C60004C2200210EA8564C75F0D8FD554A42F250
:104C70000303A4F110011268B3EB124F4FF00002CE
:104C80004FF00C0308BF0C460892E268A370002A9C
:104C90004CD1494A494B916941F440419161926933
:104CA00002F440420892DA6A42F00102DA62DB6AF8
:104CB00003F001030893089B3F4A93699D04FCD5C8
:104CC0003B4B4FF4403540480321D3F8E02042F0FD
:104CD0008002C3F8E0200122D3F8E03003F0800323
:104CE0000793079B85610D9BCDE9001300236DF0B1
:104CF0007DF8022301204FF48031A288CDE91733DB
:104D00000C231993A379CDE90E01E079217A1C9047
:104D10000EA81D91CDE91A2308220023CDE91E23F8
:104D2000FBF7F4FC032838D0A0B1FEE7234BD96A87
:104D300021F00101D962DB6A1F4903F001030893E6
:104D40008B6923F4404313438B618B6903F4404325
:104D50000893B0E71D4B1A6812F00E0F3AD11A688B
:104D600022F00F0242F002021A601B6803F00F03E8
:104D7000022B2FD0FEE723F00703154C43F002036C
:104D8000D360216805E023685B1AB3F57A7F3FF6AC
:104D90004FAF53689F04F6D54AE7FFF7DFFE00BF29
:104DA00000ED00E000000000C82F000000E30C0848
:104DB0000044025800800051004802580004005886
:104DC000DC0400240010005C001C0258002000528B
:104DD000A02B00246C4A936903F070033F2B05D885
:104DE000936923F0700343F040039361664AD369EB
:104DF00003F070033F2B05D8D36923F0700343F011
:104E00004003D361604AD36903F4E063B3F5806F74
:104E100005D2D36923F4E06343F48063D3615A4A33
:104E2000136A03F070033F2B05D8136A23F0700355
:104E300043F040031362544B9A69100705D49A69F2
:104E400022F00F0242F008029A614F4A936923F45C
:104E500070639361136899018CD5136941F28831AD
:104E60004A4C23F0070343F003031361206804E076
:104E700023681B1A8B4200F29981136903F03803EF
:104E8000182BF5D1936903F00F03082B05D993690B
:104E900023F00F0343F0080393613D4A136803F0C6
:104EA0000F03022B0BD9136823F00F0343F0020307
:104EB0001360136803F00F03022B00D05AE7324A45
:104EC000936903F07003402B05D9936923F07003B5
:104ED00043F0400393612C4AD36903F07003402BE5
:104EE00005D9D36923F0700343F04003D361264A08
:104EF000D36903F4E063B3F5806F05D9D36923F474
:104F0000E06343F48063D3611F4A136A03F07003C4
:104F1000402B00F243811C4EFDF734F91D4BB26962
:104F20001D4DC2F30322134493F8303003F01F03E6
:104F300020FA03F3D5F82C012B60FDF76BF800285D
:104F400040F035811023159017900EA80E93FBF7B3
:104F5000DDFB002840F021813368104A43F08003D4
:104F60003360D6F8F43043F00203C6F8F430D6F8D4
:104F7000F43003F002030493049B136A43F001032B
:104F80001362074B216810E000440258A02B002454
:104F900000200052D0BA0B08000000240004005882
:104FA00080380100013B3FF4F8AE22689142F9D00D
:104FB000226823689B1A0A2BFBD9A04C4FF480224D
:104FC0004FF440130EA80E924FF000082F936CF090
:104FD0004DF9D4F8EC3041F203029949032643F02D
:104FE00002030EA80227C4F8EC30D4F8EC3003F02A
:104FF00002030393039BD4F8943043F00203C4F8F4
:105000009430D4F8943023F00203C4F894300B6841
:105010008C49B2EB134F8C4B8C4A28BF0A465A601E
:105020001A6822F47C5242F400521A601A6842F064
:1050300060021A600E96CDE92B886CF017F94FF4D8
:10504000E0430EA8CDF8E4800E93CDE925886CF0FE
:105050000DF918230EA8CDF8B8800E93CDF8CC80AA
:105060006CF004F94FF4803305220EA812960E93CB
:1050700021934FF4FA73CDF858801197CDE90F239F
:105080000423CDE9148813936CF0F0F8D4F8E030E1
:105090003A464FF480716E4843F00103C4F8E030A3
:1050A000D4F8E03003F001030993099B4346CDE9AE
:1050B00000686CF09BFE23693A46664823F0FE7355
:1050C00043F088732361D4F8E03043F00403C4F85C
:1050D000E030D4F8E03003F0040306934346069929
:1050E0004FF40071CDE900686CF080FE236923F075
:1050F0007E4343F0FC432361FDF744F82860BFF38F
:105100005F8F554D4646554C01276B6A23F480331B
:105110006B62C5F8948023E0002946D0D4F8009053
:10512000637A103414F8060C1B0643EA007343EA52
:10513000410314F8051C43EA814314F8041C43EAB4
:10514000414314F8031CC5F89860013643EA014353
:10515000C5F89C90032E43F00103C5F8A03027D07A
:105160006368217A002BD7D0D4F800900029D7D1DA
:1051700029F01F01A3EB0108B8F1200F38BF4FF051
:105180002008404674F098F9411E034607FA01F0E2
:10519000804508BF1946C9B2C2E7FEE7136A23F08B
:1051A000700343F040031362B5E6FEE7E2E5E1E594
:1051B0000523C5F894306B6A43F480336B62BFF308
:1051C0004F8FBFF36F8FBFF34F8FBFF36F8F0022EF
:1051D000C5F85022BFF34F8FBFF36F8F6B6943F455
:1051E00000336B61BFF34F8FBFF36F8FC5F884201F
:1051F000BFF34F8FD5F8805043F6E0761649C5F3DC
:105200004E34C5F3C905640104EA06002B4640EAA2
:105210008372013BC1F86022F9D2203C14F1200FC7
:10522000F2D1BFF34F8F4B6943F480334B61BFF32F
:105230004F8FBFF36F8F3FB0BDE8F083004402583B
:105240000010005C7FBB2200008400407FBB223046
:10525000000002580008025800ED00E0EC040024B1
:10526000704700BF3F4B586D012830B585B06ED0F8
:105270003D494FF6FF003D4ACC683D4B04403D4D53
:105280003D482243CA605A6FC5F8582AD3F8F42023
:1052900042F00202C3F8F420D3F8F42002F0020234
:1052A0000392039AD3F8DC2042F00052C3F8DC20CA
:1052B000D3F8DC2002F000520292029AD3F8DC20EC
:1052C00042F08042C3F8DC20D3F8DC2002F08042B8
:1052D0000192019AD3F8DC2042F00042C3F8DC20AE
:1052E000D3F8DC20036802F0004224480092009AC0
:1052F000D1F8FC40224A44F08074C1F8FC40A2FB83
:1053000003420024920CC5F85C2A1E4AC0F8B02F54
:105310001D4A4460A2FB032302689B0942F001027C
:10532000013B0260B3F1807F07D34FF0E0221369A5
:1053300043F00403136105B030BD4FF0E022F020CC
:105340005361072381F8230094611361EDE7002185
:105350000DF08CFB0D4B1A6882F308885B68984748
:10536000FEE700BF0040005800ED00E00003FA0532
:1053700000440258A02B002400000024001000E08C
:1053800083DE1B4355CEACC5D34D62100098F01F91
:105390002DE9F843384E984606EB8003D3F84C418C
:1053A000002C66D004F1CA0306F5B6760546B4F8BB
:1053B000CA02A36104F5E57366601746E3614FF422
:1053C0008073261DE160C4E904332368C4F8C43047
:1053D000A36300284AD194F8C9000BF06FFD18F0C0
:1053E000080F94F8C89034D1BA0723D4FB0711D41E
:1053F000052194F8CE0268F03DF894F8CE320122EF
:105400001E4903F01F005B09824041F8232030460B
:10541000BDE8F883013548460BF050FDEDB218B1F8
:1054200040F206630572C38094F8CC2202210BF08F
:1054300023FDDDE76B1CDBB218B1037240F20653AB
:10544000C38094F8CD2202210BF016FDFB07CFD5C7
:10545000E0E70135EDB218B140F206730572C38082
:1054600094F8CD2202210BF007FDC1E767F064FB41
:10547000B1E72646CBE700BFD0BA0B0800E100E059
:105480000148FBF787BD00BF200500240148FBF75A
:1054900081BD00BFF00700240148FBF77BBD00BFC2
:1054A000C00A00240148FBF775BD00BF900D002421
:1054B0000148FBF76FBD00BF601000240148FBF7F7
:1054C00069BD00BF301300240148FBF763BD00BF76
:1054D0000016002470B52422456B00238168C0F8B3
:1054E000B42004462A6800F1340622F001022A6042
:1054F0002B606B60AB608279C0F8BC3080F8B03054
:10550000C0F8B430C364C0F8B83043659302816317
:1055100003F480534179C363130303F4005303641A
:10552000130203F48063436401F00203C90745D406
:10553000002B7BD1836412F00802D4F8B43059D028
:10554000002B7FD024233046C4F8B4302B6823F0DE
:1055500001032B60FCF7ACFF012815D0E36D002B95
:1055600077D16B68304623F490436B60AB6823F0CF
:105570002203AB60AB6843F00803AB602B6843F0D9
:1055800001032B606BF0E0FD6279D5070DD5D4F8EF
:10559000C030196841F480711960996841F00101C7
:1055A0009960196841F020011960900705D5D4F879
:1055B000C020136843F08003136070BD0421816430
:1055C00053B10C23D1078364B5D5E36D4FF480311B
:1055D00043F0020361662EE0D307ACD5C36D12F031
:1055E000080243F00203C3654FF480334366D4F8E6
:1055F000B430A5D10BB194F8B020242384F8B020A6
:105600003046C4F8B4302B6823F001032B60FCF75C
:105610004FFF0128B8D0E36DBBB96B68304623F467
:1056200090436B60AB6823F02A03A6E708238364EA
:10563000D30780D5E36D43F00103E3654FF40033F6
:10564000236678E784F8B0307CE73046FBF7C8FB88
:10565000E3E73046FBF7C4FB83E700BF816039E72F
:10566000417137E7012070472DE9F04F9C4D7C22B6
:1056700099B0002105F2145075F0D0F84FF4805322
:10568000D5F8606A4FF480423468C5F81C354FF491
:105690000033C5F820250122C5F8243595F8443596
:1056A000C5F81445C5F82825002B00F0A08003217B
:1056B0008C4B8D4A85F8441561680B4043F0FA0322
:1056C0006360236843F003032360D36CDE0340F17F
:1056D0001F8108A8FCF7B8FD0A9B4FF4FA70B3F5D8
:1056E000FA7FB3FBF0F0C0F06881804A2968B2FB12
:1056F000F0F202322B685B1A9A42FBD800227C4BF4
:105700007C490292A260E2680E6813407A4AA2FBCA
:10571000062641F2883243F48053760AE36002FBA6
:1057200006F63346002B00F04E81626B013B1106FA
:10573000F8D5724A4FF4D573A263A3606C4AE3684C
:105740001A4041F208131343E3604EB13346626BD3
:1057500012F0450F02D0920440F11383013BF6D1C1
:105760000023634AC5F85035A360E3681A40334606
:1057700042F48052E260002B00F02581626B013B15
:105780001106F8D55D4BA363029A4FF6FE739A4259
:1057900000F2AE81DFF85891594FDFF860810023A5
:1057A00037212046A36041F23713E26802EA09027A
:1057B000134341F28832E360FDF7A2FB002840F07A
:1057C0000481A76041F22913E26802EA0902134347
:1057D000E3604EB13346626B12F0450F02D0920483
:1057E00040F11F81013BF6D14FF08050EDE0454B79
:1057F0009C4259D0444B9C4200F0F38095F86C0ACF
:105800000BF05CFB834695F86E0A0BF057FB824663
:1058100095F8640A0BF052FB814695F8660A0BF086
:105820004DFB804695F8680A0BF048FB074695F853
:105830006A0A0BF043FB95F86D2A04460E21584680
:105840000BF01AFB504695F86F2A0E210BF014FB53
:10585000484695F8652A0E210BF00EFB404695F858
:10586000672A0E210BF008FB95F8692A38460E21AD
:105870000BF002FB0E2195F86B2A20460BF0FCFA88
:105880000021B6F9040067F0F5FDB6F90430002BED
:1058900007DB03F01F0001225B091C49824041F82D
:1058A0002320D5F8144502E70F4BD3F8D42022F477
:1058B0008032C3F8D420DA6F42F48032DA67DA6FCC
:1058C00022F48032DA67D3F8D42042F48032C3F86D
:1058D000D420D3F8D43003F480330193019B8DE7B7
:1058E000A02B0024002CC0FF00440258102101000E
:1058F000C0E0FEFF00000024D34D6210C500200070
:10590000000010C1007000520024024800E100E0D5
:10591000906A916AD76A11F47C7F536BC1F30516C4
:105920004BD0C3F3CC0307F0010700F0030007EEF0
:10593000906A07FB03F30128F8EEE76A07EE103AD6
:10594000BAEEE97A00F0B083022800F02D84002836
:1059500040F0AA831368980640F132841168B7EECC
:10596000006A136BC1F3C102C3F3080307EE903A58
:105970005C4BF8EEE77AD34037EE877A07EE903A41
:1059800037EE067AB8EEE76AC6EE267A67EE877AD1
:10599000554AF7EE006A136B136B126BC3F30643A1
:1059A00007EE103AB8EEC77A37EE267AC7EE876A66
:1059B000FCEEE67A17EE903A8FE62A682B689B1A7F
:1059C000022BFBD99AE64FF00040012385F84435BD
:1059D000D5F848351843C5F84805012019B0BDE889
:1059E000F08F414BD3F8DC2022F40072C3F8DC20A6
:1059F000D3F8842042F40072C3F88420D3F88420C2
:105A000022F40072C3F88420D3F8DC2042F4007240
:105A1000C3F8DC20D3F8DC3003F400730093009B60
:105A2000ECE6636B5B0700F1A981C4F8388062691A
:105A3000029B002A03F101030293029B04DB4FF651
:105A4000FE718B427FF6ABAE02994FF6FE73994220
:105A500000F2648357004FD5236801279807C5F8E3
:105A60004C7500F0B4810023DFF880802046A360ED
:105A700041F20233E26802EA08021343E360FBF7F3
:105A80000FFA28BB636904F1180A04F11C09C5F870
:105A90008035A369C5F88435E369C5F88835236A7C
:105AA000C5F88C3541F20313A060E26802EA0802EF
:105AB00004F120081343E36046B1636B13F0450F14
:105AC00002D09A0440F12D83013EF6D14FF0004000
:105AD000012385F84435D5F848350343C5F84835E2
:105AE0007BE700BF0090D00300440258C0E0FEFFF7
:105AF000029A9A4200F212832368990700F06781A4
:105B0000D5F84C75032FAED1D5F87025D5F874357E
:105B1000A169090DC5F85415910F8DF82010C2F335
:105B200083618DF82110C2F301618DF82210C2F358
:105B300007418DF82310C2F30721D2B28DF824104B
:105B40008DF825201A0DADF82620C3F303428DF8F9
:105B50002820C3F3C0328DF82920C3F380328DF89A
:105B60002A20C3F340328DF82B20C3F300328DF886
:105B70002C2000228DF82D20002F40F0A98240F625
:105B8000FC71D5F8782501EA830343EA92730C93FC
:105B9000C2F3C2638DF83430C2F302638DF835303E
:105BA000C2F342538DF83630C2F382438DF837305A
:105BB000C2F3C2338DF838300C999DF8383001317A
:105BC0009DF8280003F0070300F00F00023399400E
:105BD00001238340C5F85C15C5F860355B0A01FBFD
:105BE00003F3C5F864354FF40073D5F85865DFF852
:105BF0003CA40721C5F86835C2F38033360420463B
:105C00008DF83930C2F3C61302F07F028DF83A30B6
:105C1000D5F87C358DF83B20DA0F8DF83C20C3F3A6
:105C200041728DF83D20C3F382628DF83E20C3F3AC
:105C300083528DF83F20C3F340528DF8402000225C
:105C40008DF84120C3F300428DF84220C3F3C032E7
:105C50008DF84320C3F380328DF84420C3F34032E3
:105C60008DF84520C3F300328DF84620C3F381221E
:105C70008DF84720C3F30122C3F346038DF8482073
:105C80008DF8493001238DF84A3041F20713A660A0
:105C9000E26802EA0A02134341F28832E360FDF748
:105CA0002FF900287FF414AFD5F8008063699901BB
:105CB00061D44FF0400941F2101310212046C4F87E
:105CC0000890E26802EA0A02134341F28832E36074
:105CD000FDF716F900283FD1A66041F23713E268BC
:105CE0003721204602EA0A02134341F28832E36078
:105CF000FDF706F980BB4FF0FF330D216362C4F856
:105D00002890E36A23F0FF0343F06303E36241F268
:105D10000D13A0602046E26802EA0A02134341F232
:105D20008832E360FDF7ECF8B0B908AB04E02A680C
:105D3000A2EB0802013247D0626B12F4957F626BCE
:105D400048D11204F3D503F12001D4F8802043F8A0
:105D5000042B9942F9D1EAE7D5F84835C5F848351A
:105D6000B14A0123A263D5F848251043C5F8480578
:105D700085F8443531E64FF40060F1E70423A3636E
:105D800032E5636B5B0700F11282636BDF0700F1A2
:105D90000782636B580601D54023A36301220023C9
:105DA00037212046C5F85025A360A04AE3681A4071
:105DB00041F23713134341F28832E360FDF7A0F854
:105DC00000283FF4E1AC0FE54FF00040C8E74FF08A
:105DD00080607DE6100700F1EE81626B910700F1B3
:105DE000F581626B920609D5F2E1D4F8802043F880
:105DF000042B2A68A2EB08020132E5D0626B12F490
:105E0000805CF2D1DDE90A230899012F09984FEA55
:105E100012485FFA83F990FA80FE28F0FF084FEAF3
:105E2000112048EA0908DFF8109220F0FF00C4F8BA
:105E30003890C1F3811940EA1160C1F340118DF827
:105E40000C9080B28DF80D10D1B2ADF80E00CDF8E7
:105E500010E08DF81410C2F30721C2F303528DF83D
:105E600015108DF81620C3F38522ADF818808DF833
:105E70001A20C3F30122D5F820858DF81B20C3F327
:105E8000031203F00F038DF81C208DF81D309DF8D0
:105E900033308DF81E309DF81C309DF81D20DBB28C
:105EA000D2B272D00323C5F86CC585F84435B8F575
:105EB000004F7ED0B8F5804F00F0C080B8F1000FE1
:105EC0007ED0D5F8483543F00063C5F84835D5F89D
:105ED0004835002B53D1D5F82815D5F818350329A6
:105EE000D5F81C05D5F8242509D8D5F86C65B6F584
:105EF000007F04D0B6F5807F14BF04210221034344
:105F0000606813434A4A02401343012243EA0803EC
:105F10000B43636085F844252C6803E02B681B1B4A
:105F200001333ED067F00AF90428F7D1002301219C
:105F3000D5F84C25C5F84835C5F8403585F84415E1
:105F4000AAB18A427FF449AD02233A4C85F88830E1
:105F500004F26C530FCB84E80F0004F27C5310342E
:105F60000FCB84E80F00002019B0BDE8F08FD5F802
:105F70005035002BE9D0012B7FF42FADE5E72A4AFD
:105F80000123A26385F8443527E5134314BF4FF47A
:105F900000734FF48073C5F86C35032385F84435DE
:105FA00085E74FF000420123C5F8482585F84435C0
:105FB00013E5D5F8483543F08053C5F8483586E7F2
:105FC0006369002000219A01CDE9080100F1A38056
:105FD00008A867F0D5F800BB099BDB0340F1ED8012
:105FE000A66041F23713E2683721104E2046324056
:105FF000134341F28832E360FCF782FF68B9C4F8CA
:10600000088041F20613E26806212046324013431D
:1060100041F28832E360FCF773FFD5F8483503435B
:10602000C5F8483553E700BFFF0FE01FC0E0FEFF93
:10603000002CC0FFA42B00243A0F00180020636935
:106040000021CDE90801980100F1A78008A867F0B8
:1060500097F8034610BB099B590340F1B480A66032
:1060600041F23713E2683721604E20463240134335
:1060700041F28832E360FCF743FF034670B9022324
:1060800006212046A36041F20613E2683240134322
:1060900041F28832E360FCF733FF0346D5F8482528
:1060A0001343C5F8483512E7DFED517A87EEA66A4B
:1060B000136BC3F3080307EE903AF7EE005AF8EEBD
:1060C000E77A77EE877A77EEA57A67EE867A5FE4ED
:1060D000012F13D11B04D5F8782503F47C1343EA70
:1060E00012430C930C9B01339B02C5F85C35C5F839
:1060F00064354FF40073C5F8603574E53D4B4FF0DF
:1061000080500122A363D5F848350343C5F84835CC
:1061100085F84425DCE44FF400607EE74FF08070A2
:1061200053E4636B5B0759D4636BDE0752D4236976
:10613000DBB2032B50D1304BA363636913F4604F80
:1061400009D05C044ED413F4004F14BF4FF48050B8
:106150004FF48030BCE41B0C244A2046C5F8583567
:106160001B04A360E3681A4041F209331343E36060
:10617000FAF796FE00287FF4ABAC6269C5F870258B
:10618000DAF80030C5F87435D9F80010C5F878157C
:10619000D8F80010C5F87C15BAE44FF400637DE729
:1061A0000123A363FFF7DCBADFED147A7EE7042353
:1061B000A363FFF7D5BA0820D2E54FF080602CE743
:1061C000DFED0F7A72E74FF0806367E70220C7E5E3
:1061D0002020C5E50123A363012079E404231846A8
:1061E000A36375E44FF4005072E400BFC0E0FEFF0B
:1061F0000024744AFF0FE01FC500200020BCBE4BE6
:106200000024744C66F0F6BD66F0F4BD2DE9F84349
:10621000384E96F86C0A0AF051FE054696F86E0A5A
:106220000AF04CFE044696F8640A0AF047FE8146DE
:1062300096F8660A0AF042FE804696F8680A0AF066
:106240003DFE074696F86A0A0AF038FE06461DB17A
:106250000D23EB8000232B721CB10D23E380002360
:106260002372B9F1000F05D00D23A9F806300023E1
:1062700089F80830B8F1000F05D00D23A8F80630D2
:10628000002388F808301FB10D23FB8000233B72E8
:106290001EB10D23F38000233372484607F090FAB5
:1062A000012148460AF0C6FD404607F089FA384603
:1062B00007F086FA304607F083FA404601210AF0DB
:1062C000B9FD384601210AF0B5FD012130460AF03A
:1062D000B1FD284607F074FA204607F071FA284607
:1062E00001210AF0A7FD20460121BDE8F8430AF08C
:1062F000A1BD00BFA02B002410B51C200AF0DEFDBC
:10630000044611210AF096FD204607F05FFAC820E6
:106310000EF030FB2046BDE8104007F051BA00BF38
:106320002DE9F04FDFF8109587B0D9F8704A63690E
:1063300013F0010B02D007B0BDE8F08F6269A369CA
:106340001A42F8D06369A26913409D0703D56369B7
:1063500003F0020363616369A26900941340D806E5
:1063600014D5A36923F01003A361236A03F4F01288
:1063700003F00F05B2F5802F00F09C84B2F5402F9A
:1063800000F08E82A36943F01003A3616369A269E0
:10639000134019037CD46369A26913405F0300F1C1
:1063A000B5806269A3691A4256D46369A269134031
:1063B0001E0509D5009BD3F80838DD0700F1B1842C
:1063C000636903F4006363616369A26913401801A0
:1063D00010D5636903F00063636199F8643E002B94
:1063E00040F03C82012389F8643E636DC3F383036C
:1063F000C9F8683E6369A2691340D90400F1B2810B
:106400006369A26913409B0400F14B816369A2692F
:1064100013401E0700F117826369A2691340DD0271
:1064200000F10C826369A2691340980200F1F981BE
:106430006369A2691340590000F1EE816369A269A2
:1064400013405A077FF577AF65686B0700F15B84EF
:1064500063681D4365606EE7009B03F50062D3F837
:10646000043823F00103536099F8643E012B00F0D7
:106470000A82D9F8743E93F89C22042A03D193F837
:106480009D2283F89C22636903F0004363618CE7DB
:10649000D4F81858D4F81C381D402D0C3FF47BAFAD
:1064A00004F53067DFF884834FF0000A2046CDF80A
:1064B00004B008E06D080AF1010A07F1200708F1AD
:1064C0001C0800F0038215F0010BF3D000F53061D9
:1064D0004FEA4A1401EB4A139E68D0F8142816407C
:1064E000F20700F1B483310700F1F481F10601D520
:1064F0001023BB60B20601D52023BB60B30402D5D4
:106500004FF40053BB60D9F8700AD3E7D4F8187879
:10651000D4F81C381F40BFB2002F3FF442AF009B9D
:106520004FF00008CDF808B0A346C04D03F5106A3F
:10653000444609E004F1010C7F08644605F11C059E
:106540000AF1200A00F0A183FE07F3D5DBF810382A
:1065500004F00F02DBF83468E1B2D640F601F6B27F
:106560001E430BF5106303EB44139B681E4063014D
:10657000F007019327D50120009BD9F8748E00FA0B
:1065800002F2D3F8343823EA0203009AC2F834380E
:10659000CAF80800D9F8800AAB6C012800F0CC8357
:1065A000002C40F07783D8F89422022A00F0DE8491
:1065B00032F0040300F02F8598F8A032012B02D1AD
:1065C000002388F8A032330702D50823CAF8083020
:1065D000F00602D51023CAF80830710602D5402310
:1065E000CAF80830B20702D50223CAF808303306C9
:1065F000A0D5D5E914E070459CD86301AEEB00024C
:1066000004F1010C03F510686B6CD844934228BF69
:106610001346D8F81820033392B2B2EB930F32D35B
:1066200073460BEB0C36A646CDF804B01C468442EC
:1066300040F2EC83221A6B6C99F8801A9A4228BFB8
:106640001A46AB6C02F1030B4FEA9B0B69B991B28E
:106650000331890809D003EB810153F8040B8B4205
:106660003060FAD1AB6CD5E9144013441044AB64EC
:10667000D8F8183068659BB29B45D8D92346DDF819
:1066800004B074469E4686453FF656AF04F00F04AC
:106690000122DBF83438A24023EA0203CBF8343875
:1066A0004AE7D4F800296FF30A02C4F80029D4F8A5
:1066B000042842F48072C4F80428D4F808389F07EC
:1066C00000F1028113F0060318BF0F23C9F87C3ACA
:1066D000FBF77AFDD9F87C6AF3B2022B00F0408315
:1066E0004FF41053E268003ED9F8745E4FF0400753
:1066F00022F4705218BF0126D5F8D002E260E26899
:1067000013430022E3600124114640236AF0FAF9A2
:106710003B4600228021D5F8D002C5F86471C5F847
:1067200058416AF0EFF90023AC61C5F894326B6010
:10673000C5F8A432D5F8C8326F6285F89C42002BA8
:1067400000F05983D5F8B432002128465B68984799
:10675000D9F8743ED9F8704A1E74636903F4005383
:10676000636153E6009B03F50060436823F0010377
:1067700043604FF4846323612D4B013B02D02269B7
:106780009206FAD4D9F8745A1DB3009B4FF67F31A4
:1067900003F5106399600BF1010B1A682033AB45C8
:1067A00022F4001243F8202C53F8202C42F000620F
:1067B00043F8202CC3F8E811D3F8E02122F40012AA
:1067C000C3F8E021D3F8E02142F00062C3F8E021F1
:1067D000E0D1C36943F00113C361D9F8A03A002B9B
:1067E00046D1426942F22B0313434361036943F0EC
:1067F0000B030361009920460E4AD1F8003823F4B8
:10680000FE63C1F8003899F8801A6AF0FBF96369F1
:1068100003F480536361F3E5636903F080436361CC
:106820000CE6636903F40013636101E6103600248B
:10683000410D0300D4390024A02B0024636903F424
:1068400080136361EEE5D9F8740E90F89C32032B47
:106850001DD0636903F008036361DDE5D9F8743E78
:10686000042193F89C2283F89C1283F89D22C1E5B1
:10687000D0F8843043F00B03C0F88430436C43F00D
:106880000B034364B6E7002389F8643EFBE5D0F8C8
:10689000B432DB69002BDCD09847D9F8704AD8E7CE
:1068A000C5EBC50204F58051C3F30A1309EB82025C
:1068B000D2F8840C03440868C9F8340E0968C2F899
:1068C000843CC9F8381E5DE50223FFE60446DDF886
:1068D00004B060E5D9F8702A0823BB6002F5306384
:1068E000126C234410460292B84A9968904204D927
:1068F0000A0402D54FF400429A60D9F8744E99F810
:10690000343E04F52A7184F8A83299F835EE84F8FB
:10691000A9E2B9F8362EA4F8AA2203920122B9F806
:1069200038CEA4F8ACC2B9F83A0EC4F8942203F0F9
:106930001F02A4F8AE02012AC4F8980200F06A828D
:10694000022A00F09182002A40F0878203F060035F
:10695000202B00F05A83402B00F05783002B40F08F
:106960008A83BEF1090F14D8DFE80EF0CD9F13C360
:10697000138C72134C2DBBF1000F00F02F850323F5
:10698000012184F89C32D4F8B4326160002B40F0CD
:106990000F858021D4F8D0026AF05AF9D4F8D002D9
:1069A00000216AF055F9894B029A9A427FF69EAD12
:1069B000D9F8801A01297FF499AD854AD9F8700A6F
:1069C0006AF020F992E59DF80CB0BBF1010F89F84F
:1069D00078BEDED894F89C32022BCCD0032B00F08A
:1069E000D284D4F8D00280216AF032F9D4F8D002EF
:1069F00000216AF02DF9D4F8B432594620465B687C
:106A00009847D0E70128D4F8D03244D194F89C229A
:106A1000022A00F27884002A3DD0002122464FF05D
:106A2000020C42F8081FC4F894C2C4E90700C3E985
:106A300014019A6418694FF480710128998703F151
:106A40003C0108BFDA64C2B218686AF06BFAAAE7C0
:106A5000039B00221B0AADF81620013B062B98D899
:106A600001A252F823F000BFA16B0408856B040853
:106A7000B36B040893690408936904086D6B0408F8
:106A80003D6B04085CEA000CD4F8D03203D1039AC1
:106A90007F2A40F29F80184680216AF0D9F8D4F806
:106AA000D00200216AF0D4F87DE794F89C32013BD3
:106AB000022B3FF66EAF039B012B7FF474AF0020D7
:106AC000D4F8D032C4F8A402E061042203F13C01FE
:106AD000C4F894224FF4807298649A871A69012A44
:106AE000C3E9140008BFD864D2B218686AF01AFA71
:106AF00059E7039B012B7FF456AFC4F8A432D4F8B6
:106B0000D0320020E0E794F89C22D4F8D032013A49
:106B1000022AC0D80228BED1D4F8A4220021002A1B
:106B2000224618BF4FF0030B42F80CBFC4F8940282
:106B3000C4E9070018659A6459657BE7237C002B3C
:106B40007FF427AFD4F8B4320DF116001B6B9847D1
:106B5000072203464270BDF81620B4F8AE12002A90
:106B600040F0C38300297FF41EAFC8E7237C002BCD
:106B70007FF40FAFD4F8B4320DF116005B6B984779
:106B80000346E8E7227CD4F8B432002A40F05C8463
:106B90009B6A0DF116009847022203464270DAE71D
:106BA000D4F8B0320DF11601207C1B6898470346DB
:106BB000D1E79DF80C30052B3FF6EBAEDFE813F084
:106BC00065045D0455044D04D20226040A30544F76
:106BD000D439002494F89C22032A3FF45CAF039933
:106BE0005FFA81FB84F89EB293F8BC23012A11D08E
:106BF0001A68002083F838B0D2F800C82CF4FE6C74
:106C0000C2F800C8D2F800C84CEA0111C2F8001856
:106C100083F8BC030422002003F13C01C4F8942251
:106C20004FF48072E0619A871A699864012AD2B29F
:106C300008BFD864C3E9140018686AF073F9BBF19F
:106C4000000F00F0F283022384F89C32ABE60122AD
:106C5000BA60D9F8802AD0F840E0012AD3F808C0F9
:106C600000F0B880AC4A964500F0B981D9F8803C74
:106C70005AEA030300F03B82D8F808225FFA8AF14F
:106C8000D9F8740E6AF0CAF92DE45C46DDF808B054
:106C9000FFF787BBD8F8B4325B69002B3FF493ACA5
:106CA00098F89C22032A7FF48EAC40469847D9F886
:106CB00070BA88E447F6F07213423FF463ABC3F353
:106CC0000A13C5EBC502EF00D91C09EB8202890843
:106CD000D2F878CC09D00CEB810004F580566246DE
:106CE000316842F8041B8242FAD17A1B0CEB030193
:106CF00009EB8202C2F8781CD2F8841C1944C2F84D
:106D0000841CFFF73FBBD9F8740E0122D0F8B432CF
:106D100080F89C2201795B689847D9F8704AFFF7A0
:106D200097BBD9F8743E042193F89C2283F89C12F7
:106D300083F89D22FFF744BB6A6C1344AB64002CBC
:106D4000A8D1D9F8C02AD9F8B83A002A7FF42BACD8
:106D50000146724A5846019369F054FF019B22E4B0
:106D60006F4B704A0344934240F244816E4B6F4A2A
:106D70000344934240F258816D4B6E4A0344934260
:106D800040F2CC816C4B6D4A03449342C0F0FD81CC
:106D90006B4B6C4A0344934240F26D826A4B6B4AE0
:106DA00003449342C0F08582694B6A4A034493428C
:106DB000FFF496AC684B694A03449342C0F0DF820B
:106DC000674B684A034493422CBF4FF4C0534FF4BF
:106DD000E05387E41CF0080F00F01081624A9645EA
:106DE0007FF681AB1CF4004F3FF47DAB4FF40042C3
:106DF0009A60FFF778BBD5F8B832002B7FF4A2ACCD
:106E0000D5F8C032002B7FF49DACA1E4DDF804B0CE
:106E100074463BE403F060025B0602D5402A7FF42F
:106E2000B8AD94F89C32013B022B3FF6B2AD5FFA4D
:106E30008CFCBCF1030F3FF6ACADD4F8B432204665
:106E40009B689847B4F8AE32002B7FF4ACAD0028B5
:106E50007FF4A9ADD4F8D03236E603F08001D4F83F
:106E6000D00269F0F5FE9EE503F0600BBBF1200F48
:106E700000F0CB80BBF1400F00F0C780BBF1000FEA
:106E80007FF487AD5FFA8CF3BEF1010F194600F075
:106E90009681BEF1030F00F07C81BEF1000F40F03F
:106EA000698194F89C32D4F8D002022B00F005825C
:106EB000032B7FF4F1AD1CF0800F01F00F024FF0B7
:106EC000140340F0418203FB0242D2F858B1BBF1F7
:106ED000000F00F0C68103FB014303F5AA730029EC
:106EE00040F0B58200221A600222C4F89422C4E95C
:106EF000072202650022836442654FF4807200F12C
:106F00003C0182870269012AD2B208BFC3640068CB
:106F10006AF008F847E500BF0A31544FD43900241D
:106F2000405327FFFF340C00401E1BFF3F420F0061
:106F300000DC0BFF7F4F1200808CF9FE20D613007F
:106F400060B6E5FE5FE3160000D3CEFE40771B007F
:106F5000C05BB3FEC091210000CA91FE20753800CD
:106F6000E05459FEE09C41000A30544FD8E9081221
:106F7000914200F28D80D8F81C10B1FBF2F302FBB5
:106F8000131313B98A4240F2CD80D8F8B432DB68CB
:106F90002BB198F89C22032A01D1404698478021C2
:106FA000D8F8D00269F054FED8F8D032052200207B
:106FB00003F5FE71C8F894221A69C3F80802012A81
:106FC000A3F8FC01D2B208BFC3F80C02C3E98400E5
:106FD000186869F0A7FFD9F870BAFFF7EDBA1CF48A
:106FE000004F7FF403AF1CF0200F3FF445AE20228A
:106FF0009A6041E64FF47053FFF774BB1CF0200F0A
:1070000016D020229A60FFF76EBAD4F8B432204628
:107010009B689847C7E48021D8F8D00269F018FE31
:10702000D9F870BAFFF7C8BA4FF46053FFF75ABBEC
:10703000C34A964503D91CF4004F7FF4D7AE1B69B1
:10704000D8F80422C3F31203D31AC8F81432D8F8BC
:1070500008321344D9F8802C5AEA0202C8F80832E0
:1070600000F00D811A465FFA8AF1D9F8740E69F0C2
:10707000D5FFFFF738BAD4F8D0028021039269F027
:10708000E7FD039AD4F8D002114669F0E1FD8AE4E5
:107090008A1AD8F8D002C8F8202092B200F13C0138
:1070A000C8F81C2002650022836442654FF4807298
:1070B00082870269012AD2B208BFC364006869F0FE
:1070C00031FFD8F8D03200211A69C3F80812012A1A
:1070D000A3F8FC11D2B2186808BFC3F80C12C3E9B8
:1070E000841103F5FE7169F01DFFFFF765BA026CAC
:1070F000934B9A4203D90B68002BFFF6BDAD0023DA
:107100000B610B6943F400230B610B6943F0180317
:107110000B610B6943F0C0430B61ADE54FF4505375
:10712000FFF7E0BAD8F898329942BFF42EAFD8F8FA
:10713000D03200204FF48072C8F81C0003F13C01EB
:107140009A871A699864012AD2B2C3E9140008BF69
:10715000D864186869F0E6FE0021D8F8D032C8F883
:107160009812B1E7D4F8B032D3F814B0BBF1000FE5
:1071700040F05481D4F8D002802169F069FD59466D
:10718000D4F8D00269F064FD0DE44FF44053FFF7EA
:10719000A9BA94F89C22D4F8D032022A00F0848054
:1071A000032A5DD1039A10437FF4ABAC48063FF449
:1071B000A8AC1846039369F04BFD039BA1E494F837
:1071C0009C32022B62D0032BD4D1039B002B7FF483
:1071D000EAAB0A46D4F8D03251063FF492AC02F042
:1071E0000F015A6891423FF68CACC1EBC1021CF012
:1071F000800F4FEA820240F01D8102F5FE721C20D2
:107200004FF0000C00FB01301A4480F8FDC11170F2
:107210000021917093F8BC1301293FF472AC012155
:1072200083F8BC1392F801C01078D178BCF1010F3B
:107230001A68A1F102010CBF02F5106202F530627A
:10724000012902EB4012106820F40010106003D8EE
:10725000116841F080511160002283F8BC2350E492
:107260001846802169F0F4FC5946D4F8D00269F040
:10727000EFFCFFF798BB4FF43053FFF733BA314AB6
:107280000121029369F0BEFC029BEBE611F07F0B3B
:10729000D4F8D002E5D069F0DBFCD4F8D00280212C
:1072A00069F0D6FCFFF77FBB11F07F0B1846D8D0F2
:1072B000F1E74FF42053FFF715BA0B465B067FF456
:1072C000EBAB1CF0800F4FF002024FF0000114BF37
:1072D00004F1140304F5AA731960C4F89422C4E9F4
:1072E0000722C0E91421836407E600293FF407ACB4
:1072F0008A42D4F8D00228BF0A460221C4E90722F4
:10730000C4F89412F5E5032A7FF4C5AB0222211DCF
:10731000C4F894220022C4E907005A654FF4807231
:10732000186503F13C009A871A699964012AD2B260
:1073300008BFD9640146186869F0F4FDFFF733BB54
:107340000A30544FD439002403FB0243D3F818B059
:10735000BBF1000F85D001F07F02531C03EB8303C8
:1073600004EB8303002A3FF4BDAD1C2101FB0202A4
:1073700092F83E20003A18BF01221A60B4E54FF49B
:107380000053FFF7AFB9BBF1000F1CD061680129B2
:107390003FF4B5ABD4F8B432C9B220465B68984725
:1073A00099F8781ED4F8B4326160002B3FF4F1AA4A
:1073B0001B682046984700287FF4EBAAD4F8D03207
:1073C000E061FFF782BB022359462046C4F804B0AF
:1073D00084F89C32D4F8B4325B6898470422D4F81D
:1073E000D032C4F81CB0C4F894224FF4807203F178
:1073F0003C01C3F848B09A871A69012AC3E914BB53
:107400007FF472ABC3F84CB0FFF76EBBD4F8B03268
:10741000D3F818B0BBF1000F3FF4ACAE0DF116017C
:10742000207CD8470346FFF796BB012384F89C32A3
:10743000FFF7B9BA1C203C324FF0010C00FB0130C1
:107440001A4480F83DC0E2E6DB6AFFF7A2BB1C22CB
:1074500002FB010191F8FE218CE7D4F8B032D3F899
:1074600010B0BBF1000FD9D184E6D4F8B032D3F814
:107470000CB0BBF1000FD1D17CE6D4F8B032D3F818
:1074800008B0BBF1000FC9D174E6D4F8B032D3F81C
:1074900004B0BBF1000FC1D16CE600BFF8B5594D87
:1074A000D5F8CC4323699E0702D5E368980748D4F2
:1074B0002369590702D5E3685A073AD423691B07A1
:1074C00002D5E3681F072CD42369DE0602D5E368E2
:1074D000D8061ED42369D90702D5E368DA0738D461
:1074E00023691B0602D5E3681F066ED42369DE05F7
:1074F00002D5E3681D066FD42369580602D5E368F8
:10750000590670D423699A0602D5E3689B0671D4A4
:10751000F8BD6FF0100200232261E26985F8E833BC
:10752000D8E76FF0080200232261E26985F8E833AA
:10753000CAE76FF0040200232261A26985F8E833EC
:10754000BCE76FF0020200232261A26985F8E833EC
:10755000AEE72D4B6FF001029C422261C0D1D5E90C
:10756000D967BE42BCD0D5F848238CBFC6F580573A
:10757000BF1B264BD2F814C23344B9B2C2F808324A
:10758000C2F81012BCF1000FAAD14FF0010ED5F8CD
:1075900060033E44C5F8C010C2F814E240F2011284
:1075A0004366A0F8582002697245D2B2C0E91B1C9C
:1075B00008BF836600F15801006869F0A3FBB6F5C7
:1075C000805F1BD0C5F864638AE76FF08003236196
:1075D0002369DE0590D58CE76FF4807323612369FE
:1075E00058068FD58BE76FF04003236123699A0615
:1075F0008ED58AE76FF020032361F8BD0023C5F81C
:1076000064336DE7A02B0024001400401C4A0024C2
:1076100008B5FEF729F858B10E4A92F88C330133B9
:10762000DBB2072B82F88C3303D9002382F898331E
:1076300008BDD2F8C43323B1186899880369194288
:10764000F3D0D2F80C140123C2F8881382F89833CF
:1076500008BD00BFA02B002438B5184C00201849E5
:1076600041F20D13D4F85825D4F814551204C4F877
:1076700094032846AA60EA68114041F288320B431D
:107680000D21EB60FBF73CFC68B1D4F848350343AF
:10769000C4F84835D4F80C2409230020C4F8882302
:1076A00084F8983338BD6B6903F4F053B3F5006F79
:1076B000F0D10423022084F8983338BDA02B002495
:1076C000C0E0FEFF70B5834C94F898536B1E082BF6
:1076D0001DD8DFE803F0776A7B1C4E05351C2600B9
:1076E000A36A002B6CD10722D4F80C34D4F8805351
:1076F00084F89823C4F88833002D61D0D4F88433FB
:107700000120D4E9DD21A84794F898536B1EDBB221
:10771000022B4ED9042D18BF082D0CBF01200020CC
:1077200070BDFBF78FFC002840F0C980D4F8883387
:10773000D4F80C24FA339342ECD2FFF769FFC3E785
:10774000FBF780FC0028F1D0D4F894330022012B01
:1077500084F88C2340F2B780D4F89023013B0821B1
:107760000132C4F8943384F89813C4F890230120AC
:1077700070BD666A002E70D1FBF764FC0028A3D0B0
:107780000423D4F8805384F88C6384F89833002D54
:10779000EDD0D4F884333046D4F87423D4F8781379
:1077A000A84794F898536B1EB1E765F0C7FC04280E
:1077B0005CD0D4F80C34D4F888239B1AC82B73D827
:1077C000002070BD022384F898337DE7F9F768FD47
:1077D0000028EED194F85C500422B4F85E10236EB9
:1077E000C4F894031B0E206EA4F8A01384F8982309
:1077F000000C216E84F8A333226E090A94F86430D9
:1078000084F8A62384F8A73394F8653084F8A40399
:107810001B0994F8652084F8A513A06E02F00F02EE
:10782000B4F86E1084F8AC33B4F86E3084F8AD233D
:10783000C3F30B13B4F86E2084F8A25343EA112368
:1078400002F00F02C4F8A80303F00F0384F8B0237A
:1078500003F5FA63A4F8AE3336E7D4F88833D4F8E6
:107860000C2464339342FFF42FAF53E7F9F718FD6C
:1078700000289ED194F88830002BA3F10203B3FABC
:1078800083F308BF01255B0984F88D5384F88E3398
:10789000F9F706FD00287FF450AFA26F0323C4F868
:1078A0009C2384F898330FE7FFF7B2FE94F898030F
:1078B000042818BF08280CBF0120002070BD042335
:1078C00084F8983353E7FAD1FFF7C6FE94F898533B
:1078D0006B1E1CE7A02B00242DE9F04706460D4641
:1078E00090461F465F4C94F8981304290BD0082942
:1078F00007D1D4F89033B34205D0FFF7ADFE02288C
:10790000F1D001209FE00123C4F88083C4F8847380
:1079100084F87C33A362062384F89833EB06C4E929
:10792000DD564CD1BFF34F8F4F4A05F500712B4602
:10793000C2F8683220338B42FAD1BFF34F8FBFF3C6
:107940006F8F002D50D094F84435012B37D1731C24
:10795000D4F8641500228B42C4F848253DD803238F
:10796000D4F814754FF4007AC4F8305584F84435CF
:107970004FF40073FA621021C4F834353846D4F855
:107980004C35C7F808A0FA68012BDFF8E49041F203
:10799000101318BF760202EA0902134341F288323B
:1079A000FB60FBF7ADFA804628B3304B0122BB6386
:1079B000D4F848350343C4F8483584F84425FFF724
:1079C00027FED4F8805335B1D4F884330022D4F89C
:1079D00078130120A847032035E0D4F8483543F058
:1079E0000073C4F84835EAE7D4F8483543F000633B
:1079F000C4F84835E3E74FF0FF33182138467B627F
:107A0000C7F828A0FB6A23F0FF0343F09003FB6252
:107A1000FB6843F04003FB609023BD6501253D6595
:107A2000C4F8403541F21813BE60FA6802EA090250
:107A3000134341F28832FB60FBF762FA28B9FB6B13
:107A400043F48D73FB63BDE8F087084BBB63D4F848
:107A500048350343C4F8483584F84455C4F8408594
:107A6000ADE700BFA02B002400ED00E0FF0FE01FFA
:107A7000C0E0FEFF034B93F82400032894BF0020CE
:107A800001207047142F0024004870473C2F002429
:107A900070B4154D00202B4693F82A4014B1DE69CE
:107AA0008E4205D0013010330828F5D170BC7047E4
:107AB000AAB1AB6903EB40239A4201D1022C07D053
:107AC00095F8B83113B9012385F8B83101236B70EB
:107AD00005EB0015012385F82A3070BC704705EBD3
:107AE000001585F82A20E1E7205A002430B400234D
:107AF000184C204684F8A43003E001331030082BE2
:107B00001AD0C5698D42F8D190F82AC0BCF1030F94
:107B1000F3D19AB1A16901EB43218A4207D094F8CD
:107B2000B82112B9012284F8B8210122627004EB55
:107B30000314012384F82A3030BC7047D4F8A02005
:107B400004EB03130421013283F82A10C4F8A020A7
:107B5000F2E700BF205A0024A0B183681BB10C4B90
:107B600007229A7070470A4A042110781375032877
:107B70009170C2E9033314BF4FF480738023C2E9CC
:107B800001337047024B012283F8B8215A707047C5
:107B9000205A00240346202201481A80704700BF63
:107BA000CC1800240346202201481A80704700BFE9
:107BB000EC1800240346202201481A80704700BFB9
:107BC0000C19002403460A2201481A80704700BF9E
:107BD0002C190024034B0020D3F84C25B3F8503562
:107BE00093617047205A0024044B4FF4007C00201E
:107BF000D3F8F035A2F800C00B607047205A00247B
:107C00000020704701207047012070470020704716
:107C100010B41C6994420CD394460A4661448C42C9
:107C2000996938BFA4EB0C0261445DF8044B71F014
:107C3000CDBC5DF8044B704710B50E4B0E4C03F1F4
:107C40006C02DB6ED4F84C15B4F85005C4F820264D
:107C500088619847D4F82036002BFBD01B699847E1
:107C60000028F7D0B4F850350020D4F84C251B0478
:107C7000936110BDCC180024205A002438B5084B5D
:107C8000D3F8203653B1DB6914460D4698474FF4BC
:107C90000073026800202A60238038BD1B68FFDE65
:107CA000205A002408B5064BD3F8203623B11B69AF
:107CB0009847013840B208BD4FF0FF3008BD00BF03
:107CC000205A0024002070472DE9F041164C15463B
:107CD000B4F85C25D4F858051604866103B30E4643
:107CE00003EB0508D4F820260023314628466AB164
:107CF00057681A46B847D4F820260028F4D012B1A5
:107D00001369984718B9D4F82026F8E7FEE701353B
:107D100006F500764545E5D1D4F85805B4F85C255C
:107D200082610020BDE8F081205A00242DE9F04155
:107D3000184C1546B4F85C25D4F85805160486612D
:107D400023B30E4603EB050801E01B699847D4F8FE
:107D5000201651B10023CF68284631461A46B8474D
:107D6000D4F8203610B1002BEFD1002313B11B69DA
:107D7000984710B9D4F82036F8E7013506F50076B3
:107D80004545E4D1D4F85805B4F85C25826100205B
:107D9000BDE8F081205A002400207047704700BFE2
:107DA000704700BF03685A1C02601970704700BF1B
:107DB00003685A1C02601970704700BF024BD3F869
:107DC000240603681B681847205A00242DE9F04157
:107DD0003A4E33787E2B03D000273846BDE8F08139
:107DE00008214FF4FC4341F221041AB25B00002A3F
:107DF00084EA42009BB2B8BF83B20139F5D1B6F82C
:107E00000140002C37D02E4A2E4DAA42E4D2052C38
:107E1000A2F106028CBF002701271444AC4228BF00
:107E200047F00107002F47D141F2210EA24214D0A2
:107E3000501E04F1FF3810F8011F082283EA0123C5
:107E400019B25B0000298EEA410C9BB2B8BF1FFA41
:107E50008CF3013AF4D14045EDD1218861B1A21DE6
:107E6000AA42BAD2052904EB01002246B5D9A8429C
:107E7000B3D20446DAE7144C671E41F22105BC4632
:107E800017F8012F83EA0223082219B25B000029A8
:107E900085EA41009BB2B8BF83B2013AF5D164458F
:107EA000EDD16788094AFF1A231DB7FA87F79B1B94
:107EB0007F09A2F8283690E70F468EE700000208F7
:107EC000070002080000040801000208205A0024EC
:107ED00070B50C4D04460E4695F82430042B0AD09C
:107EE000082B06D1EB6983420AD0FFF7B5FB0228C5
:107EF00001D0012070BD0823C5E9074685F824306C
:107F0000022070BD142F00242DE9F04F6B4D1F4649
:107F100083B0064695F824300C469046042B09D0D1
:107F2000082B03D0002003B0BDE8F08FFFF794FBCF
:107F30000228F7D114F01F014DD1614B0122614895
:107F4000C3F8382602624FF40072C3F83046C3F813
:107F50003426002C4AD0DFF874B19BF83030012B66
:107F600039D1701CDBF85030CBF83410984245D82A
:107F70000323DBF800A08BF83030DBF83830CAF888
:107F80002C10012BCBE9094236D0730200934FF439
:107F9000007941F2101310215046CAF80890DAF81F
:107FA0000C2022F48F3222F49F7222F0010213433C
:107FB00041F28832CAF80C30FAF7A2FF034620B328
:107FC000414A0121CAF83820DBF834201343CBF8AA
:107FD00034308BF83010FFF71BFBEC68002CA1D07D
:107FE00000222B6969681046A0479BE7374A536B0C
:107FF00043F000635363EEE70096C8E7DBF83430E4
:1080000043F00073CBF83430E5E74FF0FF32009BCC
:1080100001905046CAF82420CAF828904FF0010970
:10802000DAF82C2022F0FF0242F09202CAF82C204B
:10803000DAF80C2042F04002CAF80C208122CAF87B
:108040005840CAF85090CBF82C2041F21112CAF8CF
:108050000830DAF80C1021F48F3121F49F7121F0EF
:1080600001010A431121CAF80C2041F28832FAF7C3
:1080700047FF68B1144A019BCAF83820DBF8342066
:108080000243CBF834208BF83090CBF82C30A2E7A9
:1080900005230F4A4846C5F80C8085F82430DAF8E5
:1080A0003C302F6143F49573CAF83C301368C5E93E
:1080B00000466B6103B0BDE8F08F00BF142F0024B1
:1080C000205A0024A42B0024FF0FE01FB43000240A
:1080D000AC2F002410B50B4C236D23B119689A887E
:1080E0000B691A4202D0FDF7BFFA18B1002384F8D9
:1080F000243010BD044B012220761B6884F8242014
:10810000636110BD142F0024AC2F002438B5037C0C
:108110000446D0F8D002002B52D14FF40073022253
:10812000012168F0EFFC01204FF40073C4F86C01EA
:108130000222D4F8D002812168F0E4FC244B002014
:10814000D4F8CC22012103F5C865E162C4F8C85215
:10815000A3F84808A3F89C0813689847D4F8D042BD
:1081600094F8BC332068012B12D01022194B026105
:10817000013B02D00269D106FAD46022154B02619C
:10818000013B02D002699206FAD4002384F8BC3382
:108190000022114B1F2504F50671C4F8302201227C
:1081A000C4F82C52A4F818222269C4F82432012AF7
:1081B000D2B208BFC4F8283268F0A4FD002038BD50
:1081C00040230222012168F09DFC01204023ADE7FD
:1081D000205A0024410D03006C62002470B5002277
:1081E000D0F8C84205461C4B84F838120D2684F896
:1081F000082204F50B70C4F82C3204F50374D5F88A
:10820000D0322E631A6740F2011203F15801DE6684
:10821000A3F858201A695866012AD2B208BF986696
:10822000186868F06FFDD5F8D0321F2000220121B8
:10823000C3F82442C3E98B021A69A3F818128A42D0
:108240001868D2B203F5067108BFC3F82842BDE82A
:10825000704068F057BD00BF555342532DE9F043BD
:10826000177883B0164605468846D0F8C8425A2F7C
:108270005CD8DFE817F0C5005B005B0076005B00B0
:108280005B005B005B005B005B005B005B005B0016
:108290005B005B005B005B005B00A7005B005B00BA
:1082A0005B005B005B005B005B00600171005B00DA
:1082B0005B0071005B005B005B005B0010025B0019
:1082C00073015B005B0097015B0007015B005B00D3
:1082D0005B005B00D5005B005B005B005B005B004C
:1082E0005B005B005B005B005B005B005B005B00B6
:1082F0005B005B005B005B005B005B005B005B00A6
:108300005B005B005B005B005B005B005B005B0095
:108310005B005B005B005B005B005B005B005B0085
:108320005B005B005B005B005B00F30094F85D2288
:10833000002105254FF0FF30531C04EBC202DBB2D5
:1083400082F83C5282F84012042B08BF0B4684F896
:108350005D3203B0BDE8F0830023A4F80A320020A8
:10836000F7E77021002294F85C3221700C21C4F8E8
:108370000520E17194F85D12C4F801209942C4F817
:108380000920C4F80D20627413D004EBC30101333B
:1083900091F83C02DBB2A070042B91F841022073EB
:1083A00091F8401218BF84F85C32617308BF84F8FA
:1083B0005C221223A4F80A323379122BCFD8A4F806
:1083C0000A32CCE75378DB0700F18981D0F8CC3250
:1083D00001EBC1011279D86900EB81000379053303
:1083E000934228BF1346A4F80A32002BB7D0C21814
:1083F000234412F8011D824203F8011DF9D1AEE7B2
:10840000D4F81462002E40F01382D5F8CC3208461E
:108410009B689847002840F05982A4F80A029EE71A
:10842000537813F0020340F0DE81D4F86012D4E9EF
:10843000992002448A42C2D994F85D22052011464F
:108440000132D2B204EBC101042A81F83C0281F866
:10845000403200F0FC8184F85D2280E7C84B08229E
:1084600003CBA4F80A22206040466160D5F8CC32E4
:10847000DB68984700283FF472AFE37863F07F032E
:10848000E3706CE794F80892B9F1000F40F047816F
:1084900094F91832002BC0F26A82D0F8CC32084628
:1084A0009B6898470746002840F04D82D5F8CC32AB
:1084B0004046DB6898470146002840F01B81D6F80B
:1084C0000220D5F8C80212BAC4F86422B6F8073000
:1084D000D0F860625BBA9BB21A44C4F86832B24208
:1084E00000F22082B4F85E2202FB03F3D4F81422D7
:1084F000934240F06881B3F5007F4FF0010028BF40
:108500004FF4007384F808021A46D5F8D032C3F845
:108510002C221A69C3F8301203F506718242A3F8BF
:108520001802D2B21868C3F8244208BFC3F8284220
:1085300068F0E8FB13E70023082208462360636025
:10854000D5F8CC32A4F80A22DB68984700283FF41B
:1085500006AFA37863F07F03A37000E7D0F8CC32B6
:1085600004F25E22084604F518715B6898470028FB
:1085700040F07081D4F860320822A080013BA4F85A
:108580000A22190E1A0C61F30700190A62F30F2070
:10859000B4F85E2261F3174052BA63F31F60E280C1
:1085A0002060DCE694F80872002F40F0B68094F961
:1085B0001832002B80F2A581D0F8CC3208469B6897
:1085C0009847002840F09680D6F8022012BAC4F8E6
:1085D0006422B6F80730D5F8C8625BBAD6F86012E4
:1085E0009BB21A44C4F868328A4200F24781B4F858
:1085F0005E2202FB03F3022284F80822D4F814223C
:108600009A4240F03B814FF40073D5F8CC224046AB
:108610003146A4F80A32B6F85E32D6F868421769D5
:1086200003FB04F4D6F86422B4F5007F28BF4FF4AE
:108630000074B4FBF3F39BB2B8470028C0F2348156
:10864000D5F8D03200222C6303F1580118685E6619
:10865000C3E91B4240F20112A3F858201A69012A0B
:10866000D2B208BF9E6668F04DFBB6F85E22B4FB3E
:10867000F2F2D6E9991311449B1AD6F83422121B50
:10868000C6E99913C6F83422002B7FF468AE0323A1
:1086900086F8083263E6002608460DF1020201A9B9
:1086A00026606660A660D5F8CC325B6898470028E3
:1086B00040F0AB8008200223BDF802200C21E070BE
:1086C000238152BA019BA4F80A12013B6281180E61
:1086D000E371190C1A0A20716171A2713FE6294BEE
:1086E0000722186899889B79A180A4F80A22206043
:1086F000A37134E6D5F8C822022092F85D3202EB6D
:10870000C3010133DBB281F83C0281F84072042BD3
:1087100000F0F48082F85D3221E6264673E7B4F873
:108720005E320846D4F868622146D5F8CC2203FBB5
:1087300006F65769B6F5007FD4F8642228BF4FF4D7
:108740000076B6FBF3F39BB2B8470028C0F2218154
:10875000B4F85E32D4F86422D4F86812B6FBF3F0B1
:108760000244091AC4F86422D4F83422C4F8681206
:10877000921BC4F8342239B92846FFF72FFDEEE5E5
:10878000ACBC0B08A4BC0B08D5F8D00201FB03F36A
:1087900001220021B3F5007FC0F82442A0F818227E
:1087A000026928BF4FF40073C0F8301200F506715B
:1087B000012AC0F82C32D2B208BFC0F828420068A3
:1087C00068F0A0FACBE590F85D3205245A1C00EB66
:1087D000C303D2B283F83C4283F84012042A60D02B
:1087E00080F85D22BBE594F85D32052000215A1C1B
:1087F00004EBC303D2B283F83C0283F84012042A8C
:108800007FF429AE84F85D12A9E5D5F8C8220220CC
:1088100092F85D3202EBC3010133DBB281F83C0216
:1088200081F84062042B7FF475AF82F85D6296E5B3
:1088300094F85D32052000211A460133DBB204EBC7
:10884000C202042B82F83C0282F84012DAD084F88B
:108850005D3284E5D5F8C8220224002192F85D3209
:1088600002EBC3000133DBB280F83C4280F84012D7
:10887000042B7FF44FAF82F85D1270E596F85D32FD
:1088800005211A460133DBB206EBC202042B82F843
:108890003C1282F8400214BF86F85D3286F85D0211
:1088A0005DE580F85D125AE5D5F8C8220424002160
:1088B00092F85D3202EBC3000133DBB280F83C4238
:1088C00080F84012A3427FF425AFD4E7D5F8C82240
:1088D0000520022592F85D3292F85D12013302EB19
:1088E000C101DBB281F84062042B08BF3B4681F82E
:1088F0003C5282F85D3284F8080230E582F85D72FD
:108900002DE594F85D3205211A460133DBB204EB04
:10891000C202042B82F83C1282F8407297D184F88C
:108920005D721CE590F85D3205241A460133DBB216
:1089300000EBC202042B82F83C4282F84012B0D015
:1089400080F85D320BE5D5F8C822022092F85D323E
:1089500019460133DBB202EBC101042B81F83C0262
:1089600081F840927FF4D6AE82F85D92F7E494F8F5
:108970005D3205211A460133DBB204EBC202042B3F
:1089800082F83C1282F840927FF461AF84F85D92E5
:10899000E5E4D5F8C8220424002092F85D32194697
:1089A0000133DBB202EBC101A34281F83C4281F802
:1089B00040027FF4AFAE82F85D02D0E4D0F8C81276
:1089C00010B591F80832022B07D0033B012B02D8D7
:1089D0000021FFF703FC002010BD01F21B2291F8DB
:1089E00019120446FFF73AFC0028F4DA0121204668
:1089F000FFF7F4FBEFE700BF70B5D0F8D0520121CC
:108A0000044695F8BC33A5F818128B4208D0002212
:108A1000286885F8BC1368F061FB002385F8BC3337
:108A2000D4F8D052002640F20112C4F86C6195F8D7
:108A3000BC33A5F85820012B08D001222868114624
:108A400085F8BC2368F04AFB85F8BC630025D4F8A0
:108A5000C802E56271F01AFE2846C4F8C85270BD1B
:108A600038B5D0F8C8520446D0F8D00295F818327C
:108A700013B9D5F814323BB9812168F0E9F895F8BB
:108A80000932022B0ED038BD95F80932002BF3D1F4
:108A9000012168F0DDF8D4F8D0028121BDE838402A
:108AA00068F0D6B8D4F8D0321F20002205F503753F
:108AB0000121C3F82452A3F8181203F50671C3E983
:108AC0008B021A691868012AD2B208BFC3F828526B
:108AD000BDE8384068F016B970B5D0F8C842054610
:108AE00094F8086286B1012E01D0002070BD04F216
:108AF0001B2294F81912FFF7B1FB0028F5DA0121C7
:108B00002846FFF76BFBF0E7D4F81432D4F81022B4
:108B1000C4F83432D0F8D032C4F83022D3F830322E
:108B20001F2B08D1324BD4F80C229A4203D194F86F
:108B30001912012918D994F85D320021052628461A
:108B400004EBC3020133DBB282F83C6282F84012CC
:108B50000222042B84F8092208BF0B4684F85D32F8
:108B6000FFF77EFF002070BD94F81A32013B0F2BF7
:108B7000E1D804F21B22FFF771FB002894F80832B9
:108B80002BDB013B022BB0D9B4F80A1259B3D5F84C
:108B9000C832042283F80822D3F8342283F83862DA
:108BA000521AC3F83422D3F81432994228BF194616
:108BB000D5F8D0321A692963012AD96640F2011129
:108BC000D2B21868A3F8581003F158015C661E670A
:108BD00008BF9C6668F096F887E7052B8FD028467B
:108BE000FFF73EFF81E72846FFF7F8FA7DE700BF71
:108BF000555342432DE9F041002382B00446D0F89A
:108C0000C852ADF806300B7813F0600239D0202A34
:108C10000DD08021D4F8D00268F01AF80021D4F8E1
:108C2000D00268F015F8022002B0BDE8F0814A7861
:108C3000FE2A00F0DD80FF2AEBD14A88002AE8D125
:108C4000CA88002AE5D11B06E3D44FF4807305F5EA
:108C500003700121A5F80832D4F8D0321F24C3E9EB
:108C60008B421A69C3F82402012AA3F81812D2B25F
:108C700003F5067108BFC3F82802186868F042F8C7
:108C800025E04B780B2BC4D801A252F823F000BF8B
:108C9000B38D0408F38C0408138C0408138C0408A7
:108CA000138C0408138C0408138C0408138C040818
:108CB000138C0408138C0408D38C0408C18C04089A
:108CC00090F89C32032BA4D18B78C5F80432002095
:108CD000AAE790F89C32D0F8D002032B00F0B280C3
:108CE000802167F0B5FF0021D4F8D00267F0B0FF13
:108CF00099E7D0F8D0628F8896F8BC3391F90420B8
:108D000007F00F07012B00F006810123002A3168CC
:108D100086F8BC33C0F2AC801023884A0B61013A5C
:108D200000F000810B6913F01003F8D186F8BC3312
:108D3000C7EBC7039B00C7EBC7024FF0000803F562
:108D4000FE7306EB8202F11882F8FC7182F8FD8155
:108D500096F8BC23012A09D00122306886F8BC238A
:108D60004A78F15C68F0BAF986F8BC8307EB8707AC
:108D70000023D4F8D00204EB8707C7F85831237CCE
:108D8000002B40F0BC804FF400730222012167F0F9
:108D9000B9FE0123C4F86C3195F80932022B96D143
:108DA0008121D4F8D00267F053FF002385F80932FF
:108DB0008DE790F89C32D0F8D002032B90D102239B
:108DC000002200F13C01C4F89432C4E90733426543
:108DD0000DF10604026903654FF48073012A84646F
:108DE000838700D1C464D2B2006868F09BF86EE754
:108DF0004E88002E7FF40DAFCF88012F7FF409AF8E
:108E00001A067FF506AFD0F8CC3205F500759B69E0
:108E1000984702222860D4F8D032C4F894224FF444
:108E2000807203F13C011868C4E907779A871A69D0
:108E30009D64012A1F65D2B25E6508BFDD6468F0DB
:108E400071F844E70222012305F501754FF48071A2
:108E5000C4F894220022C4E90733C0E9143202693D
:108E6000818700F13C019A42856408BFC564BAE776
:108E7000BB01324A43F020030B61013A58D00B6921
:108E800013F02003F9D186F8BC33C7EBC7039B006E
:108E9000C7EBC70201213C3306EB8202F01882F8CF
:108EA0003C7082F83D1096F8BC238A4209D086F8BF
:108EB000BC134278F15C306868F010F9002386F842
:108EC000BC3307EB87070023D4F8D00204EB8707F5
:108ED000BB61237CCBB94FF400730222812167F080
:108EE00011FE0121E16295F80932022B3FF458AFDF
:108EF000012B3FF4ECAE2046FFF770F9E7E6402384
:108F00000222012167F0FEFD43E740230222812176
:108F100067F0F8FDE5E7C7EBC703002A4FEA8303D4
:108F2000B6DB08E7C7EBC70386F8BC239B0002E764
:108F3000C7EBC70386F8BC239B00A9E7410D0300DC
:108F40002DE9F843DDF820800F4616460021202247
:108F500004461D4671F062FCB8F1000F0CD0D8F841
:108F60000030B8F80A20E3811B0C2382D8F80430C3
:108F70006282E3821B0C2383384669F059FBF306B7
:108F800019D4431EB8B107EB000C01E0013B12D32A
:108F90001CF801EDBEF12E0FF8D1C01A03F1010942
:108FA000421EB944032AA8BF0322082BA8BF0823E6
:108FB00090461A4606E008280246B9464FF00008D7
:108FC000A8BF08224FF02033394620462360636053
:108FD00070F0FCFA164B04F1080042464946238122
:108FE000837070F0F3FA611EE21D11F801CFACF14D
:108FF0006103ACF1200C192B98BF81F800C091429D
:10900000F3D104F10A0011F8013FA3F16102203B02
:10901000192A98BF0B708142F5D1182365832D0C56
:10902000E6722373099BA582E361BDE8F88300BF64
:10903000202020002DE9F04FDFF868940C4685B021
:10904000B9F85015D9F84C050D048561002B63D093
:10905000154604F5FE7603EB020B1FE0002D69D0E8
:10906000D9F8FC35AB4200F0CC80D9F8F835AB42EA
:1090700000F0FE80D9F80036D9F80416AB4250D87B
:109080008D42C0F07981691A204663F013FC0135E6
:1090900004F5007406F500765D4539D0D9F8082648
:1090A000AA42DBD8AA1AD9F81876D308396B02F08D
:1090B000070802338B4202D3BA6B93420BD939466D
:1090C0001846039363F0C6FB039B0746002800F095
:1090D0007381C9F818063A79002A40F02481D7F83C
:1090E00028A0BAF1000F00F060813A6B01352046EC
:1090F0004FF400719B1AFA6804F5007406F50076C7
:1091000008EBC3083B4602EB4822D0475D45C5D17A
:10911000D9F84C05B9F850158161002005B0BDE8BB
:10912000F08F8D42AFD24FF400720021204671F0D3
:1091300075FBACE74FF400722946204671F06EFBD8
:109140008023CC4A84F8BE310C2384F8C231D9F88C
:10915000F815D9F8F0359142C4F8C611C4F8CA31EF
:1091600000F30F81C44A013BC44F82FB0102C817C0
:1091700087FB01C70A44C0EB6212C0EB2730C04F27
:1091800087FB02C7C2EB821C84F8C1018010A1EBEF
:109190000C01174420F03F0001310843D117C1EB07
:1091A000E71184F8C0010A4484F8BF21B14A934210
:1091B00000F3F380B04AB14882FB0312D91780FB59
:1091C00003701A44C1EB6212C1EB2031AC4880FB42
:1091D0000270C2EB821784F8C5118910DB1B1044A2
:1091E00021F03F0101331943D317C3EBE01384F897
:1091F000C4111A4484F8C3214AF65523A4F8FE3159
:1092000045E74FF0FF3300274FF4F072201D84F83C
:10921000EC31394684F8ED3184F8EE3184F8EF31E1
:109220005223237063706123A37084F8E7314123D4
:10923000E37084F8E631722384F8E43184F8E53190
:10924000D9F81036C4F8E83171F0E8FA5523C4F8BB
:10925000F07184F8FE316FF05503C4F8F471C4F86E
:10926000F87184F8FC7184F8FD7184F8FF310EE721
:109270004FF400720021204671F0D0FA814B022297
:1092800003CB45F6EB032274227323809023A27351
:10929000A370F82384F82C200822C4F8030062731A
:1092A000C4F807106375D9F8F815D9F8F0355B1ACA
:1092B000D9F800162362D9F804365B1A4AF655210C
:1092C00063620023E372E3736377A377E37784F841
:1092D0002D3084F82E3084F82F3084F831306A4BEA
:1092E000A3613E232377012384F83030802384F860
:1092F0004030664BC4F84230654B84F84620A4F8F1
:10930000FE11644A03CBC4F84B101988C4F8470017
:109310009B78A4F84F1084F8513003CAC4F8520067
:10932000C4F85610B3E64FF400720021204671F0E5
:1093300075FA3B6CB8F1000F45D104F1200A002BFF
:1093400000F081803B6B112253492046CDE9008813
:10935000FFF7F6FD3B6C1A6C002A00F081801B6B56
:10936000504611224D49CDE90088FFF7E9FD04F18F
:10937000400A4FF4E07871E0E91A204663F09AFA67
:1093800085E6FF22013B84F8C1214FF6FF72A4F865
:10939000BF21384A93427FF70DAFFF2384F8C531D0
:1093A0004FF6FF73A4F8C33126E751464FF400721D
:1093B000204671F033FA6AE6231F394A43F8042F36
:1093C0009E42FBD163E6002B7F6C14BF0223012376
:1093D000C3EB0813002F3FF45AAE013BBF6C002BC8
:1093E00001DD002FF9D1A2464FF40078002F3FF4A1
:1093F0004EAE0AEB080303959A460BE00025A8F150
:109400002008CDE900E5FFF79BFDBF6CCFB1B8F1B7
:109410001F0F16D93D7907F11C0E112239683B6BDD
:10942000AAEB0800002DE9D17A79A8F120083D695E
:1094300042F02102CDE900E5FFF782FDBF6C002F6D
:10944000E5D1039D23E6CDE9008843464FF4F0784B
:109450000822D9F8F4152046FFF772FD7F6CC5E7A6
:109460005046434611220D49CDE90088FFF768FDBB
:109470007DE700BFFF03FB0083200882975545412D
:1094800081808080E0690C083F00FF0029940E0D68
:10949000EC690C08F8690C08F4720C08E0740C080C
:1094A000DEADBEEF205A00248C46134601466246CC
:1094B000184641F013BF00BF2DE9F8430D46D0E92F
:1094C000003113448B4220D80446AE18476BCAB112
:1094D0004FF0000900F1100801E0AE4212D0236BFA
:1094E0005A1C23442263202A15F8011B1974F4D155
:1094F0004146204617B9F9F7E9FD0746AE42C4E9EF
:109500000C97ECD13846BDE8F8834FF0FF37F9E708
:1095100000680379012B0AD0022B01D0002070478C
:109520008368F022DB0718D5FF2104F025BA826892
:1095300090F910C002F00102417C60464FF0F00C3F
:1095400010B584B00DF10F040192FF228DF80FC009
:109550000094FAF7A1F804B010BD7F2104F00CBA12
:1095600070B5056884B004460E462B79012B16D0E1
:10957000022B02D0002004B070BDAB68E122DB07F3
:109580001DD52846114604F0F7F90028F2D03246DE
:10959000FF21206804B0BDE8704004F0E3B8AA6879
:1095A000697C02F0010295F910000DF10F0501929E
:1095B000E12200958DF80F20FAF76EF8E5E76121BA
:1095C000284604F0D9F9E0E770B5056884B0044690
:1095D0000E462B79012B17D0022B02D0002004B0AD
:1095E00070BDAB68C3222846DB074CBFE121612177
:1095F00004F0C2F90028F1D03246FF21206804B0FF
:10960000BDE8704004F0AEB8AA6895F9100002F009
:109610000102697C01920DF10F020092C3228DF8C4
:109620000F20E122FAF738F8E4E700BF0068CA43E8
:10963000037941EA0211012BCAB209D0022B01D0F1
:10964000002070478368DB0716D5D22104F094B957
:1096500010B584B0846890F910C08DF80F200DF11A
:109660000F0204F00104417C0092D2226046019472
:10967000FAF712F804B010BD522104F07DB900BF12
:1096800002784368022A0FD00B490269D1F81C0204
:10969000023A184010B4400AD1E9841404FB0200D5
:1096A0005DF8044B08447047034AD2E9812102EB7C
:1096B000410202EB53207047205A00242DE9F04F5D
:1096C00083B002F002077D4D019308B9002F65D1E8
:1096D000D5F80C42002C4FD14FF0FF3E774C4FF0A5
:1096E000000CF146F046F246E36994F82A6098428D
:1096F00000F09580C6B3012E05EB0C1B0AD19BF838
:109700002B60F30706D416F07E0F03D1F60900F0A4
:109710008980E0460CF1010C1034BCF1080FE3D154
:10972000BEF1000F04DAB8F1000FC0F28D80C6461A
:10973000D5F89C4005EB0E1C0EF102060134CCE975
:10974000070405EB061CC5F89C40CCF80440002437
:10975000CCF8084005EB0614A47A042C1ED8DFE8E8
:1097600004F0274119414300E6460CF1010C103486
:10977000BCF1080FB8D1D3E7D5E9843606FB043431
:10978000A042A9D395F8B83113B9012385F8B831AF
:1097900001236B70002003B0BDE8F08F95F8B8315D
:1097A000002B4DD0012302206B7003B0BDE8F08F79
:1097B00012F00104D5F818C06CD105EB0610019B1E
:1097C0004FEAE20C90F80B80032B6CF3C71880F87B
:1097D0000B805DD94FF6FF70834228BF034605EB2F
:1097E00006100381002F41D1500705D505EB061067
:1097F000C37A43F00103C372D30608D505EB0616FE
:10980000F37AC3F34502013262F34603F372AB69A4
:10981000012003EB4E230B6003B0BDE8F08FC6B907
:10982000E64685E7666A1034B24588BFE1460CF12A
:10983000010C88BFB246BCF1080F7FF455AF6FE74B
:10984000012385F8B831ADE7B9F1000FA2DBCE46B0
:109850006EE7D5F89C400CF10206E646013405EBB4
:10986000061CC5F89C40CCF8044073E7D5F8A0006E
:10987000D5F89C3001300133C5F8A00005EB0E107F
:10988000C5F89C30036205EB061304209872ABE721
:109890002346A4E7D5F82036002B3FF47BAF5C6865
:1098A0000CEB4E210023064AA04700283FF472AF7C
:1098B00005EB06160223B3726CE700BF205A0024A2
:1098C000917A040870B5104D82B00E462B78022BA9
:1098D00015D1020AC4B2D5F80402002301A910442C
:1098E0000322FFF7EBFE012807D12B78019A022B08
:1098F0000CBF22F8146042F8246002B070BDC0F3BF
:10990000D41200F07F04E6E7205A00242DE9F04F3E
:10991000434E0D4683B0174631782B6803293DD05E
:1099200002295FD14FEA13294FF4807A5FFA83F856
:10993000421E012A23D84FF0010B9F421AD9012859
:109940008CBF00240124D6F87C211AB1D6F89811D6
:1099500099424AD0D6F804020023092201A94844BA
:10996000FFF7ACFE012822D0022813D020B12B68CB
:109970009F42E8D803202F6003B0BDE8F08FB8F114
:10998000000F12D096F8B83113B9012386F8B83118
:1099900001237370022003B0BDE8F08F4FF0800AFE
:1099A000C3F3D41903F07F08C2E7D346C5E7317883
:1099B000022913D00329EDD1019B53F8282022F06E
:1099C0007042B2FA82F22B685209A2421FD0D844E8
:1099D0005B44D0452B601DD20229EDD1019B33F8A9
:1099E0001820EEE74FF4807ADAE7D6F81412013A3D
:1099F00002EB41224902B2FBF1F21344B3FBFBF24A
:109A00000BFB12320AB15B449B1A2B60B0E79F42FA
:109A1000B2D8AFE709F101094FF00008A8E700BF8D
:109A2000205A00242DE9F04FDFF884918B4685B051
:109A3000174699F800C00968BCF1020FD9F8045222
:109A400040F08280CEB24FF4807305EB1125A6EB77
:109A5000010890449844B94208F1FF38B8FBF3F884
:109A60004AD200F00103A8446FF0404A0193BCF1D0
:109A7000030F07EB0604A8EB0503284614BF4FF4B9
:109A800080728022641A03A9944228BF144694422B
:109A900028BF002E14BF012200220A32FFF70EFE5B
:109AA00001282AD199F800C0DBF800E0BCF1020FD0
:109AB0000EF1010324D0B44255D9039806EB0A02F3
:109AC000011F00EB820201EB840142F8043F8A424D
:109AD00003F10103F9D1DBF80030A11B19448F42D7
:109AE000CBF8001002D1019B002B48D18F4205F129
:109AF00001054FF00006BAD8012005B0BDE8F08F8F
:109B0000B44246D903986FF00042811E324401EB03
:109B1000440100EB420222F8023F914203F10103AB
:109B2000F9D1A11B71448F42CBF80010DED1019B0B
:109B3000002BDBD086466FF000434FF6FF7201200A
:109B400023442EF81320D8E701F07F06C1F3D41385
:109B5000BCF1030FA6EB01081D4414BF4FF4807342
:109B60008023904476E7AEEB060E0EEB04018F42A5
:109B7000CBF80010BAD1019B002BB7D003986FF03F
:109B800040434FF0FF32234440F82320DBF800101D
:109B9000ACE7AEEB060E0EEB04018F42CBF80010E3
:109BA000A4D1019B002BA1D0DDF80CE0C3E700BFDE
:109BB000205A002430B50446C06983B010B9012092
:109BC00003B030BD0D460023032201A9FFF776FD47
:109BD0000128F5D1B4F92020002A19DB019B012DC1
:109BE0004FEA421103EB421203D0022D1AD1E520B5
:109BF0005854A368D3612378032B04D1002313772F
:109C000053779377D377636A190C53839182D6E79E
:109C1000054A92F8B81109B982F8B8010123022067
:109C20005370CDE7E368E5E7205A00242DE9F041C1
:109C3000044682B00D4694F83C30042B7DD8DFE812
:109C400003F02A03684839003D4E4FF6F777DFF8F6
:109C5000F48016E0BA425AD862F01AFF01284FF099
:109C6000000133D1206BFFF72DFE01282ED1019A80
:109C7000D6F81812531E22638B4228BF0B46C6F833
:109C80001832327801A9236B032A18469AB2E1D11F
:109C90004345E1D93BE06900204601F0FE01FFF7B2
:109CA00089FF01283FD1636B002B18BF022084F885
:109CB0003C00C0E794F82830042B02D1002384F83C
:109CC0002830A36B0BB120469847012002B0BDE8B5
:109CD000F0811B4E0021E26AD6F8983106F5BA7081
:109CE000C6F898219B1AD6F8142202FB03F3D6F883
:109CF0007C2102EB4322C6F87C21D6F8802102EBBE
:109D00004322C6F88021FFF755FF01280BD104201C
:109D1000CDE7626B04F130010020FFF783FE0128DC
:109D200001D10320C3E70228D0D194F82830042BB6
:109D3000CCD1002384F82830C8E70220F5E700BF23
:109D4000205A0024F7FFFF0F38B5044694F834304A
:109D5000052B60D8DFE803F031251D130D0394F8BF
:109D60002830082B3FD02D4B0122022083F8B92147
:109D700038BD94F82830082B30D0012038BD0021A0
:109D80002046FFF717FF012845D1042084F834004E
:109D9000DCE7D4E90B01FFF795FD01283BD1032057
:109DA000F4E74FF0FF31206BFFF78CFD012832D133
:109DB000E36A002BF3D00220E8E7184D04F13001EC
:109DC0000120D5F80C220232FFF7A0FD012813D0A4
:109DD0000238C0B201281ED80520D7E70023012091
:109DE00084F82830CAE700230122022084F82830B2
:109DF0000A4B83F8B921BBE7E368D5F81412226B4C
:109E000003EB4123C5F81822C4E90332E36A002BAF
:109E1000BCD16262BAE7002038BD00BF205A0024DE
:109E2000F8B5044694F83830032B4BD8DFE803F03C
:109E300021180B0200212046FFF7BCFE431EDBB2B7
:109E4000012B40D9F8BD0120626B04F13001FFF70E
:109E5000E9FD01284FF00303F0D184F83830E1E741
:109E600000211E48FFF7A6FE01284FF00203F4D0A0
:109E7000E4E71B4BE6681A78D3F81412032AD3F8E8
:109E80007C51D3F8980114BF4FF480728022206176
:109E900002FB01F1871A0244A5EB412506EB41269E
:109EA000E660C3F87C51D3F88051C3F89821A5EB44
:109EB0004121C3F88011E36AC4E90C025BB9606216
:109EC0000123CAE7022094F82830062BBAD10023D8
:109ED00084F82830F8BD2763F2E700BF945B0024C4
:109EE000205A00244368C3F308020A44B2F5007FF5
:109EF0002DE9F041054682B00C4605D223446B6043
:109F0000012002B0BDE8F08190F91A20501C09D060
:109F10004449023201EB0212D17A21F00101D172DF
:109F2000FF22AA7695F91B20511C13D03D4E023218
:109F300006EB0211C97AC1F34501012941D9013962
:109F400001F03F0106EB0212FF26D07A61F34600D2
:109F5000D072EE762A78022AD0D0324ED6F8142269
:109F6000B4EB422F4FEA42282DDCD6F81C721F407A
:109F70007A42A24227DCE2192869424513D32A7E9D
:109F800012072BD5D6F89821411C8A421DD300D147
:109F900000214344A4EB080868610846DB1B08EB7A
:109FA000070429616B600028AAD03278032A33D0D5
:109FB00080B24FF6F7729042A2D81A4614446C60F1
:109FC0009EE70021BEE700209BE796F8B82102BB80
:109FD000012386F8B83173706B68DAE701A962F083
:109FE00057FD0128EFD16B68A4EB08042869984459
:109FF000297868613C44A8EB0703019802291A46B6
:10A000006B602861CFD1D6F82412B3EB412FD5D3A2
:10A0100076E701227270BCE7034A90423FF670AFC8
:10A02000CBE700BF205A0024F7FFFF0F2DE9F047D0
:10A030004FF0010882B0044694F83830032B00F248
:10A04000A580DFE803F055170C020020236C84F88C
:10A05000280003B19847022002B0BDE8F087002233
:10A06000236C84F828200BB120469847012002B0C9
:10A07000BDE8F08723786768022B03D0444BD3F800
:10A080001C321F40C7F34F272046FFF7F9FA404E16
:10A090003F1A0546BFB207EB050C022201A90023B7
:10A0A00028461FFA8CF9FFF709FB01284FF40072CC
:10A0B0004FF00001D0D1019870F0B0FBE3694FF48C
:10A0C000007120460BB16368EBB1D6F814325A1E0A
:10A0D000914547D20135FFF705FF0028DBD196F8FF
:10A0E000B83113B9012386F8B83186F80180D2E778
:10A0F0002046FFF729FE012802D0022846D103207E
:10A1000084F8380098E7019B4FF020324FF0100E92
:10A110004FF02E0C42F62E6AC3F80120C3F805203A
:10A12000A3F8092083F800C0D4F824C0A3F820A025
:10A1300083F80BE0C3F82220C3F8262083F82A20F6
:10A14000E26BA3F81AC02CFA0EFC5A8722FA0EF220
:10A15000A3F814C09A8683F82BE0D6F814325A1E5E
:10A160009145B7D3C3EBC3532046590201F50071A3
:10A17000FFF7B8FE20B996F8B8311BB10123737010
:10A180000220BDE7012386F8B831F7E7002063E736
:10A19000205A0024B1F904300F2B2DE9F0410D466F
:10A1A00082B00446164631D02046FFF769FA94F98A
:10A1B0001B80B8F1FF3F3AD0584F07EB0813DB691B
:10A1C000984211D097F8B831002B6BD001237B70E7
:10A1D0002378022B5CD02269002A71D10023012050
:10A1E000336002B0BDE8F081B96901EB4821002974
:10A1F00064D0AB88204601331BB201EB4311AB8026
:10A200003160FFF73DFA28600120EAE74FF4007162
:10A21000FFF768FE002841D04FF6FF732046AB8061
:10A22000FFF72EFA94F91B80B8F1FF3FC4D12378D1
:10A23000022B3BD02269002AD0D0384F3B78032B29
:10A2400062D093B24FF6F7718B4294BF0023012383
:10A25000002BC1D128B997F8B831002B47D0012382
:10A260007B700023112201A9FFF728FA012825D1CC
:10A270000199BB69CB1A48BF03F2FF13B3F5805FA6
:10A280004FEA63222AD24FFA82F884F81B80AEE7A5
:10A29000D7F824226368B3EB422F9FD2002002B08C
:10A2A000BDE8F081012387F8B8318FE71B4F636861
:10A2B000D7F82422B3EB422FCCD38FE7237888E75B
:10A2C0003B78032B17D093B24FF6F772934294BFAB
:10A2D00000230123002B81D10020E0E797F8B8315B
:10A2E00013B9012387F8B83101237B70CDE701232F
:10A2F00087F8B831B3E70A4B9A4294BF0023012391
:10A30000002B7FF46BAFE7E7054B9A4294BF002325
:10A310000123002B7FF460AF9CE700BF205A00248C
:10A32000F7FFFF0F70B50378044690F818C0023BA2
:10A33000012B02D91CF0060F66D11CF0200F3FD173
:10A3400094F91A30591C09D0364A0233FF2102EB26
:10A350000313DA7A22F00102DA72A17694F91B3043
:10A360005A1C13D02F48023300EB0312D27AC2F3E7
:10A370004502012A45D9013A02F03F0200EB0313DE
:10A38000D97A62F34601FF22D972E2761CF0080FF7
:10A390000DD0244890F89C31072B05D090F8B831A7
:10A3A000002B39D001234370002380F89C31002317
:10A3B000E26A237084F828302AB3BDE87040104761
:10A3C00018480023E5690246D16910328D4206D053
:10A3D0000133082BB4D0D16910328D42F8D1023349
:10A3E00000EB0312D27AC2F34502012A18D9013ACE
:10A3F00002F03F0200EB0313D97A62F34601D972EF
:10A400009EE70022BAE770BD0121FFF7D3FB0128C8
:10A41000F9D194F818C090E7012380F8B831C1E76A
:10A420000022E7E7205A002438B5194C94F8E431AB
:10A430002BB970B190F828201AB1184638BD002009
:10A4400038BD0146442204F5DE706FF0BFF80120EC
:10A4500038BD04F5DE7501464422284670F0DEF969
:10A46000237803224FF6FF71022B2846A4F8D61159
:10A4700018BF1346D4F8201284F8D421102284F88F
:10A48000BC31C4F8E01184F8D52163F0FFFCDEE7AD
:10A49000205A0024F8B54FF0FF312C4C00232246FF
:10A4A0000D4603E001331032082B14D092F82A0035
:10A4B0000428F7D104EB031090F82B00C707F1D460
:10A4C0006E1C106A01D08142ECD91D460133014651
:10A4D0001032082BEAD1002D01DA0120F8BDAE1CA4
:10A4E000D4F8202604EB06131989D1B92F0127448B
:10A4F000A169D4F82036F86901EB4521CBB1DD68BC
:10A500000023134AA847A0B1022808D1D4F8A030EC
:10A5100004EB06160122013BB272C4F8A030002001
:10A52000F8BD04EB05132F01D86912B19368984761
:10A53000DDE7D4F8A03004EB061603210122013B2D
:10A54000B17284F8A420C4F8A030E8E7205A0024AF
:10A55000ED7A0408704700BF0369416853EA0102BD
:10A56000F0B43B4E5DD0C56A013390ED067A6A1CAB
:10A57000876830EE077A0361012AC26280ED067AAD
:10A5800042D090ED075A07EE902AD0ED096A70EE9E
:10A59000455A3468B8EEE76A611AC5EE867AB94260
:10A5A00077EE857A30EE670AC0ED087AC0ED077A5B
:10A5B000F0EE667AE5EE807AC0ED0A7AC0ED097AAF
:10A5C00001D8F0BC7047012A28DD06EE905AF8EE5B
:10A5D000E66A87EEA66AB5EEC06AF1EE10FA1DDBF8
:10A5E000F1EEC67AF4EE677AF1EE10FA16D6D0EDF7
:10A5F000056AF4EEE76AF1EE10FA15D5037BFBB1BC
:10A600000323F0BC03707047326880ED080A521AC9
:10A61000002180ED070ABA424162D2D9DFED0D7AFE
:10A62000E5E7316841609EE707EE903A0223F8EED5
:10A63000677A0370F0BCC7EE276AC0ED066A704700
:10A64000316800220361C36241608261B9E700BFE3
:10A65000AC2F00240000000010B5DFED4F4A844607
:10A6600000F1480E0346DA6AB1EC017AD3ED067ABE
:10A67000013277EE877A012ADA62C3ED067A71D069
:10A6800093ED075A07EE902A93ED096A77EE455A43
:10A69000F8EEE77AC5EEA76A76EE857AF0EE466ABE
:10A6A00037EE677AC3ED087AE5EE876AC3ED0A6A8A
:10A6B000C3ED077A1833C3ED036A7345D3D1374C22
:10A6C000416822680369521A816801338A42036132
:10A6D00047D990ED056A0022DFED2F5ADCF82C10E7
:10A6E000F0EE657ADCED0A6A012901F1FF3E11DD29
:10A6F00007EE90EAF8EEE77A86EEA77AB5EEC07A32
:10A70000F1EE10FA45DBF1EEC77AF4EE677AF1EE7E
:10A7100010FA3ED6B4EEE76A01320CF1180CF1EEF5
:10A7200010FA26D4022AD9DDB4EEE76AF1EE10FA67
:10A730001FD407EE903AD0ED066A90ED0C7A022312
:10A74000F8EE677AD0ED125A037086EEA76AC7EE6C
:10A75000276A85EEA77A80ED066AC0ED0C6A80ED67
:10A76000127A10BDF0EE477A83ED087AF0EE646A53
:10A770009EE7037B13B10323037010BD0022216801
:10A780000361C36241608261026343648264C365A2
:10A7900010BDDFED017ABDE700000000AC2F002402
:10A7A000B0EEC06AF0EEE05AF0EE407AF4EEC65A2F
:10A7B000F1EE10FA0EDCB5EE400AF1EE10FA4AD0D6
:10A7C000F4EEC65AF0EE466AF1EE10FA4FD5B0EE4E
:10A7D000655A03E0F0EE656AB0EE465A85EE267AD9
:10A7E0009FED242A9FED243A9FED244ADFED244A71
:10A7F000DFED242ADFED243AB7EE005ADFED236ABD
:10A80000F4EEC65AF1EE10FAA7EE023AE7EE223A5B
:10A81000A7EE034AA7EE235AE7EE044AE7EE246ABE
:10A82000B1EE667A87EE050A10D4F5EEC00AF1EEB5
:10A8300010FA03D59FED167A37EE400AF5EEC07A8E
:10A84000F1EE10FA48BFB1EE400A70479FED117A61
:10A8500037EE400AE9E7F5EEC00ADFED0F7A9FED2B
:10A860000F0AF1EE10FA58BFB0EE670A7047B0EE6B
:10A87000465AB3E739094E3DE3B59EBE88FA16BE87
:10A8800045FE7FBF99FB243F69A2163EA7DFA8B40F
:10A89000DB0F4940DB0FC93FA7DFA834DA0F49407F
:10A8A000D1ED007AF7EE002AD0ED043A90ED054A9A
:10A8B000E7EEA73AD0ED064A90ED075AD0ED085AD8
:10A8C00090ED096AD0ED0A6A90ED0B7AC0ED043A7A
:10A8D00091ED003AD1ED013AD0ED0C7AA3EE234A86
:10A8E00080ED054AD1ED003A91ED024AE3EE844A4B
:10A8F000C0ED064AD1ED004A35EE245A80ED075AE4
:10A90000D1ED014A91ED005AE4EE855AC0ED085AA6
:10A91000D1ED015AA5EEA56A80ED096AD1ED015A83
:10A9200091ED026AE5EE866AC0ED0A6AD1ED016A30
:10A9300037EE267A80ED0B7AD1ED026A91ED007A3E
:10A94000E6EE877AC0ED0C7A91ED027AD1ED017ACC
:10A9500090ED0D3AD0ED0E3AA7EE273A90ED0F4A62
:10A96000D0ED104A90ED115AD0ED127AD0ED135A75
:10A9700090ED006A80ED0D3A75EEA25A91ED023A23
:10A98000D0ED016AE3EE033A90ED027AC0ED0E3AA3
:10A99000D1ED023A34EE234A80ED0F4A91ED004AA0
:10A9A00074EE844AC0ED104AD1ED014A35EE245AC6
:10A9B00080ED115A91ED025AC0ED135A77EE857A67
:10A9C000C0ED127AD1ED017AD1ED005A67EEA77A87
:10A9D00091ED025AE5EEA57AE5EE057AA5EEA76AB5
:10A9E00080ED006A91ED016AE6EE276AC0ED016A2A
:10A9F000D1ED026AA6EEA77A80ED027A90ED037A95
:10AA000077EE277AC0ED037A704700BF2DE9F04F4B
:10AA10004FF00009864600F110050646034689B04E
:10AA200000F13008074648462C468B469C46B24605
:10AA3000CDF80CE000283CD10CF1040CA445FBD16E
:10AA4000032800F1010151D09C46AA46029398B117
:10AA5000DCED047AAAEB0903B64601927246F3ECE8
:10AA6000016A0EF1100E92ED007A5345E6EEC77AB8
:10AA7000CCED047AF2D1019ADCED046A0CF1100CF1
:10AA800015ED047A0AF1100AC445C6EE877ACCEDBA
:10AA9000007ADCD1029B0436084608F1040814331E
:10AAA00014351034103709F104099C46B2460028C9
:10AAB000C2D0DCED007AD646394601927246F1ECFE
:10AAC000016A0EF1100E92ED007A9942E6EEC77A15
:10AAD000CCED007AF2D10CF1040C019A0AF1040ACF
:10AAE000A445E6D1032800F10101ADD1DDF80CE069
:10AAF0000023594604AD764677460020049305931B
:10AB000006930793F2EC017AE5EC017AB0B104AC5C
:10AB10003B46B4EC017AF3EC016AE6EEC77AB34245
:10AB200045ED017AF5D1013004280BD0F2EC017A21
:10AB300010371436E5EC017A0028E8D110371436C6
:10AB40000120DFE708AD10310EF1400E042875ED4D
:10AB5000017AA1F10402744641ED017A1ED07346D8
:10AB6000F3EC016AB1EC017AA342E6EEC77AC2EDDA
:10AB7000007AF5D15EED016A013887EEA67A82EDA2
:10AB8000007A17D0AEF1140E103C114675ED017A23
:10AB90000428A1F1040241ED017AE0D15EED016AE1
:10ABA000103CAEF1140E032087EEA67A01ED017A77
:10ABB0001146EBE709B0BDE8F08F00BF60EEA00AD8
:10ABC000E0EE000AF5EEC00AF1EE10FA07DBB1EE96
:10ABD000E00AB4EE400AF1EE10FA00D670479FED9D
:10ABE000010AFBE70000000060EEA00AE0EE000AA8
:10ABF000E1EE010AF5EEC00AF1EE10FA07DBB1EE64
:10AC0000E00AB4EE400AF1EE10FA00D670479FED6C
:10AC1000010AFBE700000000DFED297AB4EEE70A45
:10AC2000F1EE10FA28DD9FED277A30EE470AB4EEF8
:10AC3000E70AF1EE10FAF8DCDFED237AB4EEE70A6A
:10AC4000F1EE10FA2FDD30EE670A37EEC00A60EE43
:10AC5000007ADFED1E5A9FED1E6ADFED1E6AA7EE39
:10AC6000A56A9FED1D7A60EE275AE7EE866AA7EE89
:10AC7000A67AA5EE870A7047DFED187AB4EEE70AE8
:10AC8000F1EE10FAD8D59FED0F7A30EE070AB4EE48
:10AC9000E70AF1EE10FAF8D4DFED0B7AB4EEE70A2A
:10ACA000F1EE10FACFDC9FED0E7AB4EEC70AF1EEAA
:10ACB00010FACCD530EE270A37EE400AC7E700BFBE
:10ACC000DB0F4940DB0FC940DB0FC93F9A7C2E36B2
:10ACD000FAAF4FB93587083CA4AA2ABEDB0F49C09A
:10ACE000DB0FC9BF10B5404CB4FBF2F4A14219D33D
:10ACF000DFED3E7AF7EE005AB0EE677AB0EE676AA3
:10AD0000F0EE676A0023C0ED005AC0ED017A80EDD5
:10AD1000027A80ED036AC0ED046A836143610362D5
:10AD2000C36110BD07EE902ADFED315AB7EE006A1D
:10AD3000DFED306AB8EE677A07EE901AB0EE405A4F
:10AD4000F8EE677A27EE257A67EEA67AC6EE076AEE
:10AD5000C7EEA64AFDEEE47A17EE902A2032402A8A
:10AD60003FD8B0EE640AFFF757FFB0EE404ADFED80
:10AD7000227A34EEA70AFDEEC07A17EE902A20322E
:10AD8000402A29D8FFF748FFF8EE006A60EE266AED
:10AD9000012B1CD0B7EE006AF6EE004A36EE406A90
:10ADA00066EE244A35EE055AF7EE007A84EE057A0F
:10ADB00077EE275A37EEC75A84EEA57AC6EE257A83
:10ADC00086EEA56AC5EE256AF0EE475A9AE7F7EED9
:10ADD000004AB0EE666AE5E7DFED086A9FED030A18
:10ADE000D6E79FED024AC2E720A10700000000005D
:10ADF000BD378635DB0FC940DB0FC93F000000803F
:10AE0000DFED077A30EE270AFDEEC07A17EE903AB2
:10AE10002033402B00D8FFE69FED020A704700BFA9
:10AE2000DB0FC93F000000002DE9F84F9DF82840D6
:10AE30008946DDF82CB00546002C17461BF8011B8F
:10AE40000CBF4FF020084FF030081C1E08463ADBBC
:10AE500000295CD0002C53D04FF0000A5B4600E084
:10AE600064B313F8016B013C002EF9D1BAF1000F65
:10AE70002FD1264644B14D454146284600D2B84719
:10AE8000013CF8D10B9B18780146A0B14FF0FF347C
:10AE90004FF0000A00E09B464D45284600D2B847D7
:10AEA0005B4613F8011B0029F5D10B9BF61A5E4493
:10AEB000BAF1000F10D13046BDE8F88FBAF1000F9B
:10AEC0001BD15646E0E7634229B31C464FF0010A06
:10AED000C4E70028E0D10646002C04F1FF3AEADD81
:10AEE00054464D454146284600D2B847013CF8D269
:10AEF000013656443046BDE8F88F30B12646CBE7E0
:10AF000026464FF0FF34B246C6E70646D3E726464C
:10AF1000002CB0D1CFE76FEA040A0E46E0E700BF8D
:10AF20000FB430B583B00C4C06ABD4F8B018D4F8DD
:10AF3000AC0853F8042B019362F00AFE0546D4F8DE
:10AF4000240603685B6998470028F8D0284603B0B8
:10AF5000BDE8304004B07047205A00240EB410B54C
:10AF600083B00446084905AB01A853F8042BCDE98A
:10AF7000003462F0EDFD0022019B1A7003B0BDE8C1
:10AF8000104003B0704700BFB17D04080CB470B529
:10AF9000334CA4B0D4F8B438002B5BD094F8BC3850
:10AFA00099420AD90123D4F8C0288340134204D11E
:10AFB00024B0BDE8704002B070472A4B4FF47A715C
:10AFC000294A1B68A2FB030204A8920901FB123361
:10AFD0002649FFF7C3FF04AA29AB254902440646C8
:10AFE00003A802930392289A62F0B2FD039B0A22FF
:10AFF000D4F8B458591C03911A700022039B591CB1
:10B0000003911A70ADB12B681B6A1BB12846984793
:10B01000D4F8B4589DF810100029C9D00DF11104CE
:10B020002B6828461B68984714F8011B0029F7D1A4
:10B03000BEE7D4F8B838002BBAD03044022404A9B3
:10B0400002190094FD2032F045F924B0BDE87040AB
:10B0500002B07047D4F8B838002B9FD1A8E700BFE2
:10B06000205A0024AC2F0024D34D6210046A0C082F
:10B07000A57D0408184A033010B5D2F8C44804EB83
:10B080009003B3F5007F19D8C2F8C43802F6C8029D
:10B0900020F00300C3F5007302EB84040F4A9B0009
:10B0A00002EB810151F8302C10440D4A41F8300C6C
:10B0B00004210020FFF76AFF204610BD0021094A45
:10B0C00000240846FFF762FF044A2046936D43F0D0
:10B0D0000073936510BD00BF205A0024186B002434
:10B0E000106A0C08346A0C0803681A46591C01607F
:10B0F00012F8021B0260587841EA0020704700BF36
:10B1000002681346511C016013F802CB0360D31C84
:10B110005178036093781B0443EA0123111D43EA2D
:10B120000C030160D07843EA0060704712B370B539
:10B130000446864604E0981B17D114EB0C0C15D07E
:10B140001EF8013BA3F14100A2EB0E0C192811F8E7
:10B15000010BA0F1410598BF203300F12006192D05
:10B16000E9D91B1A04D10028E7D170BD604670BD33
:10B17000184670BD1046704703880021194A30B543
:10B1800003F0030E90F802C0174CA3F5FA630EEB20
:10B190004E0E0CF1FF3C40F2B5550CEB8E0C04EB5F
:10B1A0004C044FEA930C238A847905FB0C3390F806
:10B1B00003C022444FF47A740CF1FF3C634490F8CE
:10B1C00004C003EB43030CEBC30C43790089CCEBC5
:10B1D0000C1C03EB8C03C3EB031302EB8302C2FBD7
:10B1E000040130BD80436D38A4BC0B08F8B5164689
:10B1F0001F463F4D0446394630464FF47A720023CD
:10B2000068F008F83B4B05443B4F3C4E83FB051070
:10B21000E9172844C1EB601183FB0103C8170B44F5
:10B22000C0EB631087FB003CC317C3EBAC0386FB8A
:10B2300003764FEAE37ECEEBE61EC1EB0116A5EBEB
:10B24000860CC0EB00154FEA8E0684F806C0A1EB11
:10B250008501617103EB4301A0EBC10040F2B551E0
:10B2600001FB1E332071B3F5896F35DA40F2DA2124
:10B270008B4237DCB3F5B77F2149B4BF4FF0000EE6
:10B280004FF0010E0EEB4E0075464FEA4E0701EBF4
:10B29000C001C88C1B4907EB0E0C01EBCC0C0B2139
:10B2A0000CF1160C01E03CF8020D984211DD013959
:10B2B000F9D17744124901EBC701088A012106F54B
:10B2C000FA6E0133A17075441B1A22812580E37048
:10B2D000F8BD0131C9B2F2E7032540F296500627C6
:10B2E000AE46D7E7022540F229400427AE46D1E713
:10B2F00080BC92C789888888ABAAAA2A73B06D16C9
:10B30000A4BC0B08B4BC0B0830B5304C8DB08646DD
:10B310000D46EC461EF0030F0FCCACE80F000FCC2F
:10B32000ACE80F0094E80F008CE80F000FD1284B19
:10B33000284A03FB0EF3B2EBB30F44D3264AB2EB19
:10B34000331F34BF01220022C2F11D0200E01C2283
:10B350000EF1FF33019240F26D122048002B194686
:10B3600002FB0EF21E4CB8BF0EF10201EE4602EBDC
:10B37000A10280FB0310DB17ADF1040101EB850195
:10B38000A3EB6015C3EBE0132A441A44253284FB77
:10B390000230D3171044C3EBA003C3EBC303D31A8B
:10B3A0005EF8040FC218714584FB023C4FEAE27359
:10B3B0009444C3EBAC03C3EBC303A2EB0303EFD191
:10B3C000C01A0DB030BD1D22C2E700BF14BD0B086E
:10B3D000295C8FC2285C8F020AD7A3001F85EB511E
:10B3E000932449920D4B10B5D3E9184354EA030254
:10B3F0000AD10146002340F2011218460B80C1F821
:10B4000002208B710B8110BD054A1268121943F19D
:10B410000003FFF7EBFE012010BD00BF186B0024F6
:10B42000AC2F002430B5134D83B00446D5E9181372
:10B4300051EA03020AD1002340F201121846238088
:10B44000C4F80220A371238103B030BD0A4A1268F8
:10B45000521843F10003FFF7C9FEB5F868302046E3
:10B460000DF106022146ADF8063061F071FA0120B7
:10B4700003B030BD186B0024AC2F00242DE9F04739
:10B48000044688B094F83030042B11D8DFE803F07C
:10B490004C135D035600237E9A0640F1F080002392
:10B4A000112204A9E069FEF709F9012800F0E780FC
:10B4B00008B0BDE8F087C94D03AE04F11C0705F5DF
:10B4C000DE79324639464846FEF764FE012800F030
:10B4D000F1800228ECD195F9D6315F1C09D00233F6
:10B4E000FF2205EB031385F8D621DA7A22F0010258
:10B4F000DA7295F9D7315E1C14D0023305EB0312D2
:10B50000D27AC2F34502012A40F25081013A02F098
:10B510003F0205EB0313D97A62F34601FF22D97289
:10B5200085F8D721042306E0AD4862F0AFFC4FF662
:10B53000FF720123228484F83030A3E70020E36AFD
:10B54000207008B0BDE8F0471847A44D95F8E431E5
:10B55000002BADD104F11C0703AE05F5DE783246B1
:10B5600039464046FEF716FE012840F00D81039B48
:10B57000002B00F0E8801A780AB1E52AEFD1AA6919
:10B580009A1A48BF02F2FF12B2F5805F4FEA6221B9
:10B5900080F041810901934A0A44917B04290CD02F
:10B5A000D5F89C100131C5F89C10516004219173AD
:10B5B000D5F8A0200132C5F8A02095F9D621501C5D
:10B5C00009D0023205EB0212D17A21F00101D172C9
:10B5D000FF2285F8D62195F9D721511C14D00232CB
:10B5E00005EB0211C97AC1F34501012940F25681E8
:10B5F000013901F03F0105EB0212FF2085F8D70168
:10B60000D07A61F34600D0722022002118466FF0F4
:10B6100005F9D4F831100346D4F8352005A819608F
:10B620005A6094F83B20B4F839109A721981627EFE
:10B630000193DA72FFF7F6FE019B002800F0D48038
:10B640009DF816009DF817209DF8191042EA401247
:10B65000BDF814004901A0F2BC7042EA40229DF8F6
:10B660001A0041EA50019DF8180092B241EAC02147
:10B6700088B2D9811A821A83D88203235BE72046D5
:10B6800062F004FC2369002B00F08380237E03F02A
:10B69000F70213F00403227640F08A80122A00F0A9
:10B6A000A6800022E36A204684F8282008B0BDE87E
:10B6B000F0471847DDF80C80B8F1000F00F0B680B5
:10B6C00098F80030002B00F0B18098F80BA01AF029
:10B6D000080F7FF4F6AE0B2204F1310140466DF005
:10B6E000F1FE00287FF4EDAE637E8AEA0303DF06F5
:10B6F00040F1D88095F9D6315E1C09D00233FF2184
:10B7000005EB031385F8D611DA7A60F30002DA72DA
:10B7100095F9D721511C3FF405AF023205EB021316
:10B72000DB7AC3F34503012B40F2FB80013B03F0BE
:10B730003F0305EB0212D17A63F34601FF23D17276
:10B7400085F8D731EEE695F8BC310922022B3FF49B
:10B75000E9AE95F8E431002B7FF4E4AE85F8F431DE
:10B7600085F8F0311E4885F8E421C5E97E33D5F827
:10B77000D031C5F8E831D5F81832C5F8EC31FEF70C
:10B7800055FC01283FF4EBAE02287FF491AE042370
:10B79000D1E6237E1B0784D5104B93F89C21002A09
:10B7A0007FF486AE072283F89C217AE70022B0E678
:10B7B0000023A5682046E66A294684F82830FEF76B
:10B7C00091FB002864D194F82830002B7FF470AEF0
:10B7D0000223C4E90B6584F8283069E6205A002466
:10B7E000DC5B00243C5A002444F2817242E7E06AA8
:10B7F0000421626AA063204684F83C3084F8281053
:10B8000063636362C4E90B22C4E9023308B0BDE894
:10B81000F04762F03BBB95F8B82112B9012285F8D8
:10B82000B82101226FF00F016A70B4E695F9D631A4
:10B83000591C09D00233FF2205EB031385F8D621EA
:10B84000DA7A22F00102DA7295F9D7315A1C13D054
:10B85000023305EB0312D27AC2F34502012A1FD943
:10B86000013A02F03F0205EB0313D97A62F3460175
:10B87000FF22D97285F8D721237EDB067FF552AEF1
:10B880002A4862F003FB4FF6FF720223228452E63D
:10B89000002E3FF40DAE2046334652E60021AAE6C4
:10B8A0000022E0E7B8F81420B8F81A3043EA02435F
:10B8B000D5F8142263625202D8F81C30B3FBF2F1BF
:10B8C00002FB1131A36009B113445B1AE36084F8F1
:10B8D00019A095F9D6315A1C09D00233FF2205EB85
:10B8E000031385F8D621DA7A22F00102DA7295F98B
:10B8F000D721531C3FF4C1AE023205EB0213DB7AB1
:10B90000C3F34503012B0ED9013B03F03F0305EBC5
:10B910000212D17A63F34601FF23D17285F8D73141
:10B92000ABE6002305E70023F1E700BFDC5B002462
:10B930002DE9F04390F8283083B00446013B082BF2
:10B940000BD8DFE803F0393D1F24052A0A2F340005
:10B950000121FEF76BF9012802D003B0BDE8F083A6
:10B9600000222378216C84F82820002BF5D00322B4
:10B97000E162D4E9010384F82820834238BF0346FA
:10B980002046A36003B0BDE8F043FEF7CBBC002126
:10B9900003B0BDE8F043FEF749B903B0BDE8F0439A
:10B9A000FEF73EBA03B0BDE8F043FEF7CDB903B0F1
:10B9B000BDE8F043FEF73ABB03B0BDE8F0435DE5F8
:10B9C000DFF830914368D9F81C62026B19461E40BB
:10B9D000D9F8140294F800C0B5184702B5EB402F0F
:10B9E00041D34FF6F778BCF1020F14D025692846F1
:10B9F000002D5AD16168A3680020E26A8B4284F866
:10BA0000280038BF0B46A360002AA6D0204603B00A
:10BA1000BDE8F04310476168D9F82402B1EB402F2C
:10BA20005CD22069217E090732D5D9F89811451CCE
:10BA3000A9422AD299F8B811002943D1012389F8E3
:10BA4000B83189F80130226B636894F800C0D21BCA
:10BA50003B4432449B1B0026974219466360226395
:10BA6000C4E90450BFD9BCF1020F37D02569002DBD
:10BA7000C1D099F80030032B36D0ADB24FF6F77332
:10BA80009D42B8D811446160B5E7E0D10025DEE7FA
:10BA900001A960F0FDFF01287FF45FAF2069019DDF
:10BAA00094F800C06368226BD1E799F8001003296D
:10BAB0000ED0A9B2414594BF002101210029B1D087
:10BAC0006168D4E7012189F8011094F800C0BEE74D
:10BAD00007498D4294BF00210121EFE7D9F82432B4
:10BAE000B1EB432FCED386E7014B9D4283D8C9E704
:10BAF000F7FFFF0F205A002488422DE9F0419846B5
:10BB00004FF0010439D301FB04F4B0FBF4FC8C4585
:10BB1000F9D264B30025BCF1000F04FB1C00B4FB98
:10BB2000F1F7D4BF002601266DB966B9A1423546AA
:10BB300019D9C6460CF1300C0EF801CB00238EF853
:10BB40000030BDE8F081BCF1090F18DD002A0CBF00
:10BB500057233723C6466344A14205F101050EF879
:10BB6000013BF046EAD83C46B0FBF7FCD3E7C646BB
:10BB700000238EF80030BDE8F0818446CAE7302308
:10BB8000E8E700BF2DE9F041044615460846944217
:10BB9000B4FBF2F607D205FB1644134B1B5D00F80D
:10BBA000013BBDE8F0819642B6FBF2F70CD20E4B9A
:10BBB00005FB176705FB1644DA5D1B5D00F8012BDA
:10BBC00000F8013BBDE8F081BA42B7FBF2F807D9B3
:10BBD00005FB1878044B13F8082000F8012BE7E761
:10BBE0004046FFF7CFFFF3E7446A0C08B5EEC00A02
:10BBF000DFED357A0023F1EE10FA30B5C8BF30EE34
:10BC0000270A87B0D8BF30EE670ADFED307A0546E5
:10BC100003A9029320EE270ACDE90033FDEEC07A96
:10BC200017EE904A84EAE470A0EBE47061F02EFF16
:10BC3000002C03A8B4BF2D2320238DF8003066F01C
:10BC4000F7FC01282AD0022834D003281ED003A9EB
:10BC500068466FF09BFC684666F0EAFC044669465D
:10BC60002846033CE4B222466DF0B0FC002328468F
:10BC70002B5566F0DDFC2E22431C0DEB04012A54EB
:10BC8000E8186FF0F8FC284607B030BD302303A950
:10BC900068468DF801306FF079FCDCE743F2300242
:10BCA000302303A96846ADF801208DF803306FF00A
:10BCB0006DFCD0E743F2300303A96846ADF80130CC
:10BCC0006FF064FCC7E700BF6F12033A00007A44CC
:10BCD0000378202B03D110F8013F202BFBD0092B38
:10BCE000F9D02D2B63D02B2BB7EE000A08BF013003
:10BCF0000278A2F13003D9B2092961D8F2EE046AC0
:10BD0000DFED4D7A07EE103A10F8012FB8EEC77A42
:10BD1000A2F13003D9B2A7EEA67A0929F0EE477A4C
:10BD2000F0D92E2A50D0037803F0DF03452B3BD106
:10BD300010B442782D2A73D02B2A62D0A2F130039E
:10BD40000130092B63D80024002303EB830302EBAB
:10BD5000430310F8012FA2F13001303B0929F4D937
:10BD6000B3F59A7F1A46B7EE007A28BF4FF49A725D
:10BD7000072B09D91346DFED316A083B27EE267AF7
:10BD8000072BFAD802F007022AB1F2EE046A013A50
:10BD900027EE267AFBD1002C3BD0C7EE877A5DF8E0
:10BDA000044B20EE270A704720EE270A704742789E
:10BDB0000130BFEE000AA2F13003D9B209299DD9A2
:10BDC0002E2ADFED1D7AAED143780130A3F1300287
:10BDD000D1B20929A8D8B2EE047AF0EE475A06EE9D
:10BDE000902A10F8013FB8EEE66AA3F13002D1B212
:10BDF000C6EE076A092927EE257A77EEA67AEED9EC
:10BE000092E782780230A2F13003092B9BD9B7EE7A
:10BE1000007A67EE877A5DF8044B20EE270A7047B8
:10BE200082780230A2F13003092B01D801248BE77C
:10BE3000B7EE007AB1E700BF0000000020BCBE4CA6
:10BE40000378092B01D0202B05D110F8013F202BBE
:10BE5000FBD0092BF9D02D2B09D001784FF0010C24
:10BE6000A1F13002D3B2092B0AD9002070474178E2
:10BE700001304FF0FF3CA1F13002D3B2092BF4D8CE
:10BE8000002310F8011F03EB830302EB4303A1F12E
:10BE90003002D1B20929F4D90CFB03F0704700BF7E
:10BEA0002DE9F04F91B03FF04FFA3FF039FAB0F181
:10BEB000000A40F338810024DFF80493B34D27468D
:10BEC0002646A04604E006F50066B24540F394809D
:10BED000202230460DEB02013FF000FA1222AC495D
:10BEE00008A86DF0EFFA83460028ECD1BE4222D0BC
:10BEF00008EB4802A74B08F10108A74903EB8203AE
:10BF0000424618460193F31B0293FFF727F84A466F
:10BF1000019B42F84C3B029BC9F80C70C9E9043301
:10BF2000D9F81C30C9E908330123C9F808309B4B04
:10BF3000C9F8283091469A4B37461222D3F88C30F4
:10BF4000C9F81C3002F1400301320DEB03012B5DF7
:10BF500011F8201C99420BD00024202AF2D120375E
:10BF600008A9BA4538463EDB3FF0B8F90022E9E7B8
:10BF70000134152CF1D1D01920220DEB02013FF034
:10BF8000ADF9884908A807AA6DF0F5FA58B300235F
:10BF9000CDF814B01F469B46CDE90133CDE90333FC
:10BFA0007B1E042B00F2B081DFE803F05E4F666277
:10BFB0000300CDF814B0FFF743FF059B83460499B7
:10BFC00089B15B01A1F2BC71DDE9022042EA4012B5
:10BFD000019843EAC02342EA412243EA6B0343EA61
:10BFE0000243C9F81C30B8F1640F49D0374606F552
:10BFF0000066B2453FF76CAFB8F1640FC3461DD081
:10C00000BE421BD00C23634C08F1010B624903FBB9
:10C010000844F61B5A462046FEF7A0FF5F4BC9F8BE
:10C020000040C9F82830D9F81C30C9F81460C9E9B3
:10C0300008330123C9E90376C9F80830BBF1000FC2
:10C040000BF104011EDC584C4AE0FFF7F9FE0290A8
:10C0500007AA5449002001376DF08DFA00289FD1BE
:10C060005B46DDF814B0AAE7FFF7EAFE0390EFE7BE
:10C07000FFF7E6FE8346EBE7FFF7E2FE0190E7E716
:10C08000C3466821484C4C27454B4FF0010907FB3C
:10C0900001F5D4F84C613A460021C3F88C6063196D
:10C0A000DFF8148118466EF0B9FB3A4600213B4F89
:10C0B0006EF0B4FB3D4A0BF10501625105F110022F
:10C0C000C0F808901835C0F82080876244F802A0B4
:10C0D0002244C2F804A0221D565115446E604662E7
:10C0E0004FEA4A032E4AB3F1805FD2F88C501FDB2F
:10C0F0004FF498722E492C486DF068FA2D4BA3F13D
:10C100001C0203F598719D60C3E900554C338B42C6
:10C11000F9D1A06820B9237913B12368002B53D13A
:10C1200011B0BDE8F08F1E4B04211F4CD3F88C508A
:10C130004C274FF00108DFF88CB04FF0020907FBE5
:10C1400001F63A460021A31918466EF067FB3A46FD
:10C150000021194F6EF062FB44F806B0034680F8E8
:10C160000590C0F80880CAF1006006F1100206F1DF
:10C17000180100FA08F0C3E90777A0502244506084
:10C180000E4A555011444D605D62B1E7906A0C084B
:10C190006C6A0C08846B0024806A0C08A99404085B
:10C1A000CC180024A86A0C0860DD0024B06A0C08D2
:10C1B00044BD0B087CDD00240068994F64DD002439
:10C1C00090DE0024C06A0C080026002750499646DD
:10C1D000A064E063C4E9106706460746CD6C01F130
:10C1E0004C035DB39D6806F1FF3C9F646545C1E962
:10C1F0002377DF630DD006F1010C65450ED113F8EE
:10C20000486C002E8CD019642E46194643F8083C21
:10C21000E4E7002E84D053F80C1C2E46002E3FF489
:10C220007FAFAE427FF47CAF0D6CEA6B02F1010C84
:10C23000C5F83CC01D648B641946CFE772460227DF
:10C240002E46A64613E0D36B17635B01C2E9046672
:10C2500020D003F6FF7301EB133319465363CB1A57
:10C26000916352F84C4F4F1C1D440130C4B11379F7
:10C27000791E002BE7D1136917637BB103F6FF73B7
:10C2800001EB13335469536334B104F6FF7C01EBC3
:10C290001C31E4E73B46E0E73946E0E73B46F1E79F
:10C2A0001C4B01391C4A3E263F27C3F81C06C3F825
:10C2B000F42503F5BE604022C3F8105674468D0F76
:10C2C000C3F800268A00C3F80C16C0E90267C9B19A
:10C2D00040F2FF16921945F10005520A42EAC55292
:10C2E000C0E9094402F140042244C3F8044602EBC9
:10C2F000C101C3F808264C02C3F8F015CA0D40E985
:10C3000002420DE70122EBE7FFF79AFD04909FE65A
:10C3100060DD0024205A0024D06A0C08AA4BAB4AE6
:10C320002DE9F04F4FF0000A99B09E1A41F2210515
:10C330001F46342200210BA86EF070FAA34AA44BCA
:10C340000892CDE90976DA68D10707D5A14A5A6083
:10C3500002F188325A60DB68DC070DD49C4BD3F8BD
:10C360000C21D20708D59B4AC3F8042102F1883278
:10C37000C3F80421D3F80C31002101227E2308A840
:10C38000159105A98DF858208DF81430FDF794F813
:10C390000028C0F2288108214FF4FC4303E05B0031
:10C3A00001399BB207D01AB2002AF8DA85EA4202B4
:10C3B000013993B2F7D1884AADF81630874B9342D2
:10C3C00080F0508198460DF11809CDE902A7B8F820
:10C3D00002204FF0000CB8F80030C2F30B0B100431
:10C3E0008DF81DC00BF10601ADF81810C3F30B0159
:10C3F0004FEA1333ADF81A108DF81C3000F191801C
:10C400000622494608A8FDF757F80028C0F2FC802C
:10C41000BDF8164049460DF11E0011F8013B0822F7
:10C4200084EA032403E06400013AA4B207D023B2F3
:10C43000002BF8DA85EA4303013A9CB2F7D188422F
:10C44000EBD15A46D8F8041008A8FDF735F80028B3
:10C45000C0F2DA80D8F8041001EB0B00814215D04D
:10C460000139013811F8013F082284EA032403E06E
:10C470006400013AA4B207D023B2002BF8DA85EAAF
:10C480004303013A9CB2F7D18142EBD1ADF816409B
:10C4900008F11408504B984599D3DDE902A7002311
:10C4A0000222494608A8ADF81830FDF705F8002823
:10C4B000C0F29980BDF816300DF11A0041F2210149
:10C4C00019F8012B082483EA022303E05B00013CF6
:10C4D0009BB207D01AB2002AF8DA81EA4202013C84
:10C4E00093B2F7D14845EBD102220DF1160108A80D
:10C4F000ADF81630FCF7E0FF002874DB1498002834
:10C5000040F08880159800286DDB9DF85820002A9F
:10C5100040F0968000280DBF012200220123002355
:10C5200063E0E2466746019601370622494608A8BD
:10C53000FFB28DF81D70FCF7BFFF002850DBBDF87F
:10C54000164049460DF11E0011F8013B082284EA0D
:10C55000032403E06400013AA4B207D023B2002B05
:10C56000F8DA85EA4303013A9CB2F7D18842EBD16D
:10C57000D8F804105A4608A801EB0A063146FCF721
:10C580009BFF00282CDB06EB0B00864215D0711EAA
:10C59000013811F8013F082284EA032403E0640013
:10C5A000013AA4B207D023B2002BF8DA85EA43039C
:10C5B000013A9CB2F7D18142EBD1032FDA44ADF8B6
:10C5C0001640B1D1019E63E7000004080000020894
:10C5D000002000522301674504180D08C8120D08F9
:10C5E000DDE9016A039F012300220AF1010ABAF181
:10C5F000020F02DC002B7FF49CAE12B1FBF7E6FBCE
:10C6000028B9052008F0E4F9DDE902A7EBE719B045
:10C61000BDE8F08F089B099A03449342E3D80CAB22
:10C62000C0F12002214618446EF0F8F8159818B9A8
:10C630000CA908A8F6F74AFD00221590149262E7AB
:10C640000A4AD16841F00101D160D168C9077FF57C
:10C6500061AFD2F80C1141F00101C2F80C11D2F80F
:10C660000C2157E70DF1180919E700BF002000520F
:10C6700070B545880B4604460021C5F30B051846E6
:10C680002A466EF0CBF80A4A21690346914206D346
:10C69000084A914206D31846BDE870400847002971
:10C6A000F9D170BD2A46BDE870406CF08FBF00BF65
:10C6B00004180D08C91C0D08007970470079C0F3F3
:10C6C0004010704700794009704700BF90F83C2047
:10C6D000034602F0FF0012B1002283F83C207047AD
:10C6E0004FF48053838170474FF400638381704718
:10C6F0004FF40063838170474FF400638381704778
:10C700004FF400638381704770B5374CE08923880C
:10C71000B4F918501B1AA089B4F906C000FB03F342
:10C72000B4F91600666A05EBE335C00290FBF5F03C
:10C7300000EBE330B4F91230A0F57A6EE0610EFB45
:10C740000EF50EFB0CFC2D134FEAEC2C05FB03F34E
:10C750000CEBE32CB4F9103005FB03F3B4F90850EB
:10C760001B140EFB05F503EB6533B4F904500233DB
:10C770000CEB850CB4F920509B1064890CFA05FC75
:10C7800003F500430CF1020C04FB03F34CF25034AC
:10C79000A6EBAC0C2C41DB0B04FB0CF4002C1EDBD9
:10C7A0006400B4FBF3F389B11C1240F6DE3504FBE0
:10C7B00004F405FB04F40D4D241403FB05F504EB10
:10C7C000254404F6CF6403EB24130B602AB100EB7D
:10C7D00080004000083000111060012070BDB4FBE3
:10C7E000F3F35B00DFE700BFD8FC002443E3FFFF67
:10C7F00001207047012070472DE9F04F734D85B03F
:10C800000F46A86AAB8D0092C3EB2014B5F9302017
:10C810005B00B5F938E004FB04F4B5F83280C3EBF3
:10C82000E003CDF80CE02413B5F93A60B5F93C10FB
:10C8300002FB04F4B5F92E20029602FB03F3A413C5
:10C84000B5F9342004EBE324AB6CA4F5FA30019382
:10C85000B5F9363080FB00EA4FEAE37B82FB002C1F
:10C8600003FB0AF94FEA0C3C6C640EFB0B99A3FB2B
:10C870000E3B4CEA125C1203CB441B0A43EA0B63E7
:10C880009B184CEB2B2BA3FB08320BF5004B08FB42
:10C890000B2B4FEAEB734FEA6B0953EA6B0B00F07B
:10C8A0009280029E01FB0AFA019A86FB0008039E11
:10C8B000C2F5801C4A464FEA48484FEAE17948EA07
:10C8C000D0380EFB09A94004A1FB0E1E4118F1440B
:10C8D0004FF000000CF0004E49EB08094EEA5C0EE8
:10C8E00041184FEACC7C09EBC609BCEB010C6EEB9E
:10C8F000090E1CEB0C084EEB0E0118EB0C084EEB6E
:10C9000001014FEA88104FEA811918EB000049EA4B
:10C91000986941EB0901890041EA9071800010EBB0
:10C920000C004EEB0101890041EA9071800010EB90
:10C930000C004EEB010166F06DFCB5F942304FEA98
:10C94000613884464FEA503EB5F93E204FEAE37A1B
:10C9500003FB08F94EEAC14EB5F940000EFB0A99F7
:10C96000A3FB0E35A94403FB08F50EFB0955A3FBF9
:10C970000E3E75445B0E4FEAE07E43EAC51313EBAF
:10C980000C0341EB656500FB01F10EFB0C11A0FBF4
:10C990000C0C6144C00C40EA41301B1845EBE145EA
:10C9A0001B0A43EA056303EB02130FB11B0A3B604A
:10C9B000009B23B104EB8404803424121C6001200A
:10C9C00005B0BDE8F08F0023EFE700BFD8FC0024DE
:10C9D00031B10A4BD3ED197AFDEEE77AC1ED007A59
:10C9E00052B1064B9FED067AD3ED1A7A67EE877A3D
:10C9F000FDEEE77AC2ED007A01207047D8FC0024F2
:10CA00000000C8422DE9F04F5E4D934685B0B5F861
:10CA10007A30E86E1B02B5F878E0B5F87640C21AB5
:10CA2000B5F87430019167EB0707AEFB020C1B04ED
:10CA3000B5F872100EFB07CCC009B5F87C60C903CD
:10CA400040EA4C604FEAEC1CC018A4FB023E04FB19
:10CA500007EE4FEA13234CF1000C43EA0E634FEA52
:10CA60002E2E5B18A6FB021406FB07444FEAD15199
:10CA70004EF1000E41EA4421E41511F5FA6844F143
:10CA80000006B8F5FA6F029676F1000630DA01FB7F
:10CA900004F60394A1FB014A0AEB460AA6004FEAFA
:10CAA0008A09361949EA9479374C4AEB09094FEA61
:10CAB000560AB6084AEAC97A46EA8976B0EB0A0A03
:10CAC0006CEB690C9E1B50466EEBA90E3346A045DD
:10CAD000029E4FF0FF34A64126DB02FB07F7A2FBC4
:10CAE000022101EB4701D20F42EA4102B8EB0208F2
:10CAF000019C84B1D5F88010A1FB033201FB0E220A
:10CB00005B0D43EAC22352151B1A62EB0C02DB0BCE
:10CB100043EA42432360BBF1000F01D0CBF8008011
:10CB2000012005B0BDE8F08F40F6AC56039C891992
:10CB300044F1000401FB04F4A1FB016101EB440199
:10CB4000F4004FEAC109341B49EA567961EB09093F
:10CB500024184CEB090C2046B41941EB0109A41927
:10CB600041EB09094FEA890949EA9479A400A41B19
:10CB700069EB0109610841EAC971591A6EEB690E46
:10CB80000B46AAE7D8FC002424FAFFFF01207047D7
:10CB9000104B10B4104C1B68D4F884001B1AFA2BED
:10CBA0000BD811B1D4F88C300B6012B1D4F890309E
:10CBB000136001205DF8044B7047084A0021136898
:10CBC000084684F8881023F004035DF8044B1360D2
:10CBD000704700BFAC2F0024D8FC0024389C0024F0
:10CBE00001207047064B002200210120C3F8942049
:10CBF000C3F89820C3F89C20C3F8A010704700BF6A
:10CC0000D8FC0024104B11491A680346D1F8A00043
:10CC1000121AFA2A16D8D1ED256A012091ED267A4A
:10CC2000FDEEE66AD1ED277ABDEEC77AFDEEE77A32
:10CC300016EE902ADA8617EE102A1A8717EE902A37
:10CC40005A87704700207047AC2F0024D8FC00247E
:10CC5000024BD3F8A4305B68184700BFD8FC00240F
:10CC6000024B0830D3F8A4309B681847D8FC002446
:10CC70000120704701207047012070470120704754
:10CC80000120704731B10C4BD3ED2A7AF8EEE77AE8
:10CC9000C1ED007A72B10849084BD1F8AC10DFED54
:10CCA000086A0B4407EE903AF8EEE77A87EEA67A28
:10CCB00082ED007A704700BFD8FC00244D95FFFF3D
:10CCC0000000C84201207047012070477C4A01469D
:10CCD00000239446104610B490F904400C30012C07
:10CCE00049D00133082BF7D1754C002394F9040087
:10CCF0000C34022854D00133082BF7D1704C002398
:10CD000094F904000C34032867D00133082BF7D1C1
:10CD10006B4C002394F904000C34052873D00133C4
:10CD2000082BF7D1664C002394F904000C34062834
:10CD30007FD00133082BF7D1002392F904000C3285
:10CD4000072800F090800133082BF6D15D4B1B685B
:10CD5000DB0300F19E800B79142B00F0AD80173BB4
:10CD6000DAB21E2A00F2AA80574BD34003F001002A
:10CD70005DF8044B704703EB43035CF8233023B3A7
:10CD800052480B7990F8C84090F8C900984218BFF3
:10CD90009C420CBF01200020A6D15DF8044B7047D7
:10CDA00003EB43035CF823308BB149480B7990F8CF
:10CDB000C84090F8C900984218BF9C420CBF01209F
:10CDC00000209BD15DF8044B70473D4C8EE73C4CF6
:10CDD00094F904000C34032897D103EB43035CF867
:10CDE0002330002B3BD03B480B7990F8C84090F89B
:10CDF000C900984218BF9C420CBF0120002087D177
:10CE00005DF8044B704703EB43035CF8233043B3F6
:10CE100031480B7990F8C84090F8C900984218BF83
:10CE20009C420CBF012000207FF47CAF5DF8044BD6
:10CE3000704703EB43035CF82330002B3FF47DAFD6
:10CE400026480B7990F8C84090F8C900984218BF5E
:10CE50009C420CBF012000208AD003466DE7184C8D
:10CE600058E7174C60E703EB43035CF82330002BD3
:10CE70003FF46CAF1A4A0B7992F8C80092F8C920B7
:10CE80009A4218BF98420CBF012000207FF45EAF89
:10CE90006EE7144C0023224610791432182803D070
:10CEA00001330E2BF8D156E703EB83030A6854F8DD
:10CEB00023309A427FF44FAF012059E7002057E713
:10CEC00018900024D070002401000066EC070024B4
:10CED000BC0A00248C0D00245C1000242C130024B8
:10CEE000FC150024B40300240B4B8446002010B52D
:10CEF00003F58C7E02E014339E450BD01A68624520
:10CF0000F9D1DA68441C8A42F5D0D9601433E0B212
:10CF10009E45F3D110BD00BFB4030024044B03EBC6
:10CF20008003D3F8B0300BB19B681960704700BF25
:10CF3000D8FC0024044B03EB8003D3F8B0300BB1D2
:10CF40009B68196025F01CBBD8FC0024704700BF0B
:10CF500040F2FF72044B914203EBC003A8BF11469D
:10CF6000A3F8F410704700BFD8FC00242DE9F0416D
:10CF700003EB4306964686B0034602EB460675462B
:10CF800012F9067BA3EB070C92F80080BCF1000FAE
:10CF9000A3EB0804B8BFCCF1000C002CB8BF64426E
:10CFA000644502DA15464FFA88F70632B242E9D1F3
:10CFB000688803E00EF1060E764518D09EF8002032
:10CFC0008446BA42F6D10A1ABEF80280002AA1EBC2
:10CFD0000804B8BF5242002CB8BF64429442E9DA58
:10CFE00075460EF1060E4046C4467645E6D1687990
:10CFF000CDF808C02A780490287901920390012086
:10D0000000910321034AFDF7C1FF284606B0BDE8A1
:10D01000F08100BFA06E0C0838B505680446EB69C6
:10D02000F3B1987800B938BDB3F90A20012007EEB2
:10D03000902AF8EEE77AC4ED057AB3F90C2007EEF2
:10D04000902AF8EEE77AF1EE677AC4ED047AB3F944
:10D050000E3007EE903AF8EEE77AC4ED067A38BD66
:10D0600009211420FEF706F80346E861D9E700BF5E
:10D0700038B505680446EB69E3B1987800B938BD66
:10D08000B3F90420012007EE902AF8EEE77AC4ED08
:10D09000047AB3F9062007EE902AF8EEE77AC4ED99
:10D0A000057AB3F9083007EE903AF8EEE77AC4ED66
:10D0B000067A38BD09211420FDF7DCFF0346E8613C
:10D0C000DBE700BF38B505680446EB69E3B1987843
:10D0D00000B938BD9A880120D2BA07EE902AF8EE3E
:10D0E000E77AC4ED047ADA88D2BA07EE902AF8EE2D
:10D0F000E77AC4ED057A1B89DBBA07EE903AF8EEC1
:10D10000E77AC4ED067A38BD09211420FDF7B2FF95
:10D110000346E861DBE700BF38B505680C46EB69FC
:10D120007BB1987800B938BD5B890120084ADBBA29
:10D1300082FB0312DB17C3EB221303F26D13238070
:10D1400038BD09211420FDF795FF0346E861E8E7A3
:10D150007978787870B506680D461446F069A0B302
:10D16000D0F80130CDB1D0F80520B7EE006A9FEDC0
:10D170001A7A07EE902ADFED195ADFED196AF8EEF8
:10D18000677A77EEC77A77EEA77A87EEA57A77EE99
:10D19000467A67EEE67AC5ED007AACB107EE903AD2
:10D1A0009FED107ADFED105AF8EEE77A9FED0F6AE7
:10D1B000DFED0F6A67EE877A87EEA57A77EE467A1B
:10D1C00077EEA67AC4ED007A70BD09211420FDF730
:10D1D00051FFF061C4E700BF9AC9CC449AC94C46DC
:10D1E0000E76D7450000484300E0FF440000484267
:10D1F0003393884370B5066882B00D461446F069D3
:10D2000000284AD0D0F80530F3EE096ADFED265A3F
:10D21000B2EE047A07EE903A9FED246AD0F801301E
:10D22000F8EE677A77EEE57A67EE867A67EEA67AA9
:10D23000F4EEC77AF1EE10FA20DCBAEE047AF4EEDE
:10D24000C77AF1EE10FA19D42DB19FED197A67EE75
:10D25000877AC5ED007A7CB107EE903A9FED156AAA
:10D26000DFED156AB8EE677ADFED147AE7EE067A3D
:10D2700077EEA67AC4ED007A02B070BD17EE900A80
:10D2800065F042FB04460D460D4A04210320CDE91A
:10D290000045FDF77BFE02B070BD09211420FDF7AB
:10D2A000E9FEF061AEE700BF0000004600008038F4
:10D2B0000AD778430319C83D33938843000048C216
:10D2C000DC6E0C0890F91030F0B503EB4303264EEA
:10D2D000154683B056F83360044683689A0715D51F
:10D2E00001230DF106028DF8061030460DF10701FD
:10D2F000F6F722FF0123002229463046F6F71CFFED
:10D30000A3689B0716D5012003B0F0BD43691BB18C
:10D310009A88186812048261144B154A1868154BD4
:10D32000C0005768A3FB003080095368DB1B98429C
:10D33000FBD2D5E70D4A4FF4FA700E4B12680C4938
:10D3400000FB02F24868A3FB023292094B681B1AE9
:10D350009A42FBD26369002BD5D01A6801209B88C2
:10D36000936103B0F0BD00BF54030024FC350024DA
:10D37000001000E0D34D6210F0B5044683B00D46B6
:10D380001746061D20680379012B19D0022B02D005
:10D39000002003B0F0BD83683246FF21DB075CBF8D
:10D3A0003246FF21FFF78EFF0028F1D015B1237917
:10D3B000DB07E7D4002FECD023793B7003B0F0BD3E
:10D3C0008268417C02F0010C90F91000FF22CDE947
:10D3D000006CF6F791FBE7E770B50446051D82B0D7
:10D3E00020680379012B16D0022B02D0002002B056
:10D3F00070BD83682A46FF21DE075CBF2A46FF21F5
:10D40000FFF760FF0028F1D02379DB07EFD5206814
:10D410000379012BE8D18668FF22417C06F00106E2
:10D4200090F91000CDE90056F6F766FBEAE700BF79
:10D43000024630B5044652F8040B83B00379012B41
:10D440000ED0022B01D0002008E0FF21FFF73AFFA9
:10D450000028F8D02079C04300F0010003B030BDAF
:10D460008568417C05F0010590F910000092FF22CB
:10D470000195F6F741FBEBE72DE9F0414FF0B0469F
:10D48000D6F88050D6F888301D4010D0DFF82480C0
:10D490000127B5FA85F4C4F11F0458F8240007FAEF
:10D4A00004F403689847A543C6F88840F1D1BDE865
:10D4B000F08100BFD870002438B51446002944D04C
:10D4C000344B0D469FED344A93ED547AD3ED576AB1
:10D4D000B8EEC76AB3F96C21B8EEE60AD3ED557A17
:10D4E00004EE902AB3F96821C6EE046A93ED587AE7
:10D4F00005EE902AB3F96A2105EE102AB3F96621E8
:10D50000B3F96431F8EEE44A06EE102AF8EEE55A73
:10D51000F8EEE77AB8EEC55AB8EEC77AC7EE843AA5
:10D5200007EE903AB8EEC66AE6EEA45AF8EEE77A4D
:10D53000A6EE856AA6EEA57AE6EE867AA6EE870ABC
:10D54000A3EEA70A68F0B4FA28600CB3114BF6EE0C
:10D55000005A9FED115AD3ED556AB3F95A21F8EEEE
:10D56000E66AB3F9583107EE102A9FED0C6A07EE10
:10D57000903A86EE850AB8EEC77AF8EEE77A20EEA2
:10D58000070AA7EEA50A20EE060A68F091FA2060C5
:10D59000012038BDD8FC00240000F04A0000C84239
:10D5A0000C4B03EBC00310B5D3F8F04082B00191EF
:10D5B0006CB107EE901A94ED047A94ED030AF8EE3C
:10D5C000E77AA7EE870A68F073FAA368186002B0DA
:10D5D00010BD00BFD8FC0024F8B5534B0D461446CF
:10D5E0002DED048B1B7F022B18D09FED500A7DB1CF
:10D5F00020EE000ADFED4E7ADFED4E6A9FED4E7AA7
:10D6000020EE270AC0EE267A77EE877AC5ED007AFB
:10D610000CB14A4B2360BDEC048BF8BD484B494E1E
:10D620001B6896F8702103F002032AB1E3B9D6F81B
:10D63000803193ED340ADAE7002BF8D0424BB3F98E
:10D64000222001EE102AB3F92020B3F91E3000EE9B
:10D65000902AB8EEC11A00EE103AF8EEE00AB8EEE1
:10D66000C00AFDF7C1FAC2E7D6ED5D8A96ED5E9A73
:10D67000F0EE680AB0EE490AFDF792F8B5EEC00A7E
:10D68000B0EE408AF1EE10FA45D4B0EE680A2F4FA2
:10D69000F0EE490AFDF792FA9FED2D6ADFED2D6A53
:10D6A000F0EE408A28EE068AD7F8EC239FED2A7A1E
:10D6B000C8EE267AFCEEE77A17EE903A9BB29B1AF8
:10D6C00007EE903AF8EEE77AC7EE865AA5EEA67A0C
:10D6D000FDEEC77AB0EE470A17EE903A2033402BA2
:10D6E0001ED8FDF799FAF0EE407A1C4B797CA3F135
:10D6F0002C021846443BD6ED5F0A90ED000A002943
:10D7000018BF1346A8EEE70AD3ED057A70EEA70A14
:10D71000FDF754FA6BE7DFED127A30EE278AB4E7B3
:10D72000DFED027AE1E700BFE89C00240000000082
:10D73000CDCC9C3F00409C4682E6C54733139043C6
:10D74000D0750024D8FC00248C90002430BC002428
:10D750000000C84235FA8E3CDB0FC93F30C00024C0
:10D76000DB0FC94010B5037982B08E46012B0DD076
:10D77000022B02D0002002B010BD8368DB0758BF27
:10D7800041F0800102B0BDE810409BE5816814467D
:10D790007246009401F00104417C90F9100001945C
:10D7A000F6F7AAF902B010BD10B50446C06900B181
:10D7B00010BD09211420FDF75DFCE06110BD00BF24
:10D7C00010B1036882889A61704700BF18B18388DE
:10D7D00002681B0493617047184B03EB8000D0F87C
:10D7E000840138B300EB400003EB800292F995C14D
:10D7F000BCF1FF3F1FD092F89D01D8B103EB0C00A4
:10D80000002310B590F8E8E18C2092F89C111422C6
:10D8100000FB0CFC0A4C0CEB0100013A714434F89B
:10D82000100013FA80F3F6D1064AA2FB0320C0F3DE
:10D830000F1010BD70470020704700BFD8FC0024B7
:10D84000C0300030CDCCCCCC30B50D4683B00320F9
:10D850001446FFF7C1FF01909DB107EE900ADFED7E
:10D860000B5AB0EE006ADFED0A6AF8EE677AB8EE9E
:10D87000047A67EEA57AA7EE867A67EE267AC5ED7A
:10D88000007A0CB1034B236003B030BD6740533ABC
:10D8900000007A4433139043104B70B5104CA342F0
:10D8A00019D2054602E00C33A34214D293F805C006
:10D8B0008C45F8D193F804C00DB1AC45F3D1D879BB
:10D8C0009042F0D1186890F804E0E645EBD1066884
:10D8D0009E42E8D170BD002070BD00BFA0020008CC
:10D8E000740400080379022B00D0704790F91020CF
:10D8F00008311C4802EB420210B41B4C83B050F8B4
:10D90000322000946944194C11F808CCA24224D06A
:10D9100017498A4223D001F580618A4205D0154B10
:10D920009A420CBF03234FF0FF33116803EB43030C
:10D9300021F0010100EBC30011600169936851F807
:10D940002C1023F0E0430B439360136843F0010372
:10D95000136003B05DF8044B70470023E5E7012333
:10D96000E3E700BF5403002400010203003001403C
:10D97000003800400034014090F91030F0B503EB5E
:10D980004303284E154683B056F833600446836837
:10D990009A0719D501230DF106028DF806103046BD
:10D9A0000DF10701F6F7C8FB01230DF106020DF199
:10D9B000070130468DF80650F6F7BEFBA3689B07BB
:10D9C00016D5012003B0F0BD43691BB19A881868D1
:10D9D00012048261144B154A1868154BC000576831
:10D9E000A3FB003080095368DB1B9842FBD2D1E7D0
:10D9F0000D4A4FF4FA700E4B12680C4900FB02F20C
:10DA00004868A3FB023292094B681B1A9A42FBD268
:10DA10006369002BD5D01A6801209B88936103B0FD
:10DA2000F0BD00BF54030024FC350024001000E0CA
:10DA3000D34D621010B5037984B084468E46012B15
:10DA40000DD0022B02D0002004B010BD8368DB078C
:10DA500058BF01F07F0104B0BDE810408CE7816839
:10DA60000DF10F001446724601F001018DF80F40D0
:10DA7000CDE900019CF811109CF91000F5F70CFE9F
:10DA800004B010BD70B5B42282B00446FF21006816
:10DA9000FFF7D0FF10B9002002B070BD2068251D2F
:10DAA0000379012B13D0022BF5D183682A46FF217D
:10DAB000DE075CBF2A46FF21FFF704FC0028EAD0FE
:10DAC0002379DB07E8D520680379012BEBD1866841
:10DAD000FF22417C06F0010690F91000CDE90056C6
:10DAE000F6F70AF8EAE700BF70B50A4682B00446C6
:10DAF000A5210068FFF79EFF10B9002002B070BD9D
:10DB00002068251D0379012B13D0022BF5D18368E2
:10DB10002A46FF21DE075CBF2A46FF21FFF7D2FB22
:10DB20000028EAD02379DB07E8D520680379012BA8
:10DB3000EBD18668FF22417C06F0010690F91000C7
:10DB4000CDE90056F5F7D8FFEAE700BF002A34D048
:10DB5000F0B5044683B00E46051D8F1816F8012B4C
:10DB6000A5212068FFF766FF90B9002003B0F0BD43
:10DB70008268417C02F0010C90F91000FF22CDE98F
:10DB8000005CF5F7B9FF0028EFD02379DB070FD54C
:10DB900020680379012BEBD0022BE6D183682A465B
:10DBA000FF21DB075CBF2A46FF21FFF78BFBEAE77B
:10DBB000B742D3D1012003B0F0BD0120704700BFB0
:10DBC000F0B5962283B00E460446FF210068FFF7A9
:10DBD00031FF10B9002003B0F0BD251D2068037986
:10DBE000012B1DD0022BF5D183682A46FF21DF07C8
:10DBF0005CBF2A46FF21FFF765FB0028EAD02379A6
:10DC0000DB07EBD4E12220681146FFF713FF002861
:10DC1000E0D03246FF21206803B0BDE8F040A1E526
:10DC20008768FF22417C07F0010790F91000CDE9D9
:10DC30000057F5F761FFE0E7002A42D0F0B504464F
:10DC400083B00E46051D8F189622FF212068FFF72E
:10DC5000F1FE90B9002003B0F0BD8268417C02F073
:10DC6000010C90F91000FF22CDE9005CF5F744FFAC
:10DC70000028EFD02379DB070FD520680379012B2B
:10DC8000EBD0022BE6D183682A46FF21DB075CBF7D
:10DC90002A46FF21FFF716FBEAE7E122206811463A
:10DCA000FFF7C8FE0028D5D03246FF212068FFF7D5
:10DCB00059FD0028CED00136B742C5D1012003B0AE
:10DCC000F0BD0120704700BFF0B50B460546164673
:10DCD000044683B087211A4655F8040BFFF7AAFEC5
:10DCE00020680379012B19D0022B02D0002003B049
:10DCF000F0BD83682A46FF21DF075CBF2A46FF216B
:10DD0000FFF7E0FA0028F1D02379DA07E8D4002EF3
:10DD1000EDD0C3F34013337003B0F0BD8768FF222A
:10DD2000417C07F0010790F91000CDE90057F5F7A5
:10DD3000E3FEE7E7F0B5782183B0164604460022FB
:10DD40000068FFF777FE10B9002003B0F0BD251D75
:10DD500020680379012B13D0022BF5D183682A4662
:10DD6000FF21DF075CBF2A46FF21FFF7ABFA00283F
:10DD7000EAD02379DA07EBD45B09337003B0F0BD46
:10DD80008768FF22417C07F0010790F91000CDE978
:10DD90000057F5F7B1FEEAE770B5CC2282B0044631
:10DDA000A5210068FFF746FE10B9002002B070BD43
:10DDB0002068251D0379012B13D0022BF5D1836830
:10DDC0002A46FF21DE075CBF2A46FF21FFF77AFAC9
:10DDD0000028EAD02379DB07E8D520680379012BF6
:10DDE000EBD18668FF22417C06F0010690F9100015
:10DDF000CDE90056F5F780FEEAE700BF70B5B42222
:10DE000082B00446FF210068FFF714FE10B900201D
:10DE100002B070BD251D20680379012B21D0022B93
:10DE2000F5D183682A46FF21DE075CBF2A46FF2121
:10DE3000FFF748FA0028EAD02379DA07EBD4CC219F
:10DE40002046FFF751FE0028E1D002E02379DB07EE
:10DE5000DED52A46FF212068FFF784FC0028F5D193
:10DE6000D5E78668FF22417C06F0010690F9100094
:10DE7000CDE90056F5F740FEDCE700BF70B582B093
:10DE80000446CDE90023FFF7FDFD10B9002002B0E4
:10DE900070BD5522A5212068FFF7CCFD0028F5D0E4
:10DEA000251D2A46FF212068FFF75CFC0028EDD0E5
:10DEB0002379DB07F5D40DF1FF350DF1070615F8D1
:10DEC000011F2046FFF710FE0028DFD0B542F6D133
:10DED000DDE700BF2DE9F04F82468DB0002090466F
:10DEE0000AF10407089106900A930790069B504692
:10DEF000DC0008EBC3030593FFF7C4FD28B941E03C
:10DF00009AF8043013F0010208D03A46FF21DAF8FB
:10DF10000000FFF727FC0028F2D133E003929A07B4
:10DF20000B9040F1CC80F0215046FFF7DDFD48B367
:10DF3000083CDDF80C9008EB040301240993254606
:10DF4000089B003B18BF01230493049B082D8CBF42
:10DF5000002303F001039B46002B5DD06E1E089B3F
:10DF600043FA06F606F00106F2017821DAF800001D
:10DF7000FFF760FD30B1DAF800000379012B3FD0E4
:10DF8000022B07D000220A9B1046069919700DB08B
:10DF9000BDE8F08F83683A46FF21DB075CBF3A4655
:10DFA000FF21FFF78FF90028ECD09AF8043013F026
:10DFB0000102E0D199094FEA531E4FEAD31C01EA4E
:10DFC0005313DB074BD4664502D0BBF1000F73D16E
:10DFD000BCF1000F2DD0059911F80930234301F849
:10DFE00009306400013514F0FF04EDB2ADD109F140
:10DFF00001095FFA89F9B9F1080F30D00124A4E7CB
:10E000008268417C02F0010C90F91000FF22CDE9FA
:10E01000007CF5F771FDC6E7069BD3B1079BAB42C9
:10E0200017D9099B13F809301C4214BF012600269A
:10E030009AE74EEA0101039B11F0010F059908BF11
:10E040002B46039311F8093023EA040301F8093041
:10E05000C7E7079B5E1BB6FA86F6760984E7402D74
:10E0600007D80A9B069A1B7893423FF63FAF0246B9
:10E0700089E7059BDD795C1E9E1D14F801CF082100
:10E0800082EA0C0301394FEA5C0C43F3000311F000
:10E09000FF0123F0730383EA5202D2B2F0D1A64209
:10E0A000EBD19542DDD1069B0133DBB20693039B96
:10E0B000002BDCD00793D4E70B9E324663E706467D
:10E0C000324660E7F0B5046883B000210746642655
:10E0D0002046FFF707FC15227E212046FFF7AAFC09
:10E0E00006F01AFC04460D4606F016FC001B61EB18
:10E0F0000501B0F57A7F71F10001F5D3013EEFD152
:10E10000052611227E213868FFF794FC06F004FCF6
:10E1100004460D4606F000FC001B61EB0501B0F55E
:10E120007A7F71F10001F5D3013EEFD10DF10702C5
:10E1300003213868FFF716FB9DF8073003F03C0316
:10E14000142B40F09B800C2240213868FFF772FCB2
:10E1500006F0E2FB04460D4606F0DEFB001B61EB19
:10E160000501B0F57A7F71F10001F5D3454C092323
:10E17000B96B454A97F83500B4FBF1F189B2FEF767
:10E18000F5FE0346422138685A88B4FBF2F43C6439
:10E190001A79FFF74FFC06F0BFFB04460D4606F068
:10E1A000BBFB001B61EB0501B0F57A7F71F100014B
:10E1B000F5D3082241213868FFF73CFC06F0ACFBA0
:10E1C00004460D4606F0A8FB001B61EB0501B0F507
:10E1D0007A7F71F10001F5D3002243213868FFF7FF
:10E1E00029FC06F099FB04460D4606F095FB001B42
:10E1F00061EB0501B0F57A7F71F10001F5D31022D2
:10E2000051213868FFF716FC06F086FB04460D46E0
:10E2100006F082FB001B61EB0501B0F57A7F71F11E
:10E220000001F5D30A2253213868FFF703FC06F0FA
:10E2300073FB04460D4606F06FFB001B61EB050106
:10E24000B0F57A7F71F10001F5D38022562138684C
:10E25000FFF7F0FB06F060FB04460D4606F05CFBA2
:10E26000001B61EB0501B0F57A7F71F10001F5D378
:10E2700003213868FFF736FB03B0F0BD062006F037
:10E28000A7FB00BF40420F0080D10B082DE9F041F1
:10E290000768642682B0B6227E2180463846FFF7A2
:10E2A000C9FB06F039FB04460D4606F035FB001BA2
:10E2B00061EB0501B0F57A7F71F10001F5D3013E04
:10E2C000EFD102213846FFF70DFB7B691BB19A881D
:10E2D000196812048A6106F01FFB04460D4606F019
:10E2E0001BFB001B61EB0501B0F57A7F71F10001AA
:10E2F000F5D37B6913B11A689B8893610A2606F0EF
:10E300000BFB04460D4606F007FB001B61EB050105
:10E31000B0F57A7F71F10001F5D3013EEFD13246BD
:10E320007C213846FFF786FB06F0F6FA04460D46D8
:10E3300006F0F2FA001B61EB0501B0F57A7F71F18E
:10E340000001F5D3002259213846FFF773FB06F090
:10E35000E3FA04460D4606F0DFFA001B61EB050107
:10E36000B0F57A7F71F10001F5D397F910305E2195
:10E370008D4A03EB43038DF8071052F83340BB6816
:10E380009A0740F1E48001230DF1070200212046A5
:10E39000F5F7D2FE4FF4A473844A20460021F5F726
:10E3A000CBFEBB689B0740F1E6800A2606F0B4FA74
:10E3B00004460D4606F0B0FA001B61EB0501B0F50E
:10E3C0007A7F71F10001F5D3013EEFD1012259218D
:10E3D0003846FFF72FFB06F09FFA04460D4606F07D
:10E3E0009BFA001B61EB0501B0F57A7F71F100012A
:10E3F000F5D38C2240213846FFF71CFB06F08CFA3F
:10E4000004460D4606F088FA001B61EB0501B0F5E5
:10E410007A7F71F10001F5D3032241213846FFF7DD
:10E4200009FB06F079FA04460D4606F075FA001B62
:10E4300061EB0501B0F57A7F71F10001F5D35C4C19
:10E440000923D8F8382098F83500B4FBF2F291B2DD
:10E45000584AFEF78BFD43884221B4FBF3F4C8F819
:10E4600040400279384642F0C002FFF7E3FA06F076
:10E4700053FA04460D4606F04FFA001B61EB050106
:10E48000B0F57A7F71F10001F5D3082243213846B7
:10E49000FFF7D0FA06F040FA04460D4606F03CFAC3
:10E4A000001B61EB0501B0F57A7F71F10001F5D336
:10E4B000042258213846FFF7BDFA06F02DFA04462B
:10E4C0000D4606F029FA001B61EB0501B0F57A7FD5
:10E4D00071F10001F5D30A2253213846FFF7AAFA59
:10E4E00006F01AFA04460D4606F016FA001B61EB18
:10E4F0000501B0F57A7F71F10001F5D300227C218E
:10E500003846FFF797FA06F007FA04460D4606F07C
:10E5100003FA001B61EB0501B0F57A7F71F1000190
:10E52000F5D306227D213846FFF784FA06F0F4F988
:10E5300004460D4606F0F0F9001B61EB0501B0F54D
:10E540007A7F71F10001F5D302B0BDE8F0817B69FB
:10E550001BB11A689B881B049361174B17491A68F3
:10E56000174BD2004868A3FB023292094B681B1A72
:10E570009A42FBD207E7104A4FF4FA70104B126828
:10E580000E4900FB02F24868A3FB023292094B6875
:10E590001B1A9A42FBD27B69002B3FF406AF1A6824
:10E5A0009B88936101E700BF54030024B8D10B0896
:10E5B00040420F0000D30B08FC350024001000E09F
:10E5C000D34D62102DE9F041816B1023654D044657
:10E5D00007686426644A90F83500B5FBF1F189B20A
:10E5E000FEF7C4FC4388002180463846B5FBF3F5AE
:10E5F0002564FFF777F980226B213846FFF71AFA76
:10E6000006F08AF904460D4606F086F9001B61EB18
:10E610000501B0F57A7F71F10001F5D3013EEFD12C
:10E620006426072268213846FFF704FA06F074F9D9
:10E6300004460D4606F070F9001B61EB0501B0F5CC
:10E640007A7F71F10001F5D3013EEFD132466426A5
:10E650006B213846FFF7EEF906F05EF904460D46E9
:10E6600006F05AF9001B61EB0501B0F57A7F71F1F4
:10E670000001F5D3013EEFD10F2601226B21384670
:10E68000FFF7D8F906F048F904460D4606F044F9BC
:10E69000001B61EB0501B0F57A7F71F10001F5D344
:10E6A000013EEFD10F2618221B213846FFF7C2F991
:10E6B00006F032F904460D4606F02EF9001B61EB18
:10E6C0000501B0F57A7F71F10001F5D3013EEFD17C
:10E6D0000F2618221C213846FFF7ACF906F01CF96A
:10E6E00004460D4606F018F9001B61EB0501B0F574
:10E6F0007A7F71F10001F5D3013EEFD10F2698F832
:10E7000004201A213846FFF795F906F005F904466A
:10E710000D4606F001F9001B61EB0501B0F57A7FAB
:10E7200071F10001F5D3013EEFD1642698F8052080
:10E7300019213846FFF77EF906F0EEF804460D463B
:10E7400006F0EAF8001B61EB0501B0F57A7F71F184
:10E750000001F5D3013EEFD138460321BDE8F04179
:10E76000FFF7C0B840420F0038D30B082AE700BFBC
:10E77000F0B583B015461C4606460DF107020F465C
:10E78000FEF7F0FF9DF8072005EA0203A34201D13E
:10E7900003B0F0BD22EA050239463046224303B0F9
:10E7A000BDE8F040FFF746B9F8B50526782200210C
:10E7B00007460068FFF73EF906F0AEF804460D463E
:10E7C00006F0AAF8001B61EB0501B0F57A7F71F144
:10E7D0000001F5D3013EEFD1052620220121386842
:10E7E000FFF728F906F098F804460D4606F094F86D
:10E7F000001B61EB0501B0F57A7F71F10001F5D3E3
:10E80000013EEFD13246642602213868FFF712F943
:10E8100006F082F804460D4606F07EF8001B61EB18
:10E820000501B0F57A7F71F10001F5D3013EEFD11A
:10E830000120F8BD70B52422044641210068FFF78D
:10E84000F9F890B9052606F067F804460D4606F07B
:10E8500063F8001B61EB0501B0F57A7F71F10001EF
:10E86000F5D3013EEFD1012070BD20223021206878
:10E87000FFF7E0F80028E5D0062231212068FFF7F5
:10E88000D9F80028DED0002234212068FFF7D2F822
:10E89000D8E700BFF8B5052607220A210746006819
:10E8A000FFF7C8F806F038F804460D4606F034F8CD
:10E8B000001B61EB0501B0F57A7F71F10001F5D322
:10E8C000013EEFD10526242241213868FFF7B2F836
:10E8D00006F022F804460D4606F01EF8001B61EB18
:10E8E0000501B0F57A7F71F10001F5D3013EEFD15A
:10E8F0000526C02242213868FFF79CF806F00CF884
:10E9000004460D4606F008F8001B61EB0501B0F562
:10E910007A7F71F10001F5D3013EEFD10120F8BDFE
:10E9200010B50446002221210068FFF783F8FC227D
:10E9300020212068FFF77EF8402224212068FFF77D
:10E9400079F80C2223212068FFF774F80022222195
:10E950002068FFF76FF8012010BD00BFF8B5012255
:10E96000074610210068FFF765F800B9F8BD1426C6
:10E9700005F0D2FF04460D4605F0CEFF001B61EB0B
:10E980000501B0F57A7F71F10001F5D3013EEFD1B9
:10E990003868A0221121BDE8F840FFF74BB800BF4E
:10E9A000F0B5046883B00746002120461426FEF720
:10E9B00099FF0C2225212046FFF73CF80A22262148
:10E9C0003868FFF737F8002263213868FFF732F81C
:10E9D000812227213868FFF72DF805F09DFF0446B6
:10E9E0000D4605F099FF001B61EB0501B0F57A7F3C
:10E9F00071F10001F5D3013EEFD10C2225213868D9
:10EA00000A26FFF717F80A2226213868FFF712F8BE
:10EA10000F2263213868FFF70DF88122272138681B
:10EA2000FFF708F805F078FF04460D4605F074FF7F
:10EA3000001B61EB0501B0F57A7F71F10001F5D3A0
:10EA4000013EEFD10A26032301AA102138465DF0CA
:10EA5000DDFC05F061FF04460D4605F05DFF001B7F
:10EA600061EB0501B0F57A7F71F10001F5D3013E4C
:10EA7000EFD19DF804009DF805109DF80620803028
:10EA80002B4B80318032A3F8EC01A3F8EE11252145
:10EA9000A3F8F0210C223868FEF7CCFF0A222621C9
:10EAA0003868FEF7C7FF3246632138680A26FEF74A
:10EAB000C1FF812227213868FEF7BCFF05F02CFF3B
:10EAC00004460D4605F028FF001B61EB0501B0F57B
:10EAD0007A7F71F10001F5D3013EEFD10DF1030210
:10EAE0000123022138465DF091FC01230DF1030260
:10EAF000092138465DF08AFC0C2225213868FEF792
:10EB000099FF0A2226213868FEF794FF122263211A
:10EB10003868FEF78FFF812227213868FEF78AFFC9
:10EB200038680321FEF7DEFE012003B0F0BD00BF10
:10EB3000D8FC00242DE9F04180220B210746006813
:10EB4000FEF778FF1E26804605F0E6FE04460D46D9
:10EB500005F0E2FE001B61EB0501B0F57A7F71F173
:10EB60000001F5D3013EEFD1B8F1000F02D1002032
:10EB7000BDE8F081062229213868FEF75BFF0028F6
:10EB8000F5D008220B213868FEF754FF0028EED09C
:10EB90003868CF220A21BDE8F041FEF74BBF00BF25
:10EBA00010B5044694220B210068FEF743FF712242
:10EBB00001212068FEF73EFF002204212068FEF7B5
:10EBC00039FFC82205212068FEF734FF0022062104
:10EBD0002068FEF72FFFC82207212068FEF72AFFD2
:10EBE000002208212068FEF725FFC822092120689D
:10EBF000FEF720FF012010BD0A4600212DE9F0415B
:10EC0000DFF8B08084B042F001020446274EFEF7E0
:10EC100011FFD8F80070264DC6F8F47118E0022BE9
:10EC20004FF000000BD1A3680DF10F021321204615
:10EC3000DB0702D40DF10F029321FEF743FB9DF891
:10EC40000F30287013F0070318D1D6F8F8212ABB2B
:10EC50002379012BE3D1A2680DF10F0102F001022B
:10EC6000009101921322617C94F91000F4F744FFA3
:10EC70009DF80F30287013F00703E6D001220B2116
:10EC80002046FEF7D7FE002220461146FEF7D2FEB0
:10EC900001232870184604B0BDE8F081D8F80010B0
:10ECA00089B2C91B8A42D3D2F4E700BFD8FC002442
:10ECB0000C1B0024AC2F002470B5056884B00446FA
:10ECC0000E462B79012B1BD0022B02D0002004B062
:10ECD00070BDAB68F0222846DB074CBFE121612103
:10ECE000FEF74AFE0028F1D02246FF2152F8040B1D
:10ECF000FEF738FD0028E9D02379337004B070BDE9
:10ED0000AA6895F9100002F00102697C01920DF1E8
:10ED10000F020092F0228DF80F20E122F4F7BCFCE4
:10ED2000E0E700BF00680379012B0AD0022B01D075
:10ED3000002070478368B422DB0718D5FF21FEF757
:10ED40001BBE826890F910C002F00102417C60464F
:10ED50004FF0B40C10B584B00DF10F040192FF22F6
:10ED60008DF80FC00094F4F797FC04B010BD7F211C
:10ED7000FEF702BE00680379012B0AD0022B01D0F6
:10ED80000020704783680A46DB0716D5A521FEF7E9
:10ED9000F3BD10B584B0846890F910C00DF10F0276
:10EDA00004F001048DF80F10417C60460092A5220A
:10EDB0000194F4F771FC04B010BD2521FEF7DCBD11
:10EDC00000680379012B0AD0022B01D00020704784
:10EDD00083689622DB0718D5FF21FEF7CDBD826838
:10EDE00090F910C002F00102417C60464FF0960C91
:10EDF00010B584B00DF10F040192FF228DF80FC001
:10EE00000094F4F749FC04B010BD7F21FEF7B4BDB7
:10EE100000680379012B0AD0022B01D00020704733
:10EE200083680A46DB0716D58721FEF7A5BD10B516
:10EE300084B0846890F910C00DF10F0204F0010451
:10EE40008DF80F10417C6046009287220194F4F700
:10EE500023FC04B010BD0721FEF78EBD0068C90178
:10EE60000379CAB2012B06D0022B01D000207047D3
:10EE70007821FEF781BD10B584B0846890F910C088
:10EE80008DF80F200DF10F0204F00104417C009277
:10EE9000782260460194F4F7FFFB04B010BD00BF78
:10EEA00000680379012B0AD0022B01D000207047A3
:10EEB00083685522DB0718D5A521FEF75DBD826862
:10EEC00090F910C002F00102417C60464FF0550CF1
:10EED00010B584B00DF10F040192A5228DF80FC07A
:10EEE0000094F4F7D9FB04B010BD2521FEF744BD12
:10EEF00000680379012B0AD0022B01D00020704753
:10EF000083682E22DB0718D5F421FEF735BD826811
:10EF100090F910C002F00102417C60464FF02E0CC7
:10EF200010B584B00DF10F040192F4228DF80FC0DA
:10EF30000094F4F7B1FB04B010BD7421FEF71CBDC2
:10EF4000154B00681A8C03799201012B02F13402EF
:10EF5000D2B209D0022B01D0002070478368DB07B2
:10EF600016D5F421FEF708BD10B584B0846890F979
:10EF700010C08DF80F200DF10F0204F00104417C48
:10EF80000092F42260460194F4F786FB04B010BDB1
:10EF90007421FEF7F1BC00BFD8FC0024006810B556
:10EFA000037984B0012B0FD0022B02D0012004B0D2
:10EFB00010BD83683122DB074CBFF4217421FEF7BA
:10EFC000DBFC012004B010BD82680DF10F0490F944
:10EFD00010C002F00102417C60464FF0310C0192FA
:10EFE000F42200948DF80FC0F4F756FB012004B012
:10EFF00010BD00BF00680379012B07D0022B01D0A0
:10F000000020704701225821FEF7B6BC8268417C7F
:10F0100002F0010210B590F9104084B020460DF1C5
:10F020000F040192582200948DF80F30F4F734FB4E
:10F0300004B010BD00680379012B07D0022B01D06A
:10F040000020704701224821FEF796BC8268417C6F
:10F0500002F0010210B590F9104084B020460DF185
:10F060000F040192482200948DF80F30F4F714FB3E
:10F0700004B010BD00680379012B07D0022B01D02A
:10F08000002070471A460821FEF776BC826890F986
:10F0900010C002F00102417C60464FF0020C10B536
:10F0A00084B00DF10F04019208228DF80FC0009476
:10F0B000F4F7F2FA04B010BD00680379012B07D011
:10F0C000022B01D00020704701220821FEF754BC1A
:10F0D0008268417C02F0010210B590F9104084B0C2
:10F0E00020460DF10F040192082200948DF80F3094
:10F0F000F4F7D2FA04B010BD10B50446006884B02D
:10F100000379012B12D0022B02D0002004B010BDD5
:10F1100001220B21FEF730FC0028F6D01D22092128
:10F12000206804B0BDE81040FEF784BC826890F906
:10F1300010C002F00102417C60468DF80F30019250
:10F140000DF10F0200920B22F4F7A6FAE4E700BFDC
:10F150002DE9F04105461F462848164695F910301E
:10F1600082B003EB430350F83380AB689A0716D59F
:10F1700001230DF106028DF8061040460DF107013E
:10F18000F4F7DAFF3B46324600214046F4F7D4FF5D
:10F19000AB689B0718D5012002B0BDE8F0816B6910
:10F1A0001BB19A88186812048261154B1868154BB8
:10F1B000C000A3FB0030144B80095A685C68A4EBC4
:10F1C000020C6045FAD2D3E70D4A4FF4FA700D4BAA
:10F1D00012680D4900FB02F24868A3FB0232920953
:10F1E0004B681B1A9A42FBD26B69002BD3D01A686A
:10F1F00001209B88936102B0BDE8F0815403002494
:10F20000FC350024D34D6210001000E030B50579C4
:10F2100083B084468E46012D0DD0022D02D00020F1
:10F2200003B030BD8468E40758BF41F0800103B0EB
:10F23000BDE830408CE7806814460A46009400F030
:10F2400001049CF811109CF910000194F4F724FAC1
:10F2500003B030BDF0B5002383B0142607468DF807
:10F26000023005F059FB04460D4605F055FB001B26
:10F2700061EB0501B0F57A7F71F10001F5D3013E34
:10F28000EFD131460DF102023868FEF76BFA0DF14D
:10F29000020280213868FEF765FA4FF4F8428DF8D3
:10F2A00006601426ADF80420032301AA6021386803
:10F2B000FFF7ACFF05F030FB04460D4605F02CFBD4
:10F2C000001B61EB0501B0F57A7F71F10001F5D308
:10F2D000013EEFD131460DF1030238688DF803602D
:10F2E000FEF740FA4CF26243142601AA6021ADF801
:10F2F0000430042338688DF806300323FFF786FFB7
:10F3000005F00AFB04460D4605F006FB001B61EB09
:10F310000501B0F57A7F71F10001F5D3013EEFD11F
:10F3200031460DF1030238688DF80360FEF71AFAD2
:10F330004FF4E853142601AA6021ADF804300823E5
:10F3400038688DF806300323FFF760FF05F0E4FA14
:10F3500004460D4605F0E0FA001B61EB0501B0F52F
:10F360007A7F71F10001F5D3013EEFD10DF1030277
:10F37000314638688DF80360FEF7F4F90DF10202AA
:10F380001E213868FEF7EEF9012003B0F0BD00BF82
:10F390002DE9F04105461F462848164695F91030DC
:10F3A00082B003EB430350F83380AB689A0716D55D
:10F3B00001230DF106028DF8061040460DF10701FC
:10F3C000F4F7BAFE3B46002231464046F4F7B4FE5D
:10F3D000AB689B0718D5012002B0BDE8F0816B69CE
:10F3E0001BB19A88186812048261154B1868154B76
:10F3F000C000A3FB0030144B80095A685C68A4EB82
:10F40000020C6045FAD2D3E70D4A4FF4FA700D4B67
:10F4100012680D4900FB02F24868A3FB0232920910
:10F420004B681B1A9A42FBD26B69002BD3D01A6827
:10F4300001209B88936102B0BDE8F0815403002451
:10F44000FC350024D34D6210001000E030B5057982
:10F4500083B084468E46012D0DD0022D02D00020AF
:10F4600003B030BD8468E40758BF41F0800103B0A9
:10F47000BDE830408CE7806814460A46009400F0EE
:10F4800001049CF811109CF910000194F4F734FB6E
:10F4900003B030BD2DE9F043816B85B0804C102363
:10F4A000076880467F4A962690F83500B4FBF1F154
:10F4B00089B2FDF75BFD4388002181463846B4FBE5
:10F4C000F3F4C8F84040FEF70DFA80226B2138466D
:10F4D000FEF7B0FA05F020FA04460D4605F01CFAD6
:10F4E000001B61EB0501B0F57A7F71F10001F5D3E6
:10F4F000013EEFD19626032268213846FEF79AFA9C
:10F5000005F00AFA04460D4605F006FA001B61EB09
:10F510000501B0F57A7F71F10001F5D3013EEFD11D
:10F5200003226B213846FEF785FA05F0F5F904460B
:10F530000D4605F0F1F9001B61EB05010F2871F193
:10F540000001F6D310226A213846FEF773FA05F05F
:10F55000E3F904460D4605F0DFF9001B61EB0501F8
:10F560000F2871F10001F6D300226C213846FEF716
:10F5700061FA05F0D1F904460D4605F0CDF9001BFE
:10F5800061EB05010F2871F10001F6D399F8052010
:10F5900019213846FEF74EFA05F0BEF904460D462D
:10F5A00005F0BAF9001B61EB05010F2871F10001AC
:10F5B000F6D318221B213846FEF73CFA05F0ACF9C9
:10F5C00004460D4605F0A8F9001B61EB05010F2864
:10F5D00071F10001F6D318221C213846FEF72AFAF1
:10F5E00005F09AF904460D4605F096F9001B61EB0B
:10F5F00005010F2871F10001F6D399F804201A21B2
:10F600003846FEF717FA05F087F905460C4605F06F
:10F6100083F98C4208BF8542F9D003213846FEF7B2
:10F6200061F9062302AA4321D8F80000FFF70EFF74
:10F6300028B3BDF80810BDF80A30BDF80C20C9BACF
:10F64000DBBA07EE901AD2BAF8EEE76A07EE102A94
:10F6500007EE903AB8EEC77AF8EEE77AC8ED076A97
:10F6600088ED097AC8ED087AFDEEE77ACDED017AEA
:10F670009DF90430013305D005B0BDE8F083D8ED25
:10F68000087AF1E7D8ED077AFDEEE77ACDED017A59
:10F690009DF904300133EFD1062005F099F900BF40
:10F6A00040420F0038D30B0810B582B00821044641
:10F6B00000686A46FEF756F89DF80030DB0602D473
:10F6C000002002B010BD06236A4600212068FFF723
:10F6D000BDFE0028F4D09DF80120B6EE002A9DF86A
:10F6E000001012029DF80230DFED376A02EB014292
:10F6F0009DF80410134414024FEA01219DF80340C1
:10F7000048BF03F17F439DF8052001EB044107EE5C
:10F71000903A2E4B0A440902B8EEE77A48BF02F14C
:10F720007F4287EE266A07EE902AB3F9602002EE48
:10F73000902AB3F95C2005EE102AF8EEE22AF8EEE2
:10F74000E77AB3F95820B8EEC55A04EE902AB3F917
:10F750005A2087EEA64AD3ED157A06EE902AB3F921
:10F760005E2003EE102AB3F94E20F8EEE75AD3EDEF
:10F77000147AF8EEE44A07EE102AA6EE225AB3F9FC
:10F780004C20F8EEE77AB8EEC33A03EE902AF8EE92
:10F79000E66AB8EEC77AF8EEE33AE5EE065AE6EE28
:10F7A000036A27EE047A26EE043AE5EE867AA3EEA3
:10F7B000827AE4EE247A83ED1A7AE3EE267AC3EDB8
:10F7C000197A02B010BD00BF00007848D8FC0024B0
:10F7D000F0B5142683B000220A2107460068FEF720
:10F7E00029F905F099F804460D4605F095F8001B37
:10F7F00061EB0501B0F57A7F71F10001F5D3013EAF
:10F80000EFD10A260F220A213868FEF713F905F016
:10F8100083F804460D4605F07FF8001B61EB0501F7
:10F82000B0F57A7F71F10001F5D3013EEFD10A26E0
:10F83000032301AA10213868FFF708FE05F06CF8D1
:10F8400004460D4605F068F8001B61EB0501B0F5B4
:10F850007A7F71F10001F5D3013EEFD19DF80420CC
:10F860009DF805009DF806108032194B80308031DC
:10F87000A3F8FC2132460A26A3F8FE01A3F80012E1
:10F880000A213868FEF7D6F805F046F804460D461A
:10F8900005F042F8001B61EB0501B0F57A7F71F1CC
:10F8A0000001F5D3013EEFD10DF1030202213868CA
:10F8B000FDF758FF0DF1030209213868FDF752FFEB
:10F8C00011220A213868FEF7B5F8012003B0F0BD17
:10F8D000D8FC0024026830B5137985B00446012BAA
:10F8E00061D0022B03D00025284605B030BD9168B9
:10F8F00002AD1046C9072A464CBF19468221FDF7C2
:10F90000E1FC0028EFD09DF80830DA07EBD52A4655
:10F91000072303212068FFF799FD05460028E2D060
:10F9200011220A212068FEF785F89DF80E301B078A
:10F93000D9D42A49BDF80830B1F8FC2113FB02F3F1
:10F94000274A93423EDBB3F5000F39DA002BB8BFEC
:10F95000FF331B125B421BB2BDF80A20E386B1F8ED
:10F96000FE3112FB03F31E4A93422FDBB3F5000F67
:10F9700030DA002BB8BFFF3343F30F22BDF80C3051
:10F98000B1F80012228713FB01F3154A93421BDBE7
:10F99000B3F5000F1CDA002BB8BFFF331B125B421C
:10F9A0001BB26387A0E7517C02AD92F91000926808
:10F9B000009502F0010201920222F4F79DF8A0E7FF
:10F9C000084BC9E7084BC7E7074BEAE7064AD5E704
:10F9D000044BE6E747F6FF72D0E700BFD8FC0024EF
:10F9E00001FF7FFF0180FFFF0080FFFFF0B51426BD
:10F9F00083B000220A2107460068FEF71BF804F0D6
:10FA00008BFF04460D4604F087FF001B61EB0501E8
:10FA1000B0F57A7F71F10001F5D3013EEFD10A26EE
:10FA20000F220A213868FEF705F804F075FF044636
:10FA30000D4604F071FF001B61EB0501B0F57A7F04
:10FA400071F10001F5D3013EEFD10A26032301AA8B
:10FA500010213868FFF7FAFC04F05EFF04460D46FB
:10FA600004F05AFF001B61EB0501B0F57A7F71F1DC
:10FA70000001F5D3013EEFD132460A260A2138684B
:10FA8000FDF7D8FF04F048FF04460D4604F044FF9C
:10FA9000001B61EB0501B0F57A7F71F10001F5D330
:10FAA000013EEFD10DF1030202213868FDF75AFE45
:10FAB0000DF1030209213868FDF754FE01220A21E5
:10FAC0003868FDF7B7FF012003B0F0BD30B5002363
:10FAD00085B004460221C0F836300DF10702438795
:10FAE0000068FDF73FFE18B19DF80730DB0703D42F
:10FAF0000025284605B030BD062302AA0321206850
:10FB0000FFF7A4FC0DF1070209212068FDF72AFE8A
:10FB100005460028ECD09DF8073013F00C0FE7D114
:10FB2000BDF80820BDF80C30BDF80A10C2EB8232D7
:10FB3000C3EB8333206889009B0092002187638791
:10FB40000A21E2860122FDF775FF284605B030BD87
:10FB500010B50446006882B003796A46022B4FF064
:10FB600006030CBF43210321FFF770FC68B1BDF809
:10FB70000010BDF80220BDF8043049BA52BA5BBA91
:10FB8000E1866287238702B010BDC4F83600608723
:10FB900002B010BD10B5002386B0044600688DF891
:10FBA0000F300379012B31D0022B02D0002006B098
:10FBB00010BD83680DF10F02D9074CBF2721A72183
:10FBC000FDF780FB0028F1D09DF80F301B07EDD525
:10FBD000062304AA28212068FFF738FC28B3BDF9C2
:10FBE0001030002BB8BF03339A10BDF91230002B30
:10FBF000E286B8BF03339A10BDF91430002B228778
:10FC0000B8BF03339B10638706B010BD8268417C88
:10FC100002F0010290F910C001920DF10F0260464E
:10FC200000922722F3F768FFCCE7C4F8360060871C
:10FC30000020BCE730B54FF0000C0446006887B0E8
:10FC4000C4F836C0A4F83AC00379012B2AD0022B9D
:10FC500002D0002007B030BD83680DF10F02D90734
:10FC60004CBF61468021FDF72DFB0028F1D09DF8A7
:10FC70000F301B07EDD5062304AA01212068FFF7EA
:10FC8000E5FB0028E5D0BDF81430BDF81010BDF834
:10FC900012205BBA49BA52BA5B42E1862287638777
:10FCA00007B030BD85686246417C05F0010590F9DA
:10FCB000100001950DF10F050095F3F71DFFD4E736
:10FCC0002DE9F047164F81468A4697F809326BB9FD
:10FCD0000024D9F8000097F80A325246492187F8E3
:10FCE0000942FFF7B3FB0120BDE8F08704F014FEE2
:10FCF000D7F81032C51AC5F5FA55002DE8DD04F025
:10FD00000BFE04464FEAE5780E4604F005FE001BA4
:10FD100061EB0601A84271EB0801F6D3D8E700BFFA
:10FD2000D8FC00242DE9F041624C054682B0D4F89D
:10FD30001802C5F8360094F80832B4F81C22012BDA
:10FD40006A8777D0022B0FD0002B69D101220221C4
:10FD500028465EF065F9012394F81E6284F80832A3
:10FD6000304602B0BDE8F08194F8093204F5067718
:10FD700005F13608002B6FD169462846FFF7A0FF32
:10FD80009DF80630064600284AD01B0748D4B4F830
:10FD9000EC21BDF8003013FB02F3474A93427EDBAF
:10FDA000B3F5000F70DA002BB8BFFF331B125B42B4
:10FDB0001BB2B4F8EE21EB86BDF8023013FB02F360
:10FDC0003D4A93426FDBB3F5000F70DA002BB8BFEA
:10FDD000FF3343F30F23B4F8F0212B87BDF8043031
:10FDE00013FB02F3344A93425BDBB3F5000F5CDA9A
:10FDF000002BB8BFFF331B125B421BB2D5F8360095
:10FE00006B870023C4F818023046B8F8042084F841
:10FE100008320123BA8084F81E3202B0BDE8F081B6
:10FE200000231E4684F8083284F81E32304602B0A1
:10FE3000BDE8F08194F8093294F81E62D3B969469E
:10FE40002846FFF73DFF9DF8003008B19A071DD105
:10FE5000002384F8083283E704F05EFDD4F8103202
:10FE6000C01AB0F5FA5F87DA94F81E62304602B025
:10FE7000BDE8F08104F050FDD4F81032C01AB0F59E
:10FE8000FA5FFFF66DAFDAE70C4B92E7072203212A
:10FE900028465EF0C5F8022384F8083260E7084B74
:10FEA00087E7074BAAE7064B95E7044BA6E747F61B
:10FEB000FF7390E7D8FC002401FF7FFF0180FFFF64
:10FEC0000080FFFF10B500230446006886B0C4F828
:10FED000363063870379012B23D0022B02D0002018
:10FEE00006B010BD83680DF10F02D9074CBF062183
:10FEF0008621FDF7E7F90028F1D09DF80F305B0768
:10FF0000EDD5062304AA00212068FFF79FFA0028F8
:10FF1000E5D0049ABDF81430C4F83620638706B0E3
:10FF200010BD8268417C02F0010290F910C001927C
:10FF30000DF10F02604600920622F3F7DDFDDAE7CD
:10FF400010B500230446006886B0C4F836306387D5
:10FF50000379012B29D0022B02D0002006B010BD5E
:10FF600083680DF10F02D9074CBF09218921FDF7E4
:10FF7000A9F90028F1D09DF80F30DB07EDD5062355
:10FF800004AA01212068FFF761FA0028E5D0BDF836
:10FF90001210BDF81020BDF81430494252425B42A5
:10FFA000E1862287638706B010BD8268417C02F03B
:10FFB000010290F910C001920DF10F02604600920B
:10FFC0000922F3F799FDD4E710B500230446006831
:10FFD00086B0C4F8363063870379012B12D0022B28
:10FFE0000DD183680DF10B02DB074CBF3421B42126
:10FFF000FDF768F918B19DF90B30002B11DB0020DB
:020000040805ED
:1000000006B010BD8268417C02F0010290F910C078
:1000100001920DF10B02604600923422F3F76CFD61
:10002000E8E7092303AA24212068FFF70FFA002834
:10003000E5D09DF810209DF80F109DF813301204A4
:100040001B0442EA01629DF8121043EA01639DF825
:100050000C10C2F30F42C3F30F43228763879DF84E
:100060000D301B0443EA0163C3F30F43E38606B07C
:1000700010BD00BF70B5066882B00446F569002D5A
:100080005CD0002204233046FF212A700DEB0302CE
:10009000FFF7DCF910B9002002B070BD04236A46F6
:1000A000FF212068FFF7D2F90028F4D09DF8043032
:1000B0009B09023B012BEED9BDF8043043F6FF7CCF
:1000C000BDF806205BBABDF80010BDF80240C3F3CE
:1000D0000D066645DFD0002EDDD053BA40F2FF7E1C
:1000E000C3F34A1272451346D5D0002AD3D049BA79
:1000F000C1F30D0262451146CDD0002ACBD064BABF
:10010000C4F34A1272451446C5D0002AC3D0721AED
:10011000002AB8BF5242FF2ABDDC1A1B002AB8BF12
:100120005242FF2AB7DC23440E445B107610C5F818
:1001300001300123C5F805602B70ADE709211420BB
:10014000FAF798FFF061054626689AE770B50668E9
:1001500082B0F469F4B100210423304621700DEB24
:100160000302FF21FFF772F910B39DF804309B09D9
:1001700019D1BDF804200121BDF8063052BA217012
:100180005BBA92B2C3F34A13C4F80520C4F8013035
:1001900002B070BD054609211420FAF76BFFF0612B
:1001A00004462E68D7E7044A04210320FAF7EEFE3E
:1001B000002002B070BD00BF006F0C0870B506686B
:1001C00082B00546F469002C3ED03379221D012B04
:1001D0002DD0022B26D1B368304613F0010F4FF01B
:1001E0000C030CBF8C211946FFF7D2F8A070D8B1D0
:1001F000B4F9043007EE903AF8EEE77AC5ED077AE5
:10020000B4F9063007EE903AF8EEE77AC5ED087AD1
:10021000B4F9083007EE903AF8EEE77AC5ED097ABE
:1002200002B070BD0023A370002002B070BDB3689F
:10023000717C03F0010396F91000009201930C23E6
:100240001A46F3F759FCD1E709211420FAF712FFF7
:10025000F06104462E68B8E770B5066882B00546BE
:10026000F469002C3ED03379E21C012B2DD0022BF7
:1002700026D1B368304613F0010F4FF00D0314BFC1
:100280000C218C21FFF784F8A070D8B1B4F90A30A2
:1002900007EE903AF8EEE77AC5ED077AB4F90C303C
:1002A00007EE903AF8EEE77AC5ED087AB4F90E3029
:1002B00007EE903AF8EEE77AC5ED097A02B070BD24
:1002C0000023A370002002B070BDB368717C03F0FE
:1002D000010396F9100000920C2201930D23F3F70D
:1002E0000BFCD1E709211420FAF7C4FEF0610446A3
:1002F0002E68B8E7006810B5037984B00C46012B6E
:100300001AD0022B02D0002004B010BD836803AACB
:1003100013F0010F4FF0030314BF2221A221FFF7B6
:1003200037F80028EFD0BDF90D3003EB83031B1223
:10033000E633238004B010BD836803AA417C03F038
:10034000010390F910000092222201930323F3F796
:10035000D3FBE6E770B5066882B00546F469002C69
:100360003ED03379221D012B2DD0022B26D1B3682C
:10037000304613F0010F4FF00E0314BF3B21BB2199
:10038000FFF706F8A070D8B1A389DBBA07EE903A60
:10039000F8EEE77AC5ED077AE389DBBA07EE903A23
:1003A000F8EEE77AC5ED087A238ADBBA07EE903AD1
:1003B000F8EEE77AC5ED097A02B070BD0023A370AC
:1003C000002002B070BDB368717C03F0010396F9A0
:1003D000100000923B2201930E23F3F78DFBD1E72F
:1003E00009211420FAF746FE0446F061B9E700BF80
:1003F000006810B5037984B0012B10D0022B01D016
:1004000000200AE003AAF621FEF7C2FF0028F7D079
:10041000BDF80C30094A5BBA138004B010BD826885
:1004200003AC417C022302F0010290F91000CDE9F7
:100430000042F622F3F760FBE8E700BFD8FC002497
:10044000006810B5037984B0012B1DD0022B01D0B8
:10045000002017E0032303AAF621FEF799FF0028E6
:10046000F6D09DF80D309DF80CC01B020D499DF88B
:100470000E2043EA0C431343B1F92020C2F10802D5
:10048000D3404B6204B010BD826803AC417C0323AF
:1004900002F0010290F91000CDE90042F622F3F7D4
:1004A0002BFBDCE7D8FC0024006810B5037984B08E
:1004B000012B2DD0022B07D01C490020D1E9883216
:1004C0008A628B6404B010BD062302AAF721FEF7EE
:1004D0005FFF0028F0D09DF809309DF80C209DF8B2
:1004E00008C01B019DF80BE012019DF80A1043EAB9
:1004F0000C3342EA0E329DF80DC043EA11130B494A
:1005000042EA1C128B648A62C1E9883204B010BDD1
:10051000826802AC417C062302F0010290F91000CF
:10052000CDE90042F722F3F7E7FAD2E7D8FC00243E
:10053000006810B5037984B0012B1CD0022B0ED0BB
:100540009DF80D3001209DF80CC01B029DF80E1087
:10055000104A43EA0C430B43D36604B010BD8368D2
:1005600003AA13F0010F4FF0030314BF00218021F1
:10057000FEF70EFFE4E7826803AC417C032302F040
:10058000010290F91000CDE900420022F3F7B4FA1D
:10059000D6E700BFD8FC0024006810B5037984B00A
:1005A000012B1DD0022B0FD09DF80D3001209DF89E
:1005B0000CC01B029DF80E10104A43EA0C430B437B
:1005C000C2F8803004B010BD836803AA13F0010F95
:1005D0004FF0030314BF00218021FEF7D9FEE3E7AB
:1005E000826803AC417C032302F0010290F9100001
:1005F000CDE900420022F3F77FFAD5E7D8FC0024CA
:10060000006810B5037984B0012B28D0022B01D0EB
:10061000002022E0836803AA13F0010F4FF00303C8
:100620000CBF83211946FEF7B3FE0028F0D09DF8D9
:100630000C309DF90C109DF80D201B0400299DF82D
:100640000EC043EA02230D4AACBF00214FF07F41A8
:1006500043EA0C030B43C2F8543104B010BD826866
:1006600003AC0323417C02F0010290F91000CDE9B4
:1006700000421A46F3F740FAD7E700BFD8FC00243F
:10068000006810B5037984B0012B28D0022B01D06B
:10069000002022E0836803AA13F0010F4FF0030348
:1006A00014BF00218021FEF773FE0028F0D09DF8D2
:1006B0000C309DF90C109DF80D201B0400299DF8AD
:1006C0000EC043EA02230D4AACBF00214FF07F4128
:1006D00043EA0C030B43C2F8503104B010BD8268EA
:1006E00003AC417C032302F0010290F91000CDE934
:1006F00000420022F3F700FAD7E700BFD8FC00243D
:1007000010B50446006884B00379012B42D0022B57
:1007100007D0002213461046C4F83620638704B081
:1007200010BD836802AA13F0010F4FF0060314BF37
:1007300011219121FEF72CFE0028EAD0BDF90C30E2
:10074000B7EE086A07EE903ABDF9083006EE903A27
:10075000BDF90A30F8EEE77A07EE103AF8EEE66AED
:10076000B8EEC77A67EE867A66EE866A27EE067A74
:10077000FDEEE77AFDEEE66ABDEEC77A17EE903A37
:1007800016EE902A1BB2E28617EE102A63872287A4
:1007900004B010BD836802AA417C03F0010390F904
:1007A00010000092112201930623F3F7A5F9C3E785
:1007B00010B500230446006884B0C4F8363063875F
:1007C0000379012B22D0022B01D000201CE083688A
:1007D00002AA13F0010F4FF0060314BF0321832177
:1007E000FEF7D6FD0028F0D0BDF90A30BDF808109C
:1007F000BDF80C205B4201EB410102EB420203EB2E
:100800004303E1866287238704B010BD836802AA90
:10081000417C03F0010390F9100000920322019340
:100820000623F3F769F9DDE710B54FF0000C044635
:10083000006884B0C4F836C0A4F83AC00379012B2C
:1008400018D0022B01D0002012E0836802AA13F016
:10085000010F4FF0060314BF61468021FEF798FD9B
:100860000028F0D0029ABDF80C30C4F83620638717
:1008700004B010BD83686246417C03F0010390F927
:1008800010E0019302AB704600930623F3F734F9AE
:10089000E6E700BF10B5002384B004460068029369
:1008A000CDF80B300279012A1ED0022A19D18368B3
:1008B00002AA13F0010F4FF0070314BF4E21CE21FF
:1008C000FEF766FDBDF80910BDF80B20BDF80D3030
:1008D000C9BAD2BADBBA0120E1862287638704B0A5
:1008E00010BD1A461946F6E7826802AB90F910C0AF
:1008F00002F00102417C00936046019207234E22E0
:10090000F3F7FAF8DEE700BF006810B5037984B0AA
:10091000012B0BD0022B06D1012303AAFF21FEF7E6
:1009200037FD04B010BD002004B010BD826803ACD8
:10093000417C02F0010290F9100000940192FF2224
:10094000F3F7DAF804B010BD0368DA6B10B50446AB
:1009500082B012B1904740B123685B6B1BB1214656
:1009600001A8984718B9FF23E38202B010BDBDF873
:100970000630013B9BB2F7E7F0B50D4683B0044665
:10098000184616461F4661F053FE2844E673294672
:10099000A0732046256800243B46324600946C69CB
:1009A000A04703B0F0BD00BF38B58B6804460160B6
:1009B0000D46984700230B4A237522612B6B13B118
:1009C000204698472075084B93F828321BB1237DA9
:1009D00023F00103237500232046E382BDE838405D
:1009E000B2E700BF0001FF00D8FC0024144B30B573
:1009F0001C6885B084B12379012B10D0022B0BD158
:100A0000A1680246204611F0010118BF802105B0FF
:100A1000BDE83040FCF7B0BF002005B030BDA26893
:100A20000DF10F05617C8DF80F0094F9100002F0B4
:100A30000104802200950194F2F72EFE05B030BD2E
:100A4000AC770024F0B5274D85B02868002846D043
:100A5000B0228021FCF7EEFF286800283FD040221A
:100A60008021FCF7E7FF2868002838D00022802189
:100A7000FCF7E0FF286890B310228021FCF7DAFF32
:100A800028684FF4806400270DF10F0670B10379D8
:100A9000012B10D0022B09D183680022402113F0D2
:100AA000010304BF1A464021FCF766FF013CA4B2D3
:100AB0009CB12868EAE78268013C90F910E002F0F6
:100AC000010CA4B2417C402270468DF80F70CDE934
:100AD000006CF2F7E1FD002CEBD105B0F0BD002079
:100AE000CFE700BFAC77002410B50C4C2368A3B14E
:100AF000A0F1500280211846D2B2FCF79BFF20687B
:100B000058B100228021FCF795FF206828B11022FF
:100B10008021BDE81040FCF78DBF10BDAC770024EC
:100B2000A0F12003F0B503EB83031C4D1C4E85B0F0
:100B3000EC18053530681D4498B10379012B2278F3
:100B400016D0022B09D00134AC42F7D1002240214B
:100B500005B0BDE8F040FCF76DBF4021FCF70CFF8D
:100B600030680134AC42E7D10028EFD105B0F0BDC8
:100B70008168013490F910C001F00107417C8DF8C3
:100B80000F20604601970DF10F0740220097F2F702
:100B900083FDAC423068CFD1E6E700BF98D30B08A5
:100BA000AC770024F0B59B4D85B02868002800F094
:100BB0002E81D4228021FCF73DFF2868002800F018
:100BC000268180221146FCF735FF2868002800F0B6
:100BD0001E81A8228021FCF72DFF2868002800F044
:100BE00016813F228021FCF725FF2868002800F0AD
:100BF0000E81D3228021FCF71DFF2868002800F019
:100C0000068100228021FCF715FF2868002800F0EB
:100C1000FE8040228021FCF70DFF2868002800F0AC
:100C2000F6808D228021FCF705FF2868002800F05F
:100C3000EE8014228021FCF7FDFE2868002800F0D9
:100C4000E680A1228021FCF7F5FE2868002800F04C
:100C5000DE80C8228021FCF7EDFE2868002800F025
:100C6000D680DA228021FCF7E5FE2868002800F013
:100C7000CE8012228021FCF7DDFE2868002800F0DB
:100C8000C68081228021FCF7D5FE2868002800F06C
:100C9000BE80CF228021FCF7CDFE2868002800F01E
:100CA000B680D9228021FCF7C5FE2868002800F014
:100CB000AE80F1228021FCF7BDFE2868002800F0FC
:100CC000A680DB228021FCF7B5FE2868002800F012
:100CD0009E8040228021FCF7ADFE2868002800F0AD
:100CE0009680A4228021FCF7A5FE2868002800F049
:100CF0008E80A6228021FCF79DFE2868002800F047
:100D00008680AF228021FCF795FE286800287ED0DF
:100D1000A6228021FCF78EFE2868002877D0AE221C
:100D20008021FCF787FE2868002870D020228021CF
:100D3000FCF780FE2868002869D000228021FCF79B
:100D400079FE2868002862D0B0228021FCF772FE6C
:100D5000286800285BD040228021FCF76BFE2868C1
:100D6000002854D000228021FCF764FE2868002867
:100D70004DD010228021FCF75DFE28684FF480647E
:100D800000270DF10F0628B30379012B2BD0022B7E
:100D900004F1FF3215D094B2002CF6D181228021CB
:100DA000FCF748FE286848B1C8228021FCF742FEC3
:100DB000286818B1AF228021FCF73CFE012005B065
:100DC000F0BD8268402112F0010218BF0022FCF73A
:100DD000D3FD2868013CA4B2002CD4D10028DDD179
:100DE000012005B0F0BD8268013C90F910E002F0EE
:100DF000010CA4B2417C402270468DF80F70CDE901
:100E0000006CF2F749FC2868002CBCD1E6E7002012
:100E1000B4E700BFAC770024FCF72EBBFCF72CBB7B
:100E2000FCF72ABBFCF728BBFCF726BBFCF724BB6E
:100E3000FCF722BBD8B10E4B0E4A70B506680D46C2
:100E400082B0044633449B0A32F813005BF074FE10
:100E5000C5F381030022A1883046CDE90032C5F3F5
:100E6000411305F0130260F0C1FF02B070BD70477E
:100E70000000FEA758BF0B08D0B10E4BF0B50768B5
:100E800016460D4A0D463B4483B004469B0A32F891
:100E900013005BF051FEC5F38103A188384605F0CD
:100EA0001302CDE900366B0960F0A0FF03B0F0BD7E
:100EB000704700BF0000FEA758BF0B0810B504091B
:100EC000013C042C19D80F4A00F00F0332F814002B
:100ED00040FA03F212F0010211D0012202FA03F3E8
:100EE000013B18406AF056FC074B084A1B5D18444A
:100EF00000EB400002EB800010BD002010BD10464A
:100F000010BD00BF0CBF0B0868D10B08485C002463
:100F10002DE9F04F5422044600218BB0AA4869F015
:100F20007DFCAA4A611EE01C144611F8013F5D1EBB
:100F3000052D88BF0023884244F8043BF5D102F117
:100F40001003114651F8040B012800F02F818B4249
:100F5000F8D1114651F8040B022800F01D818B4294
:100F6000F8D1114651F8040B032800F00B818B4295
:100F7000F8D1114651F8040B042800F0F9808B4297
:100F8000F8D1114651F8040B052800F0E7808B4298
:100F9000F8D152F8041B062900F0D6809342F8D10C
:100FA0008B4F1A264FF0000ADFF81C8207F2BC456F
:100FB000DFF8209298F80C4054B32046FFF77EFFEC
:100FC00020B10523C6718371002303720321FFF74B
:100FD00031FF002302E001331C2B37D015F83320FA
:100FE000A242F8D107EBC303D3F8C0440123D9F8D8
:100FF000F4200621C8F81040D0189A4488F814202C
:10100000C9F8F40088F8161088F8153089F8F0301F
:10101000013608F10C08F6B2202ECBD1BAF1000F40
:1010200011D0DFF8C8A14FF0000BDFF8C4919AF897
:10103000EC306BB90BF1010B0AF1F40A09F58C796C
:10104000BBF1030FF3D10BB0BDE8F08F0024CDE767
:10105000BAF806004FF440365BF06EFDBAF80400B3
:101060005BF06AFDDAF8F0305A4CF421012BCAF833
:101070002830DAF8002001FB0B41D4BF0023012304
:101080000327CAF81020CAF81C300023CAF83830E9
:101090008AF82C30CAF83030CAF820308AF8483044
:1010A00004930823CAE905634FF48063CAF8343017
:1010B0004FF48073AAF824304FF48053CAE90F73B9
:1010C0008B6E002B7CD093689D0003D59168424BBA
:1010D0000B4093609368D80013D4404B9068196814
:1010E0003F4B034043F0805393603E4BB1FBF3F31F
:1010F0000493049B2BB1049B013B0493049B002BA2
:10110000F9D19368D9001CD4F4234FF0010803FBF4
:101110000B43996E41F010019966D96E41EA0801BE
:10112000D966F423916803FB0B4301F00401986E28
:1011300000F0100001435DD09A6E42F010029A66F2
:1011400078E74FF00008ECE7274B172193F8E821E8
:1011500083F8DC11013283F8E82121E722491424C5
:1011600091F8E80181F8D041013081F8E80110E7F9
:101170001D49342491F8E80181F8C441013081F817
:10118000E801FEE61849352491F8E80181F8B841F4
:10119000013081F8E801ECE61349312491F8E801C7
:1011A00081F8AC41013081F8E801DAE60E493024DB
:1011B00091F8E80181F8A041013081F8E801C8E622
:1011C000CB668AF860307EE76CFE00245CFE00246B
:1011D00080D10B080C1B0024C0FFFF5F000000241F
:1011E000C0FFFF6F400D0300D8FC0024101B00243B
:1011F000C0300030996E21F4817141F0020199668E
:101200009368DB0713D4784B9A4200F0078303F509
:1012100080739A4200F00283744B9B68DE0706D409
:1012200073498B6823F47C1343F440338B60714B18
:1012300071491B68D368194043F208030B43D3601C
:101240009168936801F0040103F00803194300F06A
:101250005382DAF81000DAF81C30012B00F04283D8
:10126000036B23F00F030363F42303FB0B439A6E1A
:1012700022F0030242F001029A66B8F1000F7FF4F7
:10128000D9AE9AF86020CDF81480012A3FF4D2AE8E
:101290008268012195078AF86010816802D4CA0724
:1012A00000F17A82F421554A554B01FB0B418D6EBA
:1012B0002A4042F002028A668268134043F00043EB
:1012C000836083684F4A002BC0F2E081F4204E4BCC
:1012D0004E4D4FF4005600FB0B404D490327826EE4
:1012E00022F0030242F001028266DAF80820CAF80E
:1012F0009C70AA4218BF9A424FF480650CBF01232C
:1013000000238A4208BF43F0010318318A4208BF14
:1013100043F0010318318A4208BF43F0010318313A
:101320008A4208BF43F0010318318A4208BF43F0E4
:10133000010318318A4208BF43F0010301F55671D9
:101340008A4208BF43F0010318318A4208BF43F0C4
:10135000010318318A4208BF43F0010318318A4261
:1013600008BF43F0010318318A4208BF43F001036C
:1013700018318A4208BF43F0010318318A4208BF7E
:1013800043F0010300218AF86010CAF89810CAE9F6
:101390001F11CAE92811DAF80C10CAF878104FF4B6
:1013A0000061CAE921514FF480711A4DCAE92361E5
:1013B0004FF400315646CAF89410296846F8742F45
:1013C0001BB9154B9A4240F092840020F4238AF80E
:1013D000A800022003FB0B4383F8AD00136823F041
:1013E000010313601FE000BF0020024000600258AC
:1013F000006302580010005C03C0F0FFFDEEFFFF29
:10140000C0FFFE3F00F8C325100002402800024044
:1014100040000240A02B0024B80402402B685B1A55
:10142000052B00F2AF811368DB07F7D41368304651
:10143000A0491940A04B0B431360536923F00703E5
:101440005361F0F71DFEDAF8D03003F01F013F239F
:101450008B408360DAF87420984B9949994F8A42FF
:1014600018BF9A4201F11801A2EB070C0CBF01232F
:1014700000238A4208BF43F0010318318A4208BFA3
:1014800043F0010318318A4208BF43F001031831C9
:101490008A4208BF43F0010318318A4208BF43F073
:1014A000010318318A4208BF43F0010301F5567168
:1014B0008A4208BF43F0010318318A4208BF43F053
:1014C000010318318A4208BF43F0010318318A42F0
:1014D00008BF43F0010318318A4208BF43F00103FB
:1014E00018318A4208BF43F0010318318A4208BF0D
:1014F00043F00103DCF1000701F1180147EB0C0791
:101500008A4208BF43F001036F49501A14313B432C
:10151000D0F1000EA2EB010C4EEB000EDCF100014D
:101520004EEA030341EB0C010B4301916749501A4A
:101530004142414166480B4302916649A2EB010CCE
:10154000DCF1000141EB0C010B430091111A484200
:1015500048416149A2EB010C0343DCF1000141EB7E
:101560000C01DFF88CC1624514BF4FF0000C4FF046
:10157000010C0B4302D1BCF1000F3ED047EA0E072D
:10158000019B3B43029F1F433B46009F1F43D3B237
:10159000384301435CEA010100F024831422083B34
:1015A0000127DFF850C1B3FBF2F34C4A9F401A44C5
:1015B0009200DAF87C30CAF8DC70802BCAE9352C4E
:1015C00000F00281DAF87830D8B2013B072B1060C6
:1015D000CCF8047000F2FE80471E002900F08283E0
:1015E0003F4B404903449B0001220020BA40CAE916
:1015F0003831CAF8E82018604A60F423012200213B
:10160000009503FB0B439646C3F8CC1083F8AD203E
:101610000AF110034FFA8BF2CAF85C60CAF8AC30DA
:101620009446314B06E00EF1010E0C33BEF1070F6C
:1016300000F0FE805A7D002AF5D093F90D20624516
:10164000F1D100229D7D19690692284A019502EB8D
:101650008802D2F89C059AF86020012A3FF4EAAC8F
:101660004FF001028AF86020DAF8102095686D07C3
:1016700040F10481F42303FB0B439A6E42F02002F5
:101680009A664FF000038AF86030D3E4059B01337B
:101690000593059B9342FFF414AEF422002102FB54
:1016A0000B42936E23F0120343F0100393668AF803
:1016B0006010BFE43F8010FE002D020010000240C9
:1016C00028000240085402581C540258445402583E
:1016D0006C54025858540258805402580096001610
:1016E0003F960016405902586CFE002480D10B082A
:1016F0009454025880580258D068A94B0340DAF835
:10170000440043F00303D360136923F00103136122
:10171000136923F0704303431361A24B9A4275D0BF
:1017200003F580739A4271D09F4B9B6813F4403F3E
:1017300014BF01230023002B00F0E580F0F744FDE7
:10174000DAF814300146B3F5003F00F00082B3F53B
:10175000403F00F00082B3F5803F00F0F881934BEA
:10176000DAF810001A6841F20303B3EB124FC0F02D
:10177000C2808F4B9942836800F20D8123F48073FD
